:1000000068780120BD5A00001F4E0700A95A000061
:10001000A95A0000A95A0000A95A0000A95A0000D4
:10002000000000000000000000000000F55A000081
:10003000A95A000000000000415D0000A95A00001C
:10004000015E0000015E0000015E0000015E000034
:10005000015E0000015E0000015E0000015E000024
:10006000015E0000015E0000015E0000015E000014
:10007000015E0000015E0000015E0000015E000004
:10026000015E0000015E0000A96D0200015E000059
:10027000015E0000015E0000015E0000015E000002
:10028000015E0000015E0000015E0000015E0000F2
:10029000015E0000015E0000015E0000015E0000E2
:1002A000015E0000015E0000015E0000015E0000D2
:1004C80081F0004102E000BF83F0004330B54FEAFD
:1004D80041044FEA430594EA050F08BF90EA020F6A
:1004E8001FBF54EA000C55EA020C7FEA645C7FEAFD
:1004F800655C00F0E2804FEA5454D4EB5555B8BF20
:100508006D420CDD2C4480EA020281EA030382EA90
:10051800000083EA010180EA020281EA0303362D22
:1005280088BF30BD11F0004F4FEA01314FF4801CF5
:100538004CEA113102D0404261EB410113F0004F07
:100548004FEA03334CEA133302D0524263EB4303BE
:1005580094EA050F00F0A780A4F10104D5F1200E5C
:100568000DDB02FA0EFC22FA05F2801841F10001B7
:1005780003FA0EF2801843FA05F359410EE0A5F18B
:1005880020050EF1200E012A03FA0EFC28BF4CF0BC
:10059800020C43FA05F3C01851EBE37101F0004572
:1005A80007D54FF0000EDCF1000C7EEB00006EEB7F
:1005B8000101B1F5801F1BD3B1F5001F0CD3490809
:1005C8005FEA30004FEA3C0C04F101044FEA445260
:1005D80012F5800F80F09A80BCF1004F08BF5FEAE7
:1005E800500C50F1000041EB045141EA050130BDC7
:1005F8005FEA4C0C404141EB0101013C28BFB1F5D9
:10060800801FE9D291F0000F04BF01460020B1FA23
:1006180081F308BF2033A3F10B03B3F120020CDAF6
:100628000C3208DD02F1140CC2F10C0201FA0CF0D4
:1006380021FA02F10CE002F11402D8BFC2F1200C39
:1006480001FA02F120FA0CFCDCBF41EA0C019040EF
:10065800E41AA2BF01EB0451294330BD6FEA040438
:100668001F3C1CDA0C340EDC04F11404C4F1200223
:1006780020FA04F001FA02F340EA030021FA04F335
:1006880045EA030130BDC4F10C04C4F1200220FA8C
:1006980002F001FA04F340EA0300294630BD21FACA
:1006A80004F0294630BD94F0000F83F4801306BF90
:1006B80081F480110134013D4EE77FEA645C18BF84
:1006C8007FEA655C29D094EA050F08BF90EA020F1B
:1006D80005D054EA000C04BF1946104630BD91EA13
:1006E800030F1EBF0021002030BD5FEA545C05D116
:1006F8004000494128BF41F0004130BD14F5800455
:100708003CBF01F5801130BD01F0004545F0FE41C8
:1007180041F470014FF0000030BD7FEA645C1ABFFD
:10072800194610467FEA655C1CBF0B46024650EA34
:10073800013406BF52EA033591EA030F41F4002160
:1007480030BD00BF90F0000F04BF0021704730B5E6
:100758004FF4806404F132044FF000054FF00001BB
:1007680050E700BF90F0000F04BF0021704730B57C
:100778004FF4806404F1320410F0004548BF404251
:100788004FF000013EE700BF42004FEAE2014FEAA6
:1007980031014FEA02701FBF12F07F4393F07F4F81
:1007A80081F06051704732F07F4208BF704793F084
:1007B8007F4F04BF41F40021704730B54FF4607497
:1007C80001F0004521F000411CE700BF50EA01029A
:1007D80008BF704730B54FF000050AE050EA010243
:1007E80008BF704730B511F0004502D5404261EBB3
:1007F80041014FF4806404F132045FEA915C3FF4F4
:10080800D8AE4FF003025FEADC0C18BF03325FEA90
:10081800DC0C18BF033202EBDC02C2F1200300FA41
:1008280003FC20FA02F001FA03FE40EA0E0021FA66
:1008380002F11444BDE600BF70B54FF0FF0C4CF454
:10084800E06C1CEA11541DBF1CEA135594EA0C0F06
:1008580095EA0C0F00F0DEF82C4481EA030621EA41
:100868004C5123EA4C5350EA013518BF52EA03357C
:1008780041F4801143F4801338D0A0FB02CE4FF02E
:100888000005E1FB02E506F00042E0FB03E54FF05E
:100898000006E1FB03569CF0000F18BF4EF0010E56
:1008A800A4F1FF04B6F5007F64F5407404D25FEA52
:1008B8004E0E6D4146EB060642EAC62141EA555105
:1008C8004FEAC52040EA5E504FEACE2EB4F1FD0C47
:1008D80088BFBCF5E06F1ED8BEF1004F08BF5FEAC5
:1008E800500E50F1000041EB045170BD06F0004677
:1008F80046EA010140EA020081EA0301B4EB5C0424
:10090800C2BFD4EB0C0541EA045170BD41F480111B
:100918004FF0000E013C00F3AB8014F1360FDEBF40
:10092800002001F0004170BDC4F10004203C35DA1C
:100938000C341BDC04F11404C4F1200500FA05F39F
:1009480020FA04F001FA05F240EA020001F0004240
:1009580021F0004110EBD37021FA04F642EB0601B6
:100968005EEA430E08BF20EAD37070BDC4F10C04E0
:10097800C4F1200500FA04F320FA05F001FA04F2A4
:1009880040EA020001F0004110EBD37041F1000190
:100998005EEA430E08BF20EAD37070BDC4F120059B
:1009A80000FA05F24EEA020E20FA04F301FA05F203
:1009B80043EA020321FA04F001F0004121FA04F2AB
:1009C80020EA020000EBD3705EEA430E08BF20EA7B
:1009D800D37070BD94F0000F0FD101F000464000B5
:1009E80041EB010111F4801F08BF013CF7D041EA37
:1009F800060195F0000F18BF704703F0004652003B
:100A080043EB030313F4801F08BF013DF7D043EA0B
:100A18000603704794EA0C0F0CEA135518BF95EAC1
:100A28000C0F0CD050EA410618BF52EA4306D1D148
:100A380081EA030101F000414FF0000070BD50EA67
:100A4800410606BF1046194652EA430619D094EAF1
:100A58000C0F02D150EA013613D195EA0C0F05D1DB
:100A680052EA03361CBF104619460AD181EA03012F
:100A780001F0004141F0FE4141F470014FF00000E7
:100A880070BD41F0FE4141F4780170BD70B54FF082
:100A9800FF0C4CF4E06C1CEA11541DBF1CEA135502
:100AA80094EA0C0F95EA0C0F00F0A7F8A4EB0504E4
:100AB80081EA030E52EA03354FEA013100F08880DB
:100AC8004FEA03334FF0805545EA131343EA1263A4
:100AD8004FEA022245EA111545EA10654FEA002659
:100AE8000EF000419D4208BF964244F1FD0404F512
:100AF800407402D25B084FEA3202B61A65EB03056E
:100B08005B084FEA32024FF480104FF4002CB6EB2A
:100B1800020E75EB030E22BFB61A754640EA0C00AA
:100B28005B084FEA3202B6EB020E75EB030E22BFEA
:100B3800B61A754640EA5C005B084FEA3202B6EB2B
:100B4800020E75EB030E22BFB61A754640EA9C00EA
:100B58005B084FEA3202B6EB020E75EB030E22BFBA
:100B6800B61A754640EADC0055EA060E18D04FEA78
:100B7800051545EA16754FEA06164FEAC30343EA18
:100B880052734FEAC2025FEA1C1CC0D111F4801FE5
:100B98000BD141EA00014FF000004FF0004CB6E7DE
:100BA80011F4801F04BF01430020B4F1FD0C88BF7D
:100BB800BCF5E06F3FF6AFAEB5EB030C04BFB6EB88
:100BC800020C5FEA500C50F1000041EB045170BD7B
:100BD8000EF0004E4EEA113114EB5C04C2BFD4EBA8
:100BE8000C0541EA045170BD41F480114FF0000E2C
:100BF800013C90E645EA060E8DE60CEA135594EAA8
:100C08000C0F08BF95EA0C0F3FF43BAF94EA0C0FAA
:100C18000AD150EA01347FF434AF95EA0C0F7FF41F
:100C280025AF104619462CE795EA0C0F06D152EA73
:100C380003353FF4FDAE1046194622E750EA410657
:100C480018BF52EA43067FF4C5AE50EA41047FF468
:100C58000DAF52EA43057FF4EBAE12E74FF0FF3CCD
:100C680006E000BF4FF0010C02E000BF4FF0010C9E
:100C78004DF804CD4FEA410C7FEA6C5C4FEA430C17
:100C880018BF7FEA6C5C1BD001B050EA410C0CBF66
:100C980052EA430C91EA030F02BF90EA020F0020C8
:100CA800704710F1000F91EA030F58BF994208BF2F
:100CB80090422CBFD8176FEAE37040F001007047EC
:100CC8004FEA410C7FEA6C5C02D150EA013C07D143
:100CD8004FEA430C7FEA6C5CD6D152EA033CD3D08E
:100CE8005DF8040B704700BF8446104662468C4688
:100CF8001946634600E000BF01B5FFF7B7FF0028BB
:100D080048BF10F1000F01BD4DF808EDFFF7F4FFE3
:100D18000CBF012000205DF808FB00BF4DF808ED6E
:100D2800FFF7EAFF34BF012000205DF808FB00BF91
:100D38004DF808EDFFF7E0FF94BF012000205DF8B3
:100D480008FB00BF4DF808EDFFF7CEFF94BF012068
:100D580000205DF808FB00BF4DF808EDFFF7C4FF61
:100D680034BF012000205DF808FB00BF4FEA4102B4
:100D780012F5001215D211D56FF47873B3EB6252E5
:100D880012D94FEAC12343F0004343EA505311F00C
:100D9800004F23FA02F018BF404270474FF000009E
:100DA800704750EA013005D111F0004008BF6FF0DC
:100DB800004070474FF00000704700BF4FEA410203
:100DC800B2F1E04324BFB3F5001CDCF1FE5C0DD9A1
:100DD80001F0004C4FEAC0024CEA5070B2F1004FEB
:100DE80040EB830008BF20F00100704711F0804FEE
:100DF80021D113F13872BCBF01F00040704741F4B3
:100E080080114FEA5252C2F11802C2F1200C10FAB6
:100E18000CF320FA02F018BF40F001004FEAC1239A
:100E28004FEAD32303FA0CFC40EA0C0023FA02F33E
:100E38004FEA4303CCE77FEA625307D150EA013314
:100E48001EBF4FF0FE4040F44000704701F00040E4
:100E580040F0FE4040F40000704700BF80F00040C2
:100E680002E000BF81F0004142001FBF5FEA41037A
:100E780092EA030F7FEA226C7FEA236C6AD04FEA7A
:100E88001262D2EB1363C1BFD218414048404140BF
:100E9800B8BF5B42192B88BF704710F0004F40F471
:100EA800000020F07F4018BF404211F0004F41F48D
:100EB800000121F07F4118BF494292EA030F3FD059
:100EC800A2F1010241FA03FC10EB0C00C3F120036C
:100ED80001FA03F100F0004302D5494260EB4000FB
:100EE800B0F5000F13D3B0F1807F06D340084FEA66
:100EF800310102F10102FE2A51D2B1F1004F40EB5B
:100F0800C25008BF20F0010040EA030070474900C2
:100F180040EB0000013A28BFB0F5000FEDD2B0FA5F
:100F280080FCACF1080CB2EB0C0200FA0CF0AABF82
:100F380000EBC25052421843BCBFD0401843704720
:100F480092F0000F81F4000106BF80F40000013226
:100F5800013BB5E74FEA41037FEA226C18BF7FEAFD
:100F6800236C21D092EA030F04D092F0000F08BF3F
:100F78000846704790EA010F1CBF0020704712F026
:100F88007F4F04D1400028BF40F00040704712F165
:100F980000723CBF00F50000704700F0004343F0CA
:100FA800FE4040F4000070477FEA226216BF084600
:100FB8007FEA23630146420206BF5FEA412390EAC3
:100FC800010F40F4800070474FF0000304E000BFB9
:100FD80010F0004348BF40425FEA000C08BF70476A
:100FE80043F0964301464FF000001CE050EA01022E
:100FF80008BF70474FF000030AE000BF50EA010243
:1010080008BF704711F0004302D5404261EB41012F
:101018005FEA010C02BF84460146002043F0B64354
:1010280008BFA3F18053A3F50003BCFA8CF2083A79
:10103800A3EBC25310DB01FA02FC634400FA02FC82
:10104800C2F12002BCF1004F20FA02F243EB020089
:1010580008BF20F00100704702F1200201FA02FCEB
:10106800C2F1200250EA4C0021FA02F243EB0200DE
:1010780008BF20EADC7070477BB972B90029BEBF8F
:1010880000204FF0004106E008BF00281CBF6FF0A9
:1010980000414FF0FF3000F077B8ADF1080C6DE972
:1010A80004CE002909DB002B1ADB00F0A9F8DDF8D3
:1010B80004E0DDE9022304B07047404261EB4101DE
:1010C800002B1BDB00F09CF8DDF804E0DDE90223CF
:1010D80004B0404261EB4101524263EB4303704765
:1010E800524263EB430300F08BF8DDF804E0DDE9DE
:1010F800022304B0404261EB41017047524263EB66
:10110800430300F07DF8DDF804E0DDE9022304B0D4
:10111800524263EB4303704753B94AB9002908BFE9
:1011280000281CBF4FF0FF314FF0FF3000F02CB803
:10113800ADF1080C6DE904CE00F062F8DDF804E0CA
:10114800DDE9022304B07047D0B5FFF71DFB00228C
:101158000B4B06460F46FFF76FFB00F017F80446E7
:10116800FFF7F0FA0022074BFFF766FB02460B4633
:1011780030463946FFF7A8F900F008F82146D0BDF7
:101188000000F03D0000F041704700BF4A0011D256
:1011980012F5001211D20DD56FF47873B3EB6252C9
:1011A8000ED44FEAC12343F0004343EA505323FAD5
:1011B80002F070474FF00000704750EA013002D14A
:1011C8004FF0FF3070474FF00000704710F8012BC8
:1011D80011F8013B012A28BF9A42F7D0D01A70476C
:1011E800034611F8012B03F8012B002AF9D17047A7
:1011F800034613F8012B002AFBD1181A013870474F
:101208002DE9F0478C468E46089E15460446194639
:10121800002B40F0D080724547D9B2FA82F74FB11F
:10122800C7F120030EFA07FCBD40BC4020FA03F3C7
:1012380043EA0C0C4FEA154EA8B2230CBCFBFEF88F
:101248000EFB18CC08FB00F943EA0C43994528D952
:10125800EB1808F1FF3204D2994502D9A8F102022D
:101268002B44A3EB0903A4B2B3FBFEFC0EFB1C3317
:101278000CFB00F044EA0344A04214D92C190CF1E9
:10128800FF3304D2A04202D9ACF102032C44241A41
:1012980043EA02401EB1FC40002334607360BDE89D
:1012A800F0874246DDE76346F1E7002A79D0B2FAD3
:1012B80082F3002B3FD01946C1F1200302FA01F551
:1012C80000FA01F42EFA03F20EFA01FE20FA03F3F3
:1012D800AFB243EA0E034FEA154EB2FBFEFC0EFB1B
:1012E8001C201A0C0CFB07F842EA004290455AD918
:1012F800AA180CF1FF3004D2904502D9ACF10200D3
:101308002A44A2EB08029BB2B2FBFEFC0EFB1C2295
:101318000CFB07F743EA02439F4246D9EB180CF14E
:10132800FF3204D29F4202D9ACF102022B44DB1BEC
:1013380042EA004202E0AEEB020301224FEA154EF8
:10134800AFB2200CB3FBFEFC0EFB1C330CFB07F802
:1013580040EA034398452AD9EB180CF1FF3004D230
:10136800984502D9ACF102002B44A3EB0803A4B2C0
:10137800B3FBFEFC0EFB1C330CFB07F744EA0344EB
:10138800A74216D92C190CF1FF3304D2A74202D96F
:10139800ACF102032C44E41B43EA00400F4611461B
:1013A80078E71F2188E76046ABE76246BFE76046FB
:1013B800DBE76346EFE7734506D916B9002108460F
:1013C8006DE7C6E9000EF9E7B3FA83F787B9734505
:1013D80001D3824207D8841A6EEB030301209C468E
:1013E8001EB900215BE73846FAE7C6E9004CF8E782
:1013F800C7F1200CBB4000FA07F422FA0CF520FADA
:101408000CF1BA401D432EFA0CF30EFA07FE4FEA10
:10141800154941EA0E011FFA85FEB3FBF9F809FBED
:1014280018300B0C08FB0EFA43EA00439A4540D9E2
:10143800EB1808F1FF3004D29A4502D9A8F102004E
:101448002B44A3EB0A0389B2B3FBF9F809FB183361
:1014580008FB0EFE41EA03418E452CD9691808F1B4
:10146800FF3304D28E4502D9A8F10203294443EA86
:101478000040A1EB0E01A0FB02984145CE46434631
:1014880002D306D14C4504D20138B9EB020E68EB01
:101498000503002EA5D0B4EB0E0261EB030101FA9F
:1014A8000CFC22FA07F3F9404CEA0303C6E90031C1
:1014B80097E74046C5E74346D9E70000000000002B
:1014C8000022F0B5114640F6034085B009F008FA4D
:1014D8000446002856D108F07BFC214641F203005F
:1014E80003AA09F0FDF9044600284BD1039A274DB9
:1014F800D16805F12C03D1F80100D1F8051003C318
:10150800104605F041F8214641F2010003AA09F00E
:10151800E7F90446002835D10398C3685A7885F856
:1015280023205A88EA841A7985F82420B3F80720FA
:101538002A85B3F805306B8505F026F8214641F277
:10154800020003AA09F0CCF90446D8B9039F05F1B3
:101558003406FA68531C413234461868596808330F
:1015680003C493422646F7D1384605F00DF895F89E
:101578003030580610D40121054A064875F0B0F8F5
:101588006FF01204204605B0F0BD00BF80010020B6
:101598005A780A0090870900002142F2030003AA42
:1015A80009F09EF904460028ECD1039AC04BD16893
:1015B800D1F80100D1F8051003C3104604F0E4FF88
:1015C800214642F2020003AA09F08AF904460028DB
:1015D800D8D1039EF468B4F801309AB292B1E27897
:1015E80082B1A5F8BC30E378032B06D00322022190
:1015F8000092B048B04A73F00DF9E278AF4811464E
:101608007AF06DFC304604F0BFFF002142F23A0048
:1016180003AA09F065F90446002840F020810398E0
:10162800C368B3F80130A5F8D83004F0ADFF95F8D9
:10163800306016F0200619D14FF0FF304FF0FF311F
:1016480008F07CFF0446002800F0768102210C3067
:1016580073F0EEFC0123214603704670324640F6D3
:101668006D4009F03DF9044600288BD195F85030BB
:101678001A0713D5002142F21C0003AA09F030F919
:10168800044600287FF47EAF0398C368D3F801208E
:10169800D3F80530C5E9262304F076FF95F8903095
:1016A8009B0626D50DF10A0102A809F0C3F90446E4
:1016B80000287FF467AF4FF0FF304FF0FF3108F09C
:1016C8003DFF0646002800F0378104210C3073F0F6
:1016D800AFFCBDF8083022460380BDF80A30314619
:1016E800438042F2240009F0FBF8044600287FF406
:1016F80049AF95F890305F0610D5002142F22A00D4
:1017080003AA09F0EDF8044600287FF43BAF0398DC
:10171800C3685B7885F8DA3004F036FF4FF0FF30A5
:101728004FF0FF3108F00AFF0446002800F004815A
:1017380008210C3073F07CFC95F890100246604844
:1017480011F0020F5F4B08BF034695F891008E0613
:1017580048BF43F0400310F0090F18BF43F400637B
:1017680001F0010143EA0110002174F0DDFF214678
:10177800002242F2010009F0B3F8044600287FF481
:1017880001AF95F83030B5F8BC10980673D4C9B9D4
:1017980041F2050003AA09F0A3F8044600287FF4E3
:1017A800F1AEB5F8BC30039C4BB9E368B3F801203F
:1017B800A5F8BC209A88414811467AF090FB20464B
:1017C80004F0E2FE4FF0FF304FF0FF3108F0B6FEB4
:1017D8000446002800F0B08008210C3073F028FC83
:1017E80095F890300246D90747BF2FA1D1E90001EB
:1017F8004FF00051344874F097FF2146002240F61C
:10180800014009F06DF8044600287FF4BBAE01469C
:1018180003AA4FF6014009F063F80446002834D0C3
:101828002A4A0221234874F05BFFEB79002B74D11C
:1018380075F013FA044600287FF4A4AE0CF076FF86
:10184800044600287FF49EAEEB79002B3FF49AAE55
:1018580008211F4874F04DFF08F074FF92E6411DFF
:101868007FF490AE02211B4A124874F039FF1F23FF
:10187800A5F8D830DBE60029A4D10121164A0D4885
:1018880074F02EFF6FF004047CE6039804F07CFEED
:1018980021464FF6024003AA09F022F80446F8B19F
:1018A8000E4ABEE7AFF30080908800020080002057
:1018B80010020020908709007E780A00400200206C
:1018C8000E1207002E1207001088000244790A0041
:1018D80008020020C4780A0021790A0068790A0001
:1018E8000398C368B3F80130A5F8753004F04CFECE
:1018F80095F875305A0798D521464FF6034003AA44
:1019080008F0EEFF08B11A4A8BE70398C3685B78C2
:1019180085F8743004F038FE87E72E78002E87D1DA
:1019280095F875309B061FD54FF0FF304FF0FF310B
:1019380008F004FE044610B96FF0680422E6062198
:101948000C3073F075FBD5F8013021460360094B64
:1019580032469B8883804FF6064008F0C1FF044654
:1019680000283FF465AF0DE66FF085040AE600BF76
:1019780091790A00810100204FF0FF329FED0A7B28
:101988000D4B00211A6000200C4B002283ED007BD8
:101998009FED077B0A4BC3E900010A490A4B81ED19
:1019A800007B1A6016F092BCFFFFFFFFFF1F0000CC
:1019B8001F00000000000000348A002000030020FF
:1019C80000410020F80200202C8A002000000000BE
:1019D8002DE9F047044640F2712690F8623090F8FD
:1019E800382023F00103C3F3800060F386128CB023
:1019F80004F1460184F8623084F8382015F0EAF9D9
:101A0800B4F84C300022A3FB0663A36D484D236550
:101A180003F5D673B34228BF33464649A4EB050500
:101A2800A1FB051594F83810C5F3471501F07901A5
:101A3800DFF81091C4E90222227032BF6360666049
:101A4800226584F8381005EB4502246149F82230F4
:101A580015F01AF963694FEA450A00F5D677002BA5
:101A68004BD00DF12C089121AA4409EB8A034FF0C1
:101A780000094FF0020A0993CDF820800694B4F8C3
:101A88004C302D4A2D480792A3FB000201FB03218D
:101A98002B4BCDF80C9005936368CDF82CA00493DC
:101AA80021A3D3E90023FFF737FB104619464FF46B
:101AB8007A720023FFF730FB0535EDB20321CDE93B
:101AC80001603B462A464846CDF8009014F062FF74
:101AD800414615F091FF60B994F8623043EA0A0371
:101AE80084F8623019F0E4FEB8B100200CB0BDE80B
:101AF800F0870C200CB0BDE8F0870DF12C08CDE97B
:101B08000A330320434661680AAA23F015FE002819
:101B1800A9D1DDE90A371F44A5E7504624F038FC6F
:101B2800E3E700BFAFF3008000CA9A3B0000000063
:101B3800A08D00201F85EB51556E0100002AE78417
:101B48005DDB0100948D002070B50D46044600F160
:101B58008F06334600223B3105F12B002BF05EF94E
:101B680000229FED2D7BD4F89B30D4F89710C4F851
:101B7800BC30D4F8AC30D4F89300C4F8CD3094F825
:101B8800C830D4F88FC043F0010384F8C83094F803
:101B9800A730C4F8B810D4F8A81062F30003C4F84A
:101BA800B400C4F8C9102046294684ED307BC4F837
:101BB800B0C084F89F2084F8A02084F8A12084F87D
:101BC800A22084F8A32084F8A42084F8A52084F80F
:101BD800A62084F8A7301FF091FD0646B8B1301D45
:101BE80021F090F9F37931466B7320461FF09CFD84
:101BF800204620F09BFE40F206636B8194F88E30FD
:101C080023F0180343F0180384F88E3070BD00DE0B
:101C1800E5E700BFAFF3008000000000000000000F
:101C280070B504460D461FF061FD10B90623AB726E
:101C380070BD04F18F063346002205F13B0105F122
:101C48002B002BF0EBF800229FED2B7BD4F89B3078
:101C5800D4F89710C4F8BC30D4F8AC30D4F893005A
:101C6800C4F8CD3094F8C830D4F88FC062F30003BC
:101C780084F8C83094F8A730C4F8B810D4F8A8107D
:101C880043F00103C4F8B400C4F8C910204629463B
:101C980084ED307BC4F8B0C084F89F2084F8A0207D
:101CA80084F8A12084F8A22084F8A32084F8A42032
:101CB80084F8A52084F8A62084F8A7301FF01EFD1C
:101CC8000646A8B1301D21F013F9F37931466B733C
:101CD80020461FF029FD204622F0FCFA4FF4C1638C
:101CE8006B8194F88E3043F0080384F88E3070BD11
:101CF80000DEE7E7AFF3008000000000000000000E
:101D08002DE9F04F03699146D3F8A460436891F830
:101D18002000D3F800B000F07F0440B20028B8BF1C
:101D2800A2464FF0010396F8C623A9BF04F158074D
:101D380004F1480704F1100A0BEB4717B8BF0BEB87
:101D4800471712F0100288463D6803FA0AF185B079
:101D580006F1F40334D0A4000028344417DBD4F887
:101D68003C2222F00042B9F1000F0DD042F40012DB
:101D7800C4F83C22184677F05BFE0021404605B0C7
:101D8800BDE8F04F77F087BA42F00062F0E7D4F888
:101D98007C2122F00042B9F1000F0ED142F000621E
:101DA8000120C4F87C21C2F3835200FA02F2B6F88B
:101DB8009E030243A6F89E23DCE742F00262EFE7A7
:101DC8009FED377B18468DED007B039102937AF0E7
:101DD8008AFCDDE90231D8B1B9F1000F02D045F42F
:101DE80000153D6001224FEA5A130AF01F0A02FA51
:101DF8000AF2D24306EB830303F58073D3E8EF0FAF
:101E08001040C3E8E10F0029F8D105B0BDE8F08F14
:101E180098F92020002A32DBEFF31180202282F388
:101E28001288BFF36F8F0122A240B6F8984392B28E
:101E38001443A6F89843B9F1000F04D0B6F89A43B2
:101E48002243A6F89A23DBF8042842F40072CBF860
:101E5800042880F31188BFF36F8F40F635440025BE
:101E680000221846CDE900457AF03DFC002884D1CF
:101E780098F820200C490D4877F076FD7DE7B9F1F8
:101E8800000F09D145F00065AA0303D5002DB8BF9E
:101E980045F080453D60E0E745F00265F4E700BFA6
:101EA80000000000000000009E980A00B8880900A1
:101EB8002DE9F04F984685B000F15803C0E9163374
:101EC800129B0026838104239FED257B073222F095
:101ED800070A0374119B01EB0A090F4680ED087B82
:101EE8004946C0E9066686608373C6730446DDF812
:101EF80038B003F08BFB109BC51D25F00705C4F80F
:101F08008850C4E9207A02930F9BA9EB0505CDE917
:101F180000B32A4643463946204603F071FE0F9B1C
:101F2800C4E91B8B6367109B6665A367EFF3118297
:101F3800202383F31288BFF36F8F0B4B596A5C62BF
:101F4800E16782F31188BFF36F8F9B680BB1D3F8F9
:101F58008C302846C4F88C3005B0BDE8F08F00BF3F
:101F6800000000000000000048A900200000000058
:101F78001FB513A3D3E90023FFF77EF801A951F099
:101F880005FE9DF807309DF806201B0443EA4253DE
:101F98009DF80820BDF8040043EAC2239DF80920F3
:101FA800A0F2BC7043EA42139DF80A2043EA5203A8
:101FB80043EA406005B05DF804FB00BFAFF3008062
:101FC80000CA9A3B000000002DE9F04F93B0A94ADF
:101FD80004AF1378002B30D10123A74DA74C137001
:101FE80029682A68A648C2F5806221447BF0CCFCA7
:101FF8007860F8B1022034F07DFD2B687A68267885
:1020080013442B609F4B187801281AD9320718D02F
:10201800B04216D0042387F82530002387F824001F
:1020280002229748009307F1240138F017FA02209A
:1020380034F068FD00238F4A13703C37BD46BDE875
:10204800F08F302E00F02D8227D8202E00F022812C
:1020580008D8102E3ED0122E00F0BB80012840F088
:10206800E580D0E1222EF9D140F22113BB84A36888
:102078002A68B3F57D7FC0F0CB81022387F825302D
:1020880000231422009307F124017D4838F0E6F973
:102098007D4B18687AF059FC30E0502E00F04C82E5
:1020A800602E00F04F82402ED8D140F24113BB84FD
:1020B80063882968B3F57C7FC0F01082022387F813
:1020C800253000231022009307F124016C4838F0D2
:1020D800C5F913E040F21113BB826388EB46B3F5F0
:1020E8007C7F29680FD302237B7500231022644864
:1020F800009307F1140138F0B1F9DD460023614A75
:102108002B601370DEE003F10C029142C0F03B82B9
:1021180000225E495D48CA5407F10C017AF0FCFBC5
:10212800DFF86481C8F800000028DCD034F026F914
:102138000028D8D0564B002202930023CDE9002373
:10214800F9680122D8F800007AF02CFC0028CAD1DE
:102158004F487AF0A0FCD4E90183A0EB080999451F
:1021680028BF99460023C7E90680C7F820901022A7
:10217800009307F114018246414838F06FF941464F
:1021880043487AF07FFCC144C14505D8C24519D8F7
:102198003F487AF041FCB0E7A9EB0802102A28BFB3
:1021A800102207F1100307F1240139487AF04AFC9C
:1021B80000233A6907F1240100933148904438F02C
:1021C8004DF9E1E71223DD462E4A137000232B60F8
:1021D80019E12B6840F211132D48BB827AF05BFCA1
:1021E8006368A268A0EB0309914528BF91464FF0A8
:1021F8000008C7E90630C7F8209007F114018246A5
:10220800434610221E48CDF8008038F027F961684F
:102218001F487AF037FCC1450ED8C144CA4526D8B4
:102228001B487AF0F9FB0020164B187000232B602E
:10223800002840F0E88045E0A9EB0802142A28BFEE
:10224800142207F11003124807F124017AF0FAFB6F
:102258003A690346002AE0D00028DED1009007F151
:102268002401074838F0FAF83B699844D3E712206C
:10227800DAE700BFA3D700204CAD002050AD002006
:1022880060540020A4D7002054B100205CAD002089
:102298000054002040F22113BB8463882968B3F5F9
:1022A8007B7F1CD3022387F8253000231422BA48E9
:1022B800009307F1240138F0D1F80023B74A1370CE
:1022C800B74A1360022034F01DFC402E00F28881CA
:1022D800212E00F27B81202E40F095807DE103F1D4
:1022E80014029142C0F04F814FF000092269DFF8D3
:1022F800D8A207F11401CAF80020AA4ADFF8B4826C
:10230800104602F803907AF007FBC8F8000000288E
:10231800C8D034F033F80028C4D0D8F800007AF0D8
:1023280029FB034618B9052287F82520BEE7D4E91A
:1023380002B33B60396896A3D3E900235846FEF7F9
:102348009BFE994B20F00100A0FB0303974AC2E9CA
:102358000003974BCDF800B002933B680622019327
:102368007969D8F800007AF01DFB80B102231422A5
:1023780087F8253007F124014B46CDF800908648B0
:1023880038F06CF8D8F800007AF0DFFA95E7D4F85E
:102398000490DAF80030C9F30808C8F50078A3EB10
:1023A8000903984528BF9846B8F1000F0DD1494652
:1023B8007F487AF067FB7E487AF072FB7C487AF0B7
:1023C8002BFB7C4B18687AF0C0FA784AC7F828903B
:1023D8001368C7F83480FB6253686F483B63002377
:1023E8001422009307F1240138F038F8B8F1000FEF
:1023F80003D169487BF064FB5FE72222674B1A70C0
:102408000022674B1A607B68002B3FF7E9AD11E6A5
:102418000C339A42C0F0B780D4F80480644841462F
:102428007AF030FBA268644907F1140360487AF037
:1024380019FBA268796903468A423FF61EAE002856
:102448007FF41BAEDFF880919044D9F80020C7F8DC
:102458002880A2EB0802B2F5007F28BF4FF4007273
:102468007A63524A11685268F9623A6307F12401A3
:1024780000901422484837F0F1FFD9F80030984509
:102488000DD14B487AF00CFB49487AF0C5FA494B14
:1024980018687AF05AFA40487BF012FB2EE622239D
:1024A80092E640F23113BB8463882968B3F57F7FD5
:1024B80005D30222002387F82520009304E61A1D7D
:1024C800914260D300223D490846CA547AF0BDFBC8
:1024D8008046B8F1000F52D002234EE003F11002FB
:1024E800914250D3364A581E115C2F294FF00001F3
:1024F8000CBF1154D154D4E9020125A3D3E9002318
:10250800FEF7BAFD284920F00100A0FB01012C4A82
:102518007AF06CFB804610B1022387F8253000233F
:10252800102200931C4807F1240137F097FFB8F1F7
:10253800000F7FF4E3ADAEE7286835F089FB174B51
:1025480018708BE540F261136288BB84A388296800
:102558001344B3F57E7FACDC0733994213D30023D1
:10256800184883546188A288013101448B547AF059
:1025780016FB0A288046ACD1052387F825300023AE
:1025880002220093CEE70123044A13703BE700BF01
:1025980000CA9A3B0000000060540020A4D7002025
:1025A8004CAD002064AD002000CA9A3BF8530020CF
:1025B8000054002054B100205CAD002054AD002030
:1025C80060AD002056AD002050B10020054B223EE2
:1025D800F6B2F340DB077FF516AF34F0A1FA12E745
:1025E800602E79E6014000402DE9F0412DED028B87
:1025F80090F8AD300446B0EE408A86B01BB9F7EECD
:10260800007A37EEC08AD4F884202F4B9A4213D12F
:1026180018EE100AFEF7B8F829A3D3E90023FEF74D
:102628009BFB011E18BF012104F1840039F0FEFB59
:1026380084ED288A012005E0B4F8A430B3F5807F42
:1026480005D1002006B0BDEC028BBDE8F08104F195
:102658005008404655F03EFB0028F2D0DFED1B7ACB
:1026680068EE277AFCEEE77ACDED037A94F880607D
:1026780094F8A4209DF80C30276E206D6EB18DF86B
:10268800153002238DF8142000210122009305AB98
:10269800B847404687F00BF9CAE7012531468DF85F
:1026A80013208DF814302A460DF113030095B8470E
:1026B800009532462946276E206D05ABE8E700BF36
:1026C800AE47E17A14AEEF3F9C050A0000007F4355
:1026D8002DE9F04F044685B0084661600621904612
:1026E8001D469DF838709DF83CB044F07DFDA06013
:1026F800067C16F0010602D07F484BF0D7F89DF80B
:10270800403005FB08F084F82A309DF844307D30CD
:1027180084F828307E2390FBF3F0C0011630B0F522
:10272800D07F38BF4FF4D070C4E904852773606246
:102738007EF071FF0DF1080A0622C4E907066F4909
:102748002046A66192F0AAFE022251462046ADF824
:10275800088092F0A3FE022251462046ADF80850A8
:1027680092F09CFEF623032269462046ADF800301D
:102778008DF8026092F092FE7B1EDBB2082B05D822
:1027880040F25515DD4015F0010501D15C48B4E76C
:10279800052F09D0072F06D0032F73D1012384F802
:1027A8002930002502E02E4684F82960002646F3E9
:1027B8004F10C0EB0020FDF7D5FF0022514BFDF76D
:1027C80085FE0022504BFEF761F9FEF7CFFA5FFA5B
:1027D80080F8C6F38200C0EB0020FDF7C3FF00229B
:1027E8004A4BFDF773FE0022494BFEF74FF9FEF7FF
:1027F800BDFAC7B206F00300C0EB0020FDF7B2FF38
:102808000022404BFDF762FE00223F4BFEF73EF9E7
:10281800FEF7ACFAC0B2002D5ED08DF808008DF836
:1028280009808DF80A70032251462046013692F03D
:1028380035FE802EBBD1BBF1000F1AD0354D01A952
:102848002A88AB782046ADF8042003228B7092F0DA
:1028580025FE0B222046304992F020FED5F80300D1
:10286800EB7902900522514620468AF8043092F00E
:1028780015FE204692F000FEA06992F021FE05B0F8
:10288800BDE8F08F092F84F829608AD10FF2580922
:10289800D9E90089354616A7D7E900672846FDF724
:1028A80061FF42464B46FDF711FE32463B46FEF7B6
:1028B800EDF8FEF75BFAC0B28DF808008DF8090054
:1028C8008DF80A00032251462046FF3592F0E6FDB6
:1028D800B5F5FF4FE2D1AEE78DF808808DF80970A5
:1028E8008DF80A009FE700BF0000000000C04F40BD
:1028F8000000000000C05F4028040B00F4B40A0088
:10290800F0FB0A000000F83F0000084000000C40FF
:1029180000001C40758A0900FBB40A000000000092
:1029280010EE103A33F0004210B52DED028B06D1AF
:102938000120BDEC028BBDE810406FF0F9BD002B03
:1029480005DABDEC028BBDE810406FF0FFBDB3F1B6
:10295800FF4F06DB30EE008AB0EE480ABDEC028B72
:1029680010BDB3F5000F6049BBBFDFED607A6FF0B3
:102978001802002260EE277AB8BF17EE903AF7EEF9
:10298800007ADC15C3F316037F3C1944144401F4A0
:10299800000282F07E5204EBD15403F10F011A4376
:1029A80007EE102A524A0A4037EE678AB2BBB5EEE4
:1029B800408AF1EE10FA0FD1002C00F08C8007EE5F
:1029C800904A9FED4C0A9FED4C7AF8EEE77A27EE95
:1029D800808A07EE878ABFE741A1D1E90001FEF7A7
:1029E800EDF9B6EE007A07EE900A07EEC87A68EEBF
:1029F800087A27EE277A14B938EE478AACE707EE4B
:102A0800904ADFED3C6AF8EEE77A07EEE67A37EEB1
:102A1800488A9FED397A17EE878A9DE7F0EE007AAB
:102A28009FED365ADFED364A364A78EE277A1A4451
:102A3800C3F5571388EE276A07EE904A03F5227309
:102A48001343F8EEE76ADFED307A002B66EE065A9C
:102A580025EEA57A07EE275ADFED2C7A45EE077AA0
:102A68009FED2B5A07EE875ADFED2A7A47EE274A61
:102A7800DFED297A44EE877A67EE877A45EE257A84
:102A88001ADDB6EE007A28EE077A27EE087A77EE96
:102A9800877A67EE867A14B937EE677AACE79FEDE6
:102AA800156A46EE867A37EE677A37EE488ADFEDA2
:102AB800127A16EEA78A4FE778EE677A67EE867A7B
:102AC80014B938EE678A47E79FED0A7A46EEC77A67
:102AD80037EEC88AEBE79FED118A3DE7AFF3008038
:102AE800555555555555D53F20FB4A000000004C1B
:102AF800F0FF7F00D1F717378071313F25333A3E19
:102B0800298E633E305CCFFF9788173E2549923E59
:102B1800ABAA2A3F4FD01C3ECDCCCC3E00000000D3
:102B2800F8B510EE904A10EE103A34F000472DED4B
:102B3800048BB0EE609A0DD183F480035B0013F52B
:102B4800000F40F2AA8230EE098AB0EE480ABDECC6
:102B5800048BF8BD23F000411846B1F1FF4F02D8AD
:102B6800B7F1FF4F08D9B3F17E5FECD184F480044C
:102B7800640014F5000FE4E7002B25DAB7F1974F4E
:102B880080F09482B7F17E5F39D3FA15C2F19602CC
:102B980047FA02F505FA02F2BA4229D105F0010511
:102BA800C5F10205B7F17E5F2AD1002C80F27B8245
:102BB800B5EE400AF1EE10FA1CD1D80FBDEC048B2B
:102BC800BDE8F8406FF0B4BCB7F1FF4F10D1B1F1D8
:102BD8007E5F00F0628205D9002CDFEDD17A29FEF4
:102BE800278AB2E7002C80F25B82B1EE498AACE713
:102BF8000025D7E7B7EE007A87EE008AA5E700251B
:102C0800B4F1804F0A4640F05782B1F1BF4F0CD261
:102C1800B1F1D05F02D920EE008A96E7B0EEC08A03
:102C280059BB012D00FE088A8FE723F04046B0EE1D
:102C3800C08AB6F17E5F17D1002CBCBFB7EE007A10
:102C480087EE088A002B80DAA1F17E51294305D14D
:102C5800BDEC048BBDE8F8406FF078BC012D7FF423
:102C680074AFB1EE488A70E739B9002CD9DA002B75
:102C7800A4D06B1E58425841A0E7DE0F013E55EA2A
:102C88000600E5D0B7F19A4F71D9A64B994208D8FA
:102C9800002C0BDA0020BDEC048BBDE8F8406FF087
:102CA80039BCA14B994208D9002CF3DC0020BDECBB
:102CB800048BBDE8F8406FF01FBCB7EE007ADFED7B
:102CC8009B7ADFED9B9A38EE478A93A1D1E9000100
:102CD80068EE278AFEF772F8B5EE007A07EE900ADA
:102CE800DFED946A68EE299A48EE477AB6EE007AE4
:102CF80007EEC87A68EE087A27EE277AF0EE687A47
:102D080047EE667A39EEA77A17EE103A6FF30B039F
:102D180007EE103A77EE699A77EEE97A013DF7EE19
:102D2800006ABFEE008A6FF30B04354367EE890A29
:102D380008FE268A06EE904A39EE666A67EE267A1B
:102D480046EE070A30EEA77A17EE101A002921F08E
:102D5800004340F31381B3F1864F40F2CC80B5EEC7
:102D6800C08AF1EE10FA4CBF0120002093E713F05F
:102D7800FF4F05BF9FED707A6FF01701002168EED5
:102D8800077A08BF17EE902AD315C2F316027F3BC5
:102D980042F07E500B4469498A4206DD68498A42FE
:102DA80040F3A7800133A0F500000021654A06EE34
:102DB800100AF7EE006A02EB8102D2ED005A75EEB6
:102DC800867A36EE657AC6EEA74A27EE245A15EEBD
:102DD800102A6FF30B0206EE902A5B4A02EA6002A1
:102DE80042F0005202F5800202EB415207EE902AAF
:102DF80006EEE77A77EEE57ADFED545A36EE676A43
:102E080065EE057A06EE667A9FED516A47EE865AB8
:102E18009FED506A27EE247A66EEA64A05EEA76A69
:102E2800DFED4D5A46EE275A9FED4C6A05EEA76A2C
:102E3800DFED4B5A46EE275A36EE856A67EEA77ADB
:102E480026EE076A05EEA76AF0EE085A74EEA57A30
:102E580077EE867A17EE902A6FF30B0207EE902A28
:102E680077EEE55A27EE277A66EEA76A75EEE45AFA
:102E780036EE656A06EE057A9FED3A6A76EE877A4F
:102E880017EE902A6FF30B0207EE902A364A77EE78
:102E9800E66A02EB810227EE866A37EE667ADFED94
:102EA800336A67EEA67ADFED326A47EE267A92ED4C
:102EB800007A77EE877A07EE103A2E4BF8EEC76A5B
:102EC80003EB810336EE277AD3ED005A37EE257AE5
:102ED80037EE267A17EE103A6FF30B0307EE103A27
:102EE80077EE666A76EEE56A76EEC66A77EEE67A99
:102EF80014E701215AE755D1DFED1F6A37EE677AEB
:102F080070EEA66AF4EEC76AF1EE10FA3FF727AF43
:102F180086234BE0AFF30080E13D55555555D53F2D
:102F280000000000F3FF7F3F0700803F70A5EC36EC
:102F380000AAB83F3BAAB83F0000804B71C41C00F0
:102F4800D6B35D00AC440A0000F0FFDF55326C3E9A
:102F580042F1533E05A38B3EABAAAA3EB76DDB3EBA
:102F68009A99193F0040763F9C440A00C623F6B858
:102F78004F38763FA4440A003CAA3833534A934258
:102F880007D9B5EEC08AF1EE10FA4CBF0120002037
:102F98008DE607D137EE677AB4EEE07AF1EE10FAF3
:102FA800B6DBEEE7B3F17C5F72D9DB157E3B4FF4FD
:102FB8000000474A002940FA03F00844C0F3C75309
:102FC800A3F17F0342FA03F2C3F1170302EA0002F6
:102FD800C0F3160040F4000007EE102A40FA03F090
:102FE80077EEC77AB8BF404237EEA07ADFED396A8C
:102FF800DFED395AB7EE000A9FED386A17EE103A3E
:103008006FF30B0307EE103A77EE677A67EE266ADE
:1030180070EEE70ADFED327A27EE277ADFED317AB4
:1030280000EEA77A76EE877A77EEE66A37EE667A6A
:1030380067EEA76A07EE877A16EEA56ADFED2A5AC9
:1030480046EE265A9FED296A15EEA66ADFED285A44
:1030580046EE265AB0EE676A05EEE66AF0EE006ABA
:1030680067EE865A36EE666AC5EE866A36EEC77A27
:1030780077EE677A30EE670A10EE103A03EBC0532A
:10308800B3F5000F06DA6FF0BBF820EE088A5CE5AE
:103098000020A9E700EE103AF7E7B7EE008A54E5FA
:1030A8009FED148A51E5B0EE408A4EE5B7F1FF4F27
:1030B8003FF48DAD0A460225B4F17C5F7FF4B5ADCF
:1030C800002BFFF6B2ADB1EEC08A3EE50000164314
:1030D800000080FF0072313F4CBB31330EEADD3512
:1030E8008CBEBF351872313F55B38A38610B363BF9
:1030F800ABAA2A3E0000000010EE103AB3F1FF4FD1
:1031080010B52DED048BB0EE408A06DB30EE008A58
:10311800B0EE480ABDEC048B10BD774A934276DCCA
:1031280023F00042B2F17E5F13D3FFEE007AB4EED3
:10313800670AF1EE10FA06D10120BDEC048BBDE858
:1031480010406FF0F5B9BDEC048BBDE810406FF08E
:10315800FDB9B2F1645F0FD2B2F14A5F24BF20EE2D
:10316800007AF6EE007ABDEC048B28BF07EE670AFA
:10317800BDE810406EF0FEBF604A134493424ED83B
:10318800F7EE007A38EE277A17EE103ADC157F3C16
:10319800002CD5BF77EE677A37EE488A78EE677AE3
:1031A80077EEC87A87EE879AC3F31603544A934298
:1031B800CCBF43F07C5243F07E52F7EE007AC8BF92
:1031C800C3F5000307EE102AC4BF01349B1037EE85
:1031D800678AF6EE008A68EE288A68EE888A002BED
:1031E80044D1B5EE408AF1EE10FA1DD1002C7AD008
:1031F80007EE904AB0EE498A9FED427AF8EEE77AF8
:1032080007EE878A9FED407A07EE878A80E7B3F159
:10321800B44FB5DBDC159FED3D9A7F3CC4E7012335
:1032280000249FED3A9AD4E731A1D1E90001FDF7D6
:10323800C5FDB7EE007A07EE900A07EEC87A27EECA
:10324800287A14B938EE478A62E707EE904ADFED2C
:103258002D6AF8EEE77A07EEA69A37EE497A37EE46
:10326800488A9FED297A17EE878A51E7F0EE007AAF
:103278009FED276A9FED277A78EE277AC8EE276AAE
:1032880066EEA67A07EE867A9FED236A07EE276A2E
:103298009FED227A06EE277A9FED216A07EE276ACC
:1032A8009FED207A06EE277A9FED1F6A07EE276AC0
:1032B800B0EE687A06EE277A27EE267A24B978EEF9
:1032C800C78A38EE688A23E707EE904ADFED0D6A71
:1032D800F8EEE77A07EEA69A39EE079A78EEC98AE9
:1032E80038EEC88ABDE79FED098A11E7AFF3008081
:1032F800555555555555E53FD613D43EE0096A4115
:10330800F6043500D1F717378071313F000000000F
:103318009788173E4FD01C3E25333A3E298E633E90
:103328002549923ECDCCCC3EABAA2A3F2DE9F047A9
:103338000546884600AF6FF04AFDA9680646B1F514
:10334800004F36BFA8F10403002303F00703B1F5CB
:10335800004F34BF0420082002F0070407341C443F
:103368000444E40804EBD2048C4228BF0C46012232
:10337800314628466FF0E5FC10EA020A16D1E94604
:1033880088B06A46504BCDE90538032342F8103F10
:103398004FF4C25153464D4801F006FACD468AF320
:1033A8001188BFF36F8F0423184602DF3146284681
:1033B8006FF0DDFC06EB00094946002228466FF055
:1033C800C0FCA9EB00094E4518D0E94688B069460B
:1033D8003F4BCDE90538032341F8103F3B481346DE
:1033E8000A464FF4C25101F0DFF90023CD4683F3BA
:1033F8001188BFF36F8F0423184602DF3146284631
:103408006FF0B5FC8442804623D028D2344431463C
:10341800224628466FF06DFD0122314628466FF09E
:10342800ACFC21466FF0A3FC261801223146284641
:103438006FF087FCC30708D4314628466FF009FDB2
:103448003246214628466FF07BFD214628466FF01C
:1034580095FD4FF001094846BD46BDE8F08706EBEB
:10346800000A0122514628466FF06BFC10EA020957
:1034780027D1514628466FF07AFC40448442EAD866
:10348800514628466FF0E5FC514628466FF06FFC20
:10349800A4EB0808804509D2344451462846224600
:1034A8006FF027FD214628466FF068FD52463146E9
:1034B80028466FF045FD0122314628466FF05DFC35
:1034C800C7E74FF00009C6E7FE5B0A0078880900E5
:1034D800225C0A002DE9F843884600AF00297DD018
:1034E8000568012228466FF072FC0146044628460A
:1034F8006FF027FC10EA020616D1E94688B06A4642
:10350800384BCDE90538032342F8103F4FF4C25138
:103518003346354801F048F9CD4686F31188BFF3A4
:103528006F8F0423184602DF214628466FF01FFCE0
:1035380026183146002228466FF003FC361AB4429A
:1035480018D06E4688B06946284BCDE90538032364
:1035580041F8103F244813460A464FF4C25101F07F
:1035680023F90023B54683F31188BFF36F8F042333
:10357800184602DF0022214628466FF0FEFB21464E
:103588006FF0F5FB26180122314628466FF0D9FB6B
:10359800C20708D4314628466FF05BFC3246214604
:1035A80028466FF0CDFC0022214628466FF0C9FB63
:1035B800261A0122314628466FF0C3FBC30709D4F7
:1035C800314628466FF045FC2246314628466FF0C2
:1035D800B7FC3446214628466FF0D0FCBD46BDE80E
:1035E800F88300BF4B5C0A0078880900225C0A0057
:1035F80008B5024870F05FF8002008BD785C0A0042
:103608000E4A0346904202D30D4A904211D30D4A06
:1036180022B1934202D30C4A93420AD30B4A52B1C5
:103628000B48834234BF01200020934238BF00205A
:103638007047012070471046704700BF1C81090081
:10364800FC1D0B000000000000000000000000004E
:10365800000000002DE9F04F9BB000AF04468B46F8
:10366800D7F890A0FA637B6349B9037846788078E5
:1036780000EB830020445E4522D8A0EB040B0AF03F
:10368800010394F80280FB62E378B8F1000F0CBFE5
:103698004FF000090AF001093B6313B11AF0020F59
:1036A80017D1B9F1000F14D1FB6B1BB15946204655
:1036B8007A6B98475D4628466C37BD46BDE8F08F63
:1036C800451C2846FDF794FD013028440BF1010BF9
:1036D800D1E7CAF3C003FB612378BB629B00BB61DF
:1036E80063683B62BB6A04EB8301FB6B002B7DD1F3
:1036F8005D468844B9F1000F1DD08B469946A94E06
:103708001BF8013B54F82300002808BF3046FDF79A
:103718006FFDD7F8943001304BB1D7F898304B454E
:1037280082BFD7F8943023F8190009F10109C3457D
:103738000544E5D1D8461AF0050F0CBF4FF0020B2F
:103748004FF0010B00260AF00203FB633B6B9E421D
:10375800B1D298F8013008F1020854F823A0504675
:10376800FFF74EFFFA69034602B3B86318F8021C64
:10377800386A6FF07FFFBB6BC0B1EA468AB06A4611
:10378800894B05933B6ACDE906314FF40073ADF8D8
:103798002030864B42F8103F00234FF412518448E2
:1037A80001F002F8D546023D0136CFE723B1FB6AA6
:1037B8002BB9A5EB0B05F7E7FB6B002BF4D0794889
:1037C800BAF1000F18BF5046FDF712FDD7F8943034
:1037D80053B1D7F8983099453FBFD7F89420431C88
:1037E80022F8193009F101090544DDE7B9F1000FA4
:1037F8006DD04346102B28BF10230026BB6397F8D3
:10380800389007F14800BA6B796294F0ABF9796A9D
:1038180000227A620AF0020201EB08033A610AF018
:1038280004027B61FA6002337A6A396B8A4267D391
:103838006378F96A1AF0020F7B624B4418BF0022C2
:10384800DBB208BF7208002940F0A9801AF0040F03
:1038580014BF314600216370A170E27020467A6B74
:10386800B969FB6B9847051EFFF625AFBB6A314661
:1038780023707B6A7A6B63703B6B84F80280E37019
:1038880007F15800FB6B9847061EC0F2C5803A6BDB
:10389800BB69386B03EB4203ABEB0301D7E90D239C
:1038A800C91A7B6903EB4000FB6B98470028C0F2FC
:1038B800B5804FF000082E44351807F1480AC8456E
:1038C80078D300217A6B0846FB6B9847F3E6B8F18A
:1038D800000F0CD01AF0040F0ED04346102B28BF4F
:1038E8001023BB6397F8386007F158008BE746460A
:1038F800C146C7F838808BE74E46C7F8388087E757
:1039080013F8015C13F8021C54F82500BB60FFF79C
:1039180077FE0246F869BB6838B1386AC7E90132F0
:103928006FF0A8FED7E90132F0B912B3FA6A72B1A2
:10393800B9F10F0F18D809F1280107F1400009F172
:103948000102014401F8205C5FFA82F90CE0FA6890
:1039580052B10F2E08D806F1280107F14000721C59
:103968000E1806F8105CD6B27A6A023301327A620F
:103978005AE73A69002ADBD10F2EF5D806F128005C
:1039880007F1400C6044721C00F8101C07F1680134
:10399800023651FA82F2F6B202F8105CE4E700212E
:1039A80059E700BFA65C0A00AD5C0A0004000001EC
:1039B800E887090018F80A3054F823B087F8473028
:1039C800D7F8943033B3D7F89830984522D2D7F83F
:1039D800943033F8186001217A6BFB6B07F14700CC
:1039E800984700281ADB0E4B0544BBF1000F08BFAF
:1039F8009B4626B95846FDF7FBFB461CB6B2314636
:103A080058467A6BFB6B9847002807DB054408F19A
:103A1800010854E70026DEE735464CE605464AE647
:103A2800A65C0A00014B1860704700BF980300208D
:103A3800044608B5EFF31183202383F31288BFF3FC
:103A48006F8F2DF029F8204602F074FE02486FF0BF
:103A580032FE71F001FAFCE7615D0A002DE9F047DA
:103A6800058B0446280717460CD501290CBF45F0DD
:103A7800100545F02005258387F31188BFF36F8F64
:103A8800BDE8F087022905F0070540F0948020463C
:103A980070F023F9052864D801A353F820F000BF7B
:103AA800813A0000BF3B00006B3B00002D3B00004B
:103AB800473B0000593B000001F007035A1F012A49
:103AC8001FD8002221F00701062BD4F8008089B204
:103AD800C4E9002209D1434603E0628B01326283C4
:103AE8001B68002BF9D141F002012046218370F0B8
:103AF800F4F84FF0000900286DD041F0200121832F
:103B080069E0042B0AD121F0070189B220462183FC
:103B180070F0E3F810B141F0200121834FF0000864
:103B2800C14658E02369D3F80090238B23F007039C
:103B380043F006034FF00008238346464BE0236911
:103B4800D3F80490238B23F0070343F00403F1E731
:103B58002369D3F80890238B23F0070343F0050368
:103B6800E8E74FF00008C146E7E7012243F0080301
:103B7800238387F31188BFF36F8F002A3BD1B8F1F5
:103B8800000F4AD1B9F1000F02D020462C49C8478E
:103B9800EFF31187202383F31288BFF36F8F238BF2
:103BA80023F008039BB22383D9063FD523F01002E4
:103BB800228303F007056669218B002EBFF67CAFD0
:103BC80000239946D4F8008021F00701C4E90033A6
:103BD80041F001012183238B03F0070AAA4502D093
:103BE800A268002AC1D1B8F1000F02D1B9F1000FC3
:103BF800DAD00022BAE7A1680029C0D00D680029F0
:103C0800BDD03346524620464F68B8471DB12B6891
:103C180029461D46F3E72B46FAE741463346524606
:103C28002046D8F8008070F084F8A8E79A067FF557
:103C380023AF23F02002228303F0070527E700BF04
:103C4800673D070037B504460821C06A70F024FBB9
:103C580000234FF6FF72104DADF804306368ADF8DD
:103C680000208DF80620E26819182B401344181A12
:103C780060606846ADF8021070F062FA6946204646
:103C880070F029FB2046211D70F034FA63682B4040
:103C9800A36003B030BD00BF0000FFFF2DE9F7436C
:103CA8000F4681460821C06A70F0F6FA80463C68E3
:103CB800124D241A3C6004EA0506B4421CD3A0B293
:103CC80010B903B0BDE8F08308236A462146484688
:103CD80070F0D7F90028F4D16946A0B270F0C8FA9C
:103CE80038B1BDF80230BDF804202E4013441E44FC
:103CF8003C60A4EB0804E0E70020E2E70000FFFFD7
:103D08002DE9F04704468AB000F11407384677F0E9
:103D1800F2FFA06A83681B699847E06248B9A8491E
:103D2800A84870F0A1FA6FF0150528460AB0BDE85A
:103D3800F087A06A83681B6998470368013B1F2BBB
:103D480001D9A149ECE7E368B3F5803F08D94FF4FE
:103D58008032012100929B489C4A70F05BFDE2E7AB
:103D6800A06A216807AA76F066FA08B19849D7E7E9
:103D7800E5682DB1089BB5FBF3F203FB12550DB1B5
:103D88009449CDE7238A012B01D89349C8E7E36A10
:103D9800029593F805804FF0FF334FF0FF32384615
:103DA8002FF0EAFC0821E06A70F076FAA946064688
:103DB800238A1FFA85FA534544D8238A4B4500F0D5
:103DC8000F8153450BD10299082342462046891B8F
:103DD80070F065F918B9204602A970F08BF92046F1
:103DE80002A9FFF75BFF0546002840F0FB80029917
:103DF8004FEA11494FEA09496160C4F80890A3687D
:103E08008B420DD80823204603AA70F03AF9B8B9B6
:103E180003AB13F8012B904532D101300828F8D1B3
:103E2800636820466FF30F0302A9029370F062F9EA
:103E380042462046E368029970F031F900283CDADE
:103E48000546CFE0E1682B04891B13FA81F142464D
:103E580008232046029170F022F978B1204602A981
:103E680070F048F909F101090823424620460299F1
:103E78001FFA89F970F013F900289ED0013597E7E9
:103E8800A08803A970F0F4F9626810B9911B616009
:103E9800B5E7BDF810A0BDF80E10E06AC4F80890A8
:103EA800514470F0F9F948448242A060EED1BAF169
:103EB800000FEBD06FF01C0594E05DD04FF6FF7952
:103EC800636806EB0308E3681FFA88F29B1B9A42B3
:103ED800CDF808801CD34FF000086168B8F1000FD6
:103EE80030D06FF30F012046029102A970F002F959
:103EF8002046029970F00BF90028A1D1E368A28846
:103F0800A3EB46039A426DD1204670F001FA97E779
:103F180008234146204605AA70F0B3F800288FD13F
:103F280005A91FFA88F070F0A3F930B1BDF8143074
:103F38004B4502D1BDF818300BB1B044C3E74FF080
:103F48000108CAE7204670F0E2F800287FF478AF4D
:103F58006368224AE16813400B44A3EB460363609D
:103F6800134041462046A36070F056FAC4E7E26A5F
:103F7800A36812681344A360D4E901318B4208D9BD
:103F8800424620465B1A70F08AF80028FFF658AFC0
:103F9800EDD16168E36801EB46029A42AED10F4B5E
:103FA800A06801EA03029042A8D0204670F0AFF85A
:103FB80000287FF445AF6268084B1A40A2609DE76D
:103FC800A95D0A0018880900CB5D0A00E85D0A00AF
:103FD800115E0A00295E0A003D5E0A000000FFFF2C
:103FE8006FF02C0538462FF039FC002D7FF49DAE7C
:103FF8000123A37499E600BF2DE9F04F1E46837C88
:1040080004468946904695B04BB96A496A4870F0AB
:104018002BF96FF00C05284615B0BDE8F08FC26A81
:104028000821104670F038F9B1B20190104670F0CE
:1040380033F9E368019A0746A3EB82038342C0F091
:10404800B6801EB1B8F1000F00F0B180D4F804A01A
:10405800CDF810A0204605AA04A970F093F90546EA
:104068000028D8D1BDF814304B4507D0DDF810A092
:1040780063685345EED1002E39D1CCE705A91FFA64
:104088008AF070F0F5F80028F0D0BDF8183066B363
:10409800B3422CD1B3464FEA1A43BDF816A01B040D
:1040A8009A44E36ACDF800801B685B4203F0200362
:1040B8000293029B51465B4528BF5B4620460CAAEB
:1040C80003936FF0DEFF00284DD1039B00981A463A
:1040D8000CA993F075FD50B9039B009ABBEB030B39
:1040E8001A449A440092E4D195E7002B93D0002F0C
:1040F8003CD1BA4604F1140B4FF0FF324FF0FF33B6
:1041080058462FF039FB238A9D424DD0D4E901321D
:104118000AEB02018B422ED39BB263B3FF2300212B
:10412800ADF81E200CA818228DF82230ADF81C908E
:10413800ADF8206093F03CFD20460CA9CDE90E8631
:1041480070F0B4F8074648B907A86FF0F9FF2046A1
:1041580007A970F0C0F8074600B9374658462FF04F
:104168007DFB3D4657E7C2DC054654E7019B1F44EB
:104178001FFA87FABEE72046FFF764FD3DB9ADF8A0
:104188002490CDF82880ADF82C608DF82E5020466C
:1041980009A970F041F907460028DFD19DF82E30B3
:1041A8000135002BAFD0D8E76FF01B07D6E76FF0CB
:1041B800150530E7955D0A00188809002DE9FF47C5
:1041C8001E46837C04460F469046BDF8309043B99E
:1041D8002748284970F048F86FF00C0004B0BDE893
:1041E800F0870821C06A70F057F8E368A3EB400332
:1041F800B3423AD34FF0000A65680195204602AAF7
:1042080001A970F0BFF80028E8D1BDF80830BB421A
:1042180006D102A9A8B270F02BF850441FFA80FA10
:10422800019B62689A4219D0CA4515D9BDF80C306D
:10423800C3B1CA4516D3BDF80A10B3426FF30F05D0
:1042480028BF33464246204629446FF01AFF00280B
:10425800C4D1BDF80C00C1E71D46CFE7BDF8083052
:10426800BB42E3D06FF00100B8E76FF01500B5E787
:1042780018880900955D0A002DE9F04704460746AD
:104288004FF00109DFF84C8094FAA4F5B5FA85F5EA
:1042980009FA05F32E0108EB05156FEA030A24EA6B
:1042A80003042B7B63B158F806301B696BB946448D
:1042B800736802222846196807EA0A0770F027FA85
:1042C800002CE1D13846BDE8F087284698470028F9
:1042D800F6D1ECE73089090010B5002288B00E4904
:1042E8000E4878F008F9002200230024CDE90623BF
:1042F8000E234FF44072CDE90334CDE90144084B55
:104308000849009408482FF0B5FE0849064877F098
:104318004DFF204608B010BD39430000282D00206D
:104328005946000058DA002040280020675E0A003D
:1043380001482FF019BB00BF182100202DE9F047D4
:10434800804621480F4670F0C6F90646002833D04B
:1043580000252846BDE8F087237B83B12368DB6806
:104368000BB120469847636883F8069023681B6959
:10437800D3B9636802222046196870F0C8F901367B
:1043880010345445E8D3B8F1000FE2D0002DDFD047
:104398002846FFF771FF0546002FF7D0002140F2AD
:1043A800391078F005F8F1E7204698470028E0D062
:1043B80009FA06F31D43E2E705464FF00109034CED
:1043C800DFF80CA0DDE700BF38570020308909006E
:1043D80040890900014B53F8200070475C8D0900A3
:1043E80008B5034608462BB1044A136000F04CFC9C
:1043F800002008BD6FF01500FBE700BF9C030020FC
:1044080010B5044C237813B903482FF0ADFA0123F3
:10441800237010BDA6D300201821002010B5044633
:10442800094870F058F93CB1084BD3E8EF1F01393F
:10443800C3E8E21F002AF8D1054830F03DFCBDE88A
:10444800104004482FF090BA30570020345700200D
:10445800282D0020182100200022044BD3E8EF0F5C
:10446800C3E8E12F0029F9D1704700BF3057002079
:1044780070B5FFF7F1FF0546074C084EB44200D36C
:1044880070BD63685B792BB123685B6813B12946FB
:10449800204698471034F1E730890900408909001F
:1044A80010B5044C044920466FF020FA034B1C60F9
:1044B80010BD00BFC81F0020488D090028570020E4
:1044C80000230D4A10B513700C4A0D4913600D4AAC
:1044D8000D481360FFF784FFFFF7E2FF0B4B0C4911
:1044E80018468B4200D310BD1A1A5C6812110132AB
:1044F80022711033F5E700BFA7D300203057002002
:1045080040420F0034570020DB460700308909007D
:1045180040890900014647F61222002301486FF03E
:1045280006BA00BFC81F002001486FF09CBA00BF40
:10453800C81F0020024B014618686FF0EFBA00BF91
:104548002857002001486FF024BB00BFC81F002077
:10455800F8B5284B1B78002B4AD0FFF7E5FF044637
:10456800002842D1244B254D1B68002B19DD77F01C
:104578007AFF4FF47A76A0FB060747F6122200234B
:1045880006FB0171FCF7C8FDD5E90032C01A40F2FC
:10459800E93361EB0201984271F1000101D3FFF7A1
:1045A80067FFD5E9003213F57A7342F10002C5E9D5
:1045B8000032ECB1BDE8F840FFF7C4BF6B685B7927
:1045C80023B12B68214628461B6898471035B54209
:1045D800F4D32046FFF7AEFF094BD3E8EF1F0139AC
:1045E800C3E8E21F002ABDD0F7E7064D064EEEE706
:1045F8000020F8BDA6D3002030570020202D002031
:1046080034570020308909004089090070B50D4DE4
:10461800297861B90120FFF791FE0B4C0B4EB4428B
:1046280006D3FFF795FF0028FBD101232B7070BD3F
:1046380063685B791BB1236820469B6898471034F0
:10464800EDE700BFA7D300203089090040890900A1
:1046580000212DE9F8430846FFF770FE044648B3E9
:1046680040F21B684FF0000901F0D8FB1A4B1B4AB7
:104678001B58136033B11A4B1B68092B02DD19480C
:104688002FF072F90025184F44B12046FFF7F4FDCA
:10469800044618B94FF0FF384FF0FF39FFF758FFBD
:1046A800064628B9B5B90F4842464B462FF098F947
:1046B8003546E9E74FF0FF384FF0FF39D4E72B686C
:1046C8009B691BB100222846114698471035BD4208
:1046D800F5D3E8E7054DFAE7080000002C5700205D
:1046E800345700201821002040890900308909002A
:1046F80013B518486FF0EFFF174B1B7873B1EFF342
:104708001184202383F31288BFF36F8FFFF720FFF4
:1047180084F31188BFF36F8F02B010BD0F4B1B6875
:10472800002BF9D050B9002200230D48CDE9002311
:1047380047F61222002330F099FAEDE70928EBD169
:10474800074830F0B9FA074802B0BDE810402FF02A
:104758000BB900BF34570020A7D300202C570020E6
:10476800282D00201821002010B5064B04461B6890
:1047780098472146A06004486FF056F9BDE81040FC
:10478800FFF7B6BF9C030020C81F0020044A054B52
:104798009B1AB1EBD30F34BF52F831000020704799
:1047A80028870900308909002DE9F04F8FB0C1F33F
:1047B8004A2604AF0D469046B8607B600C0D002E6B
:1047C80061D04FF000090A234FF0040B07F1140AD7
:1047D800FE60C7E90799C7F824900093CDF808B0A0
:1047E800CDF804A007F11C034A464046F968FEF7D5
:1047F80031FFB0F5006F03461CD36C468AB0D8F879
:10480800041004AB24481A46C3E9050140F2FF71BD
:10481800D9614FF400711984204B42F8103F4FF4CE
:1048280012514B461E48FFF7BFFFA5462C37BD4621
:10483800BDE8F08FC0F30A0604F11700184420F011
:10484800070080083B60FFF765FE66F353250446C2
:1048580080B13B6800F11001C7E908390A23F96102
:10486800CDE901AB009340460E4AF96807F11C03F5
:10487800FEF7F0FE66F353252A4620467B68B968A2
:104888006FF065FFD2E704F1170020F007008008F9
:10489800FFF740FE0446EDE7785E0A0004000001D9
:1048A80040880900294707002DE9F04F87B00546E1
:1048B800DDE9106BDDE9127A884614469946BFB1E6
:1048C80010213B465A460020CDF800A0CDF814A090
:1048D8006EF0F7FCB0F5006F01460BD340F2FF73A2
:1048E8000221184A184807B0BDE8F04F6FF088BF9A
:1048F8003946384604F0070305F00704E40044EAA3
:10490800831444EA402444EA065406F11700084494
:1049180020F0070080080391FFF7FCFD054640B131
:104928003FB13B465A460399CDF800A010306EF0CF
:10493800C8FC4B4622464146284607B0BDE8F04F22
:104948006FF005BFB75E0A0040880900406820B1D3
:10495800034BC01A40F3CF0070474FF0FF30704749
:10496800288709000EB403B503AB53F8042B01469E
:104978000448019301F086FC02B05DF804EB03B033
:10498800704700BF6B480700CA0605D48B064CBFAA
:1049980002490349FFF7E6BF704700BFD2AC0A00DF
:1049A800E3A30A002DE9F04F8BB099469DF8588093
:1049B800179B044607930D46DDE918A31A9F069234
:1049C8000593B8F1000F00F0BC80834B07F0020B91
:1049D80013F80830089307F4807309936FF095FE75
:1049E800024600287AD020467C49FFF7BBFF0646DE
:1049F800BBF1000F08D017F0440F71D12A462046AA
:104A08007749FFF7AFFF064407F0010353B1754B31
:104A1800204653F82820744B7449002A08BF1A46C8
:104A2800FFF7A0FF07F48073002B07F0080318BFF7
:104A38004FF00009002B7FD06D4B204653F82820FB
:104A48006C49FFF78FFF0546069B2BB11A46204697
:104A58006949FFF787FF0544B9F1000F0DD0089B9E
:104A6800002B6CD06549664BB8F1040F18BF194686
:104A78004A462046FFF776FF054462483544079BBF
:104A88001BB1224660496EF0C4FD059B002B00F067
:104A98008E80059B3946102B28BF10232046994647
:104AA8000026FFF771FFB54252DC00263346204648
:104AB8001AF803205549FFF755FF0136102E4DD03F
:104AC800710703D120465249FFF74CFF4E45334644
:104AD800EDD320464F49FFF745FFEEE7064687E747
:104AE8004D4B186800288ED04C4B4FF47A7B1B68CE
:104AF8004FF03C0CB5FBF3F5B5FBF0F14FF46163F7
:104B080000FB11550BFB05F5B1FBF3F2B5FBF0FE0D
:104B180003FB121100FB1E55B1FBFCF30BFB05F563
:104B2800B5FBF0F50CFB131120460091CDE901E52A
:104B38003B49FFF717FF66E707F0080584E73049A8
:104B480096E7B9F1010F45460CBF2E48354896E760
:104B580020462F49FFF706FF0136A4E70026204626
:104B68003149FFF7FFFE33461AF803202046A2F129
:104B780020035F2B28BF2E222C49FFF7F3FE0136B6
:104B8800102E0DD0720703D120462149FFF7EAFE07
:104B9800B1453346E8D820461D49FFF7E3FEEEE766
:104BA800059BCA44B3EB090305937FF472AFB8F1D0
:104BB800000F0AD0FB0704D520460B4A0B49FFF724
:104BC800D1FE39462046FFF7DFFE20460BB0BDE890
:104BD800F04F6FF039BE00BF63B50A00FD5E0A00F2
:104BE800015F0A006C8D0900EF5E0A007AAE0A00C8
:104BF800808D0900275F0A002D5F0A00F45E0A0015
:104C0800F85E0A006B4807008D620000315F0A00F9
:104C18007BB40A0079B40A00405700203C570020B2
:104C28000B5F0A0099480700375F0A0088AC0A0042
:104C380042F20F7373B58B4228BF0B4605680446D2
:104C4800052168460D4A6AF057F906466368284602
:104C58000B225B680A496FF0E9FD636832466946D2
:104C680028465B686FF0E2FD63681B2228465B6894
:104C780004496FF0DBFD02B070BD00BFCBB30A0082
:104C880057B50A003BB50A0000210123064A9042A5
:104C980006D8064A01B901231360054B186070470E
:104CA800012140085B00F2E740420F003C5700201A
:104CB80040570020F8B50D460446064F4618B44242
:104CC80001D12846F8BD14F8011BBB6801485B6890
:104CD8009847F4E74C830900014B036000207047B4
:104CE800C88D090070B5104B0D461C68B4B10F4B48
:104CF800196800238B4202DB6FF0010070BD224669
:104D080012F8146B864202D014460133F2E7E068C9
:104D180076F09AFE28B100202C60EFE76FF00C00C7
:104D2800ECE76FF01200E9E7A8030020C88D09003E
:104D380010B5436888B0029383680C46CDE9033206
:104D480000230A68C068CDE90623054901AA05932E
:104D580075F075FA079808B9059B236008B010BD6F
:104D68002B4A070010B54FF42814DFF820C086B08E
:104D7800CDE904C40824029404AC0194BDF8204091
:104D8800009473F055FB06B010BD00BF1800280052
:104D98002DE9F8430646FCF72BFA0546EFF3118890
:104DA800202383F31288BFF36F8F114B1C68D3F84D
:104DB80004909C4208BF002434B988F31188BFF3DB
:104DC8006F8F2046BDE8F883A7683846FCF710FACD
:104DD800A84206D12A463946304692F00EFF0028EE
:104DE800EBD04C4501D02468E6E70024E5E700BF96
:104DF800C40300202DE9F0410E461546FFF7C8FF11
:104E0800044628B3C3681BB35F690FB3062E07D0E7
:104E1800072E20D02A4631463B46BDE8F0411847C8
:104E2800838A3BB92A463146B84750B9A38A013329
:104E3800A38206E04FF6FF72934204D00133A382A7
:104E48000020BDE8F0810121114A12486FF0CFFC23
:104E58006FF01500F5E745B12A7832B10022828259
:104E680031462A465B699847EAE7A38A012B08D1AD
:104E78002A4607212046B8470028E2D1A38A013BE9
:104E8800D6E70BB1013BDAE70221034ADDE700BFB1
:104E9800915F0A0000880900B35F0A0010B5044654
:104EA80008B1806838B9104A104801216FF09FFC9A
:104EB8006FF0150010BDFFF76BFF08B10C4AF3E760
:104EC800A082EFF31181202383F31288BFF36F8F41
:104ED800084B5A68C4E9003214605C6081F3118899
:104EE800BFF36F8FE6E700BFD15F0A0000880900B3
:104EF800EA5F0A00C40300202DE9F0410C4B054687
:104F08001C680E4617467CB100F06AF963682046B3
:104F1800D3F8108032463B462946C047044600F085
:104F280069F92046BDE8F0816FF00104F9E700BF98
:104F38007057002000230360044B5A6812B9C3E974
:104F48000000704710605860704700BF7457002019
:104F5800014B1860704700BF70570020002330B520
:104F680085B0CDE902330546019000F039F9094BC7
:104F78001C6844B9284600F0D5F8044600F03AF910
:104F8800204605B030BD636820461B6801A99847D4
:104F98002468EEE7745700201FB5CDE9010103929C
:104FA80000F01EF9074B1C6824B900F023F92046CD
:104FB80004B010BD636820461B6801A9984724689F
:104FC800F2E700BF745700200022024BC3E9002219
:104FD800704700BF745700200022024BC3E900222B
:104FE800FFF7F2BF7C5700202DE9F74307460C4630
:104FF80009B100230B6000261E4DDFF880904D4557
:105008000FD31D4B1D6885B355F8188C384641469B
:1050180001AA183D6FF0EBFD10B3D6B914BB2E46AC
:105028001EE0D5F800803846414601AA6FF0DFFD42
:1050380050B116B954B92E4606E0002240463168F0
:105048006FF0D5FD0028F5D11835D8E7019B23600E
:10505800F1E70022404631686FF0C9FD0028DDD134
:10506800AD69D0E7019B2360D9E7304603B0BDE8BE
:10507800F08300BF408909007C570020D0890900CF
:105088002DE9F04784B002AFD7F8289004460D46C2
:10509800164698467860B9F1000F07D0D9F8001085
:1050A80031BBD9F804A0BAF1000F28D12046391D28
:1050B800FFF79AFF08B3D0F80C90434632462946CA
:1050C8007868C847C8B16D468AB002AA124BD06149
:1050D800C2E905344FF400731384104B42F8103FB3
:1050E80000234FF411510E48FFF75EFBAD4604E074
:1050F8003A1D6FF07CFD0028D3D1002007E0D9F8D5
:10510800083032460093294643467868D047083726
:10511800BD46BDE8F08700BF13600A000400000127
:10512800808809002DE9F04780464FF000470026A7
:10513800DFF8A490DFF8A4A03D46264C4C450DD3DB
:10514800DAF80040002C40D0183CB8F1000F24D108
:10515800226952BBA469F5E72F46EDE7B8F1000FC5
:1051680003D122694AB91834E8E700224146206889
:105178006FF03DFD0028F4D1F5E76368BB4206DD1A
:10518800AF4202D0AB42A8BF2B461D46EBE7EAD19F
:105198009047002E08BF0646E5E7002241462068F2
:1051A8006FF025FD0028D3D1D4E76368BB4206DD44
:1051B800AF4202D0AB42A8BF2B461D46CAE7C9D1B1
:1051C8009047002E08BF0646C4E7AF42C4D1304618
:1051D800BDE8F08740890900D08909007C57002084
:1051E8004FF0FF324FF0FF3301482EF0C5BA00BF31
:1051F800A420002001482EF031BB00BFA4200020CD
:1052080038B5094DFFF7ECFF2B785BB9FFF7E4FEE3
:1052180000F06AF8044608B901232B70FFF7EAFF8B
:10522800204638BD0024F9E7A9D300202DE9F04332
:1052380006460F46048F99B00134A4B200F108085D
:10524800651EADB2B5F5004F4AD04A23294605AAD6
:1052580040466FF025FA04F57F543F34A4B28146E6
:105268002146012340460DF10B026FF019FAB9F1FE
:10527800000F014610DC002810DC338FAB4209D147
:1052880032466B1E22F8383F4FF400410223404655
:10529800FEF7B2FE2C46D3E7002808DC2946404634
:1052A8006FF0FAF9214640466FF0F6F9E5E7B9F1F3
:1052B800490FEFD809F160030DEB03090023094AF0
:1052C80009F84C3C05A8009703ABCDF80C80ADF865
:1052D8001040FFF7D5FE0028DCD019B0BDE8F083F8
:1052E8000020FAE7674C07007FB5012369460420D0
:1052F8000193FFF7F7FC044668BB042002AA01A942
:105308006FF0B1FB044610B110F10C0F23D10399D3
:10531800B1F5803F24D200231846009A94680844C7
:1053280084421BD30133B3F5807FF8D10E4D6961F8
:105338002B8353682846AB60D368EB636FF027FD77
:10534800044640B9094E28466E60FFF7F3FD28462B
:105358006E60FFF7FDFD204604B070BD9BB2E5E727
:105368006FF02004F7E700BF84570020BC8E0900C7
:105378002DE9F04F8BB09146D0F808A01E4600AF3B
:10538800DAF8103080460D469847B9F1000F05DA73
:105398002B4A01212B486FF02AFA0AE0036846EAF3
:1053A80009045A1E14400BD00121274A25486FF0E2
:1053B80027FA6FF0150528462C37BD46BDE8F08F53
:1053C800DAF80CB0BBF1000F06D0294633464A463E
:1053D8004046D8470546EEE7202B01D91B4AD8E7B7
:1053E8002946202207F1080092F0E2FB2546A64252
:1053F800E1D9331B202B28BF202309EB040BDAF853
:1054080004505946404607F108027B60A847051E2C
:105418007B6812DA6C4688B06A460D4BCDF81CB032
:10542800CDE90538042342F8103F00234FF4015119
:105438000448FFF7B9F9A546BDE71C44D7E700BF04
:1054480038600A000888090055600A0087600A0069
:10545800AD600A0080B505460E46174698462FF0FF
:1054680029F9034600F0DAFC0446DFF818904246B2
:1054780049F8003039463046A84754F8090000F08A
:1054880045FC00BF0800000008B50348034A002196
:10549800121A6FF0B8FC08BD0025002058DA002069
:1054A800074808B5074A0849121A6FF0AEFCBDE86C
:1054B80008400648064A0749121A6FF0A6BC00BF02
:1054C80000000020D0240020FC1D0B00000000205C
:1054D80000000020FC1D0B002DE9F84F80460C460B
:1054E80000AF00296AD0D1E90012E9468AB0A36862
:1054F8006D464FF0050A6E463948CDE90723CDE9D8
:10550800050146F810AF002332464FF421513548C3
:10551800FFF74AF9D4E90312CD466369AD4632482C
:10552800C5E90723C5E90501C5F810A000233246DF
:105538004FF421512B48FFF737F9CD46E369012194
:105548002A4A28486FF05CF90121294A25486FF05A
:105558004EF9264600254FF00A0ADFF8A4B0E946BE
:10556800D6E908C0D6E90A138EB06A46CDF81CC041
:1055780005F1010CCDE908C0A81CCDE90A01E91C18
:10558800CDE905B5CDE90C1342F810AF002345F27B
:10559800400114480435FFF707F9102DCD4606F1F0
:1055A8001006DCD1236E0121124A0E486FF028F94B
:1055B800A3690121104A0B486FF022F9B8F1010FD5
:1055C80007D1EFF305830D4A41460648103B6FF0BB
:1055D80017F9214640462DF0FFFDBD46BDE8F88F7E
:1055E800D4600A007088090003610A0032610A0069
:1055F80041610A00BE610A00CD610A00FB610A0030
:105608007B610A0030BFFFF7FDBF00BF2DE9F04105
:1056180005460B4EDFF83080324606EB0807CC1BF8
:105628002046084992F09EFAA01942460021083CFB
:1056380092F0BEFAC5F8904007F10800BDE8F08185
:1056480000000000D08909000800000010B5244CB3
:10565800244925486FF0E6FBA36A99013ED5224804
:1056680022496FF0DFFB1E20A36ADA0104D51E4829
:105678001F496FF0D7FB1F20194CA36ADB0204D522
:1056880019481C496FF0CEFB0220A36A1C0304D5FD
:10569800154819496FF0C6FB2120114CA36A59031C
:1056A80004D5114815496FF0BDFB2220A36A9A035F
:1056B80004D50D4812496FF0B5FB2320084CA36AA6
:1056C800DB0304D508480F496FF0ACFB2420A36A1C
:1056D8006FEA03436FEA1343A36210BD1D20C3E7BB
:1056E80000ED00E00E620A007088090026620A00D8
:1056F80039620A0053620A007D620A009B620A004E
:10570800C0620A00DA620A0070B506460D46294CE6
:1057180029492A486FF086FBA36ADB0647D5274844
:1057280027496FF07FFB1120A36A1C0704D5234883
:1057380024496FF077FB12201E4CA36A990712D5F3
:1057480021491E486FF06EFB636BA26A120609D5E9
:1057580001211E4A19486FF053F81EB1A36A23F0BD
:105768008003A3621320134CA36ADE0704D51348F1
:1057780017496FF057FB1420A36A9C0604D50F48FD
:1057880014496FF04FFB15200A4B9A6AD10658BF8F
:105798009A6A9A6A920642BF5A6A22F400525A6278
:1057A8009A6A42F0FF029A6200232B7070BD1020A3
:1057B800BAE700BF00ED00E005630A007088090041
:1057C8001B630A004E630A0061630A0079630A00DA
:1057D8008F630A00AE630A0070B506460D46284C72
:1057E800284929486FF01EFBA36AD9043CD52648EE
:1057F80026496FF017FB1720A36A1A0504D522481B
:1058080023496FF00FFB18201D4CA36A9B0512D586
:105818001D4820496FF006FBA36BA26A100409D546
:1058280001211D4A18486EF0EBFF1EB1A36A23F44C
:105838000043A3621920124CA36A590504D51248E3
:1058480016496FF0EFFA1A20A36ADA050ED50E484A
:1058580013496FF0E7FA1B20094A936A43F47F4320
:10586800936200232B7070BD1620C5E7A36A9B04C2
:10587800F2D505480B496FF0D5FA1C20ECE700BFBC
:1058880000ED00E0DD630A0070880900F3630A0098
:105898004E630A0004640A001D640A0032640A00A8
:1058A8004D640A00AE630A00F0B59DB0664B05462C
:1058B8005868002600AFC0F3080386F31188BFF3C9
:1058C8006F8F02F07F44B4F17F4F07D102F00C04D0
:1058D800082C0ED15D495E486FF0A4FA5D495C481A
:1058E8006FF0A0FA00210846FFF7F6FD7437BD46B1
:1058F800F0BD14074CBF0D460126002DEED0002246
:10590800FA71DA1E092A7ED8DFE802F00575787187
:105918007D7D7D7D7D7B50494D486FF083FA002366
:10592800494CFB71E36A9A0705D54C4948486FF022
:1059380079FA00242DE0E36A002B01DA4849F5E7FB
:10594800E36A5B00F5D5474941486FF06BFA636934
:10595800AA6943F480736361BFF34F8FBFF36F8FFE
:1059680032F8023C626922F480726261BFF34F8FA1
:10597800BFF36F8F03F47F42B2F55F4F21D1DBB2E3
:10598800022B1ED12B680121374A31486EF038FFAF
:105998002C68FB79002BA9D16822294607F1080059
:1059A80092F0E0F87B6A002E4AD0C3F3080222B9CD
:1059B8006FEA53236FEA43237B62204607F108010D
:1059C80092E7214B9A6AD2B222B10120F91DFFF762
:1059D8009BFE0EE09A6A12F47F4F04D00120F91D55
:1059E800FFF7FAFE05E09B6AB3F5803FA1D3FFF706
:1059F8002DFE0446CDE70020F91DE8E70020F91D3B
:105A0800EEE71A4992E71A4A6C4610F4F87F8AB012
:105A1800184918BF11466A46103B07934FF40073A4
:105A28001548ADF82030154BCDE9050142F8103F77
:105A380000234FF411510648FEF7B6FEA54678E755
:105A48006FF30803B8E700BF00ED00E093640A00B5
:105A580070880900BE640A00FA640A0011650A0029
:105A680032650A0040650A005F650A007B650A0026
:105A78007A640A0065640A009F650A000400000150
:105A8800064B5A6942F010025A615A6942F4806220
:105A98005A615A6922F008025A61704700ED00E025
:105AA800EFF30880EFF3098101B57246FFF7FCFEBA
:105AB80001BD00BF0B4880F308882BF073F8202045
:105AC80080F3118808484FF40061401880F3098872
:105AD800EFF314800221084380F31488BFF36F8F1B
:105AE80000F068F868780120481001201EF0040FC3
:105AF8000CBFEFF30880EFF30980816911F8021CED
:105B08000229FFD001B572466FF081F901BD00BFCF
:105B18000028ACBF00F16040064B4FEA4111C9B202
:105B2800ABBF00F5614000F00F0080F80013195476
:105B3800704700BF14ED00E000B2002807DB012326
:105B48004109034A00F01F00834042F821307047A2
:105B580000E100E000B200280CDB012206494309FD
:105B680000F01F008240203341F82320BFF34F8FFD
:105B7800BFF36F8F704700BF00E100E0054B42099B
:105B880053F82220012300F01F0003FA00F0104010
:105B9800704700BF00E100E0044B054A23F07F0393
:105BA8009360BFF34F8FBFF36F8F70470000000003
:105BB80000ED00E008B5FFF7EFFF104BD3F88820A1
:105BC80022F47002C3F88820D3F8882042F4A00297
:105BD800C3F888204FF04042C3F83422BFF34F8FF8
:105BE800BFF36F8F0023E1EE103AFFF74DFCFFF78C
:105BF80057FC00F0F3F82DF01BFC00BF00ED00E0AF
:105C08008189203A41F0020181814FF47D41C0F839
:105C1800DC101360009B08495360019B21F00101CF
:105C28009360029B9161D3604FF08073D36100232E
:105C38000265C0F8943070475D540000104B9B68B3
:105C480083421AD1EFF30580B8B9EFF3118120220E
:105C580082F31288BFF36F8F9A8922F002029A8129
:105C6800EFF3148323F0040383F31488BFF36F8FD7
:105C780081F31188BFF36F8F70476FF0150070477D
:105C880048A900200E461546002300B5E1EE103A5B
:105C9800EFF3148323F0040383F31488BFF36F8FA7
:105CA800BFF36F8F0C4BD0F8902098600B4B1A60A5
:105CB800D0F8803083F30B882C4686F309880020BF
:105CC800034B98472046002100220023014C20471F
:105CD800534E07005D54000048A90020C457002017
:105CE8001022014B1A61704700ED00E0054B9A69DC
:105CF8009B689A421FBF044A536843F0805353601D
:105D0800704700BF48A9002000ED00E0084B9B68E1
:105D180083420BD1EFF3058343B1064B5A6842F037
:105D280080525A605A6A22F400425A6276F043BAA4
:105D380048A9002000ED00E025498A6882F8DDE0E6
:105D48004FF030001044EFF3098C80E8F01F1EF08C
:105D5800100F03D102F19C0080EC108A202080F300
:105D68001288BFF36F8F1B4F4FF000668A698A60F5
:105D78003E60D2F89000184C206092F9DDE0D2F82D
:105D880094000023C2F8943080F311881EF0100F9D
:105D980003D00023E1EE103A03E002F19C0090ECFE
:105DA800108AEFF3148323F0040383F31488BFF3FA
:105DB8006F8F02F1300090E8F01F8CF3098802F130
:105DC800000004B56FF03AF8BDE8044070470000E1
:105DD80048A9002004ED00E0C4570020002320213A
:105DE8000448C2180133B3F5917F82F80013F8D143
:105DF800704700BF00E100E008B5EFF30583064AED
:105E0800103B02EBC30152F8330049688847BDE8EC
:105E18000840FFF76BBF00BF8C16002001480068E0
:105E280070470000C45700201FB50121094B0A4ADA
:105E38000A4800F00FF90023064A0393084B012192
:105E4800019301A8D31A029300F00EF905B05DF88A
:105E580004FB00BF00FC072000000020DC8E0900C6
:105E6800002500200A7A0B6810B562F304031C466B
:105E7800CB68520923F01F0343EA4203044A43F064
:105E88000103C2F89800C2F89C40C2F8A03010BDC7
:105E980000ED00E010B50A4BD3F89030C3F30723A8
:105EA800013B984208D901210346064A06486EF08C
:105EB800A7FC6FF0150010BDFFF7D4FFFBE700BF8C
:105EC80000ED00E0B6650A00588809002DE9F04F9A
:105ED8008946144606464FF000084F4D85B0C84520
:105EE80027DAD6F804A0BAF1000F44D0BAF11F0F90
:105EF80017D91AF01F0F14D1D6F800B01BF01F0FD6
:105F08000FD158466EF0C4FF07460AEB0B00013864
:105F18006EF0BEFF874210D06FF015073F4A3B4630
:105F280001E043463E4A01213E486EF069FC6FF0AD
:105F38001504204605B0BDE8F08F17F1160FEDD017
:105F4800BC42EBDDC5F89870D5F89C10C5F8987080
:105F5800D5F8A03021F01F0143F01F0BD6E900321D
:105F68001A44994202F1FF3A1AD1D34507D1314672
:105F7800F8B26EF096FF08F101080C36AFE731462B
:105F8800C5F89870D5F89C30E0B263F30402C5F800
:105F98009C206EF086FF10F1160FC8D0441CEAE76B
:105FA800C5F89870D5F8A020013B23F01F0302F034
:105FB8001F021343D3453146E0B2C5F8A030E8D0FC
:105FC8006EF06FFF10F1160FB1D0C5F89870D5F8C4
:105FD8009C209DF808300BF1FF3B62F304038DF819
:105FE8000830D5F8A0309DF808205B0863F3471205
:105FF8008DF80820D6E900321344009323F01F03DC
:106008005B44A3EB0A03013023F01F036946C0B2C7
:106018000393FFF73FFFBEE700ED00E002660A00CA
:10602800DC650A00588809000522044BC3F894204F
:10603800BFF34F8FBFF36F8F704700BF00ED00E0D5
:10604800BFF35F8F0022024BC3F89420704700BF54
:1060580000ED00E010B5034C2278FFF737FF207001
:1060680010BD00BFAAD300202DE9F74F294D8A465D
:1060780006464FF00008AB46274FD0451BDAD6F846
:106088000490B9F1000F3FD03168084601916EF0D5
:10609800FFFE0199044609EB010001386EF0F8FE95
:1060A80084424FF014021D4B08D002FB08F36FF036
:1060B80015024BF8032003B0BDE8F08F14F1160F5A
:1060C8002C60F8D01978A142F5DD02FB08B0C7F8BA
:1060D8009840C7F89840D7F89C4000F10801007B29
:1060E80064F304000871D7F8A0000C79400860F345
:1060F80047140C71D7F89C1021F01F016960D7F87C
:10610800A01021F01F01296108F1010814350C368F
:10611800B3E700BFC857002000ED00E0AAD3002075
:10612800F0B55349534DD1F890302C68C3F3072389
:106138009C4287B000F299800020FFF781FF4E4B08
:10614800C1F8C030844216D14C4D01A82C70FEF71E
:10615800C3FD002607464A4CB74213D100202B78CE
:106168004349D1F89020C2F30722934277DBFFF727
:106178005BFF002046E0696801EB0011FFF772FE43
:106188000130DFE70199300101EB0613DA6822409C
:10619800B2F1807F52D00AD8B2F5001F34D0B2F5E0
:1061A800800F3ED0B2F5801F12D00136D4E7B2F18D
:1061B800006F43D0B2F1805FF7D15A689B680958E5
:1061C800013B22F01F00034423F01F03012032E0AB
:1061D8005A689B680958013B22F01F0003440120BC
:1061E800844623F01F0340EA4C10CDE902218DF8C4
:1061F800100002A928780593FFF74CFE00282ADA38
:106208006FF0150007B0F0BD5A689B680958013B4C
:1062180022F01F0003444FF0020C012023F01F035B
:10622800E1E75A689B680958013B22F01F000344C4
:10623800022023F01F034FF0000CD4E75A689B6834
:106248000958013B22F01F0003444FF0030C0120C2
:1062580023F01F03C7E72B7801332B70A5E7C1F89C
:106268009830C1F8A00001337BE74FF0FF30C9E751
:1062780000ED00E0E88E0900AAFF4400AAD3002040
:106288000000F0FFF0B587B007460E46144600211F
:10629800102268461D4691F08BFC02238DF80230CF
:1062A800054B2A4621466846CDE90476019368F0F5
:1062B800B5FF07B0F0BD00BFE34E070008B5024BBD
:1062C8001B689847002008BDDC570020034B044A90
:1062D8001860937843F0020393707047DC570020EE
:1062E800CC03002008B505486DF0E5F9002383F3D9
:1062F8001188BFF36F8F0423184602DF34660A0043
:1063080008B50549054A21F007010548521A6CF0FD
:1063180086FF002008BD00BF3BC3012000FC07200A
:10632800E05700204FF0FF324FF0FF3301482DF0C7
:1063380023BA00BFDC03002001482DF08FBA00BF4C
:10634800DC03002038B50546FFF7ECFF2A46082194
:1063580007486CF0AAFE044628B925B1FFF75EFD90
:106368000C22044B1A50FFF7E7FF204638BD00BF48
:10637800E05700200C00000038B504460D46FFF732
:10638800D1FF21462B46082207486CF010FF04462F
:1063980028B925B1FFF742FD0C22044B1A50FFF72C
:1063A800CBFF204638BD00BFE05700200C0000009E
:1063B80010B50446FFF7B6FF21460348FDF78AF8F3
:1063C800BDE81040FFF7B8BFE057002070B5A0FB4C
:1063D800015434B92846FFF7B5FF064640B93046A0
:1063E80070BDFFF71BFD0C22044B00261A50F6E780
:1063F8002A46214691F0DCFBF1E700BF0C000000C3
:1064080070B541690446867A0A4D59B1437ADB076B
:1064180006D42C2303FB06535B6A1B689B689847CA
:10642800002363612C20214600FB0650BDE8704024
:1064380075F031BD842100202C22024B02FB003074
:10644800704700BF842100202C21827A054B01FB74
:1064580002339A6A1B7F801A1B3323F00303B0FBB5
:10646800F3F070478421002038B52C24827A064B3B
:1064780004FB02335B6AD3E901240C601568FFF75B
:10648800E3FF04FB005038BD842100202DE9F043D0
:1064980085B00546684690461C46039175F0E5FFB1
:1064A800DDE90067EFF31189202383F31288BFF336
:1064B8006F8F6B8B002B41D02A8B9A4225D90022F3
:1064C800002328462DF01AFA0446F0B189F3118802
:1064D800BFF36F8F039B002B41D032463B46684683
:1064E80075F0E8FF2C21A27A254B204601FB0233E8
:1064F8005B6A03A91B681D68DDE90023A847606182
:1065080070BB2046FFF77CFF24E0698B4B1E6B8332
:1065180089F31188BFF36F8F2B7F2A8BAC6A1B33EB
:1065280023F00303521A02FB0344154B154AEB1AD6
:106538009B105343A3722B7FE372CBE789F3118837
:10654800BFF36F8F2346424628462DF0D7F90446FD
:106558000028BFD10024204605B0BDE8F083636160
:10656800012300252381039B29466382E27A656023
:1065780004F1180091F01CFB63692582E360EAE7E7
:1065880084210020A38B2EBAF8B500242C260F4DA9
:1065980000B9F8BD476800F10802D2E8EF3F591E7C
:1065A800C2E8EC1FBCF1000FF7D1DBB2012BF0D130
:1065B800837AC46006FB035344601B6A13B198478F
:1065C8003846E5E7FFF71CFFFAE700BF8421002003
:1065D8002DE9F84F06460D4617460446A34664685B
:1065E800002CFBD14FF02C09DFF878A0BBF8103055
:1065F800BBF81220DBF81410D21ADBF80C300BF1C0
:106608000C005B1AD21AAA4228BF2A461FFA82F83F
:10661800394642466EF012FDB5EB0805444447443E
:106628001DD00C9B53B1DDE90A010D9A98478346AA
:10663800A8B1014630466EF0C3FCD7E7B07A09FB33
:1066480000A0436A9B6843B1AB4228BF2B4619465A
:10665800DDE90A23FFF71AFFE9E72946F8E72046AC
:10666800BDE8F88F8421002008B5244A244B1A601D
:1066780028F0A2FC4FF47A612248D0F82436C3F3FC
:106688000802C3F309434B4382F480721E498832DF
:1066980001FB02334FF4FA215B00B3FBF1F201FB7B
:1066A80012331A49B3F57A3F28BF0132C1F80429D9
:1066B800D0F820364FF47A60C3F30802C3F30943D5
:1066C800434342F21C5082F4807202F2172200FB0C
:1066D80002334FF47A701B0AB3FBF0F200FB12335B
:1066E8000020B3F5FA7F4FF0010328BF0132C1F84B
:1066F8001C27C1F80009C1F8003608BD0020A10711
:10670800B810002000C0FF00F82A008000001250D6
:1067180048B1054B054A1B68B3FBF2F35843044BD9
:1067280043F0010318477047B810002040420F009B
:10673800908A0900BFF34F8F0549064BCA6802F4D7
:10674800E0621343CB60BFF34F8F00BFFDE700BF8C
:1067580000ED00E00400FA05F7B506460D461446BC
:10676800124F384675F070F9E0B1BB6831463846CB
:106778001B68AAB29847002802DB002003B0F0BDCE
:10678800002CFBD1AC42F8D22F1B042F28BF0427C2
:1067980074F0AEFC3A46019001A9301991F0E2F983
:1067A8003C44EFE76FF01200E8E700BF0C830900F4
:1067B80038B504462DF05AFF20466EF0A9FCA069B2
:1067C800C8B194F86C30DB070DD50221154A16487C
:1067D8006EF09CFC6FF07705201D6EF0A0FC2DF08C
:1067E80059FF284638BD75F02FF938B901210F4AED
:1067F8000D486EF08BFC6FF01205EDE7204600F0B7
:10680800B5FF05460028E7D10146242204F12800F7
:1068180091F0CEF994F86C3043F0010384F86C30B1
:10682800DAE700BF50660A00F08809007A660A00B5
:1068380070B504462DF01AFF20466EF069FC94F8F6
:106848006C30DA070DD40221254A26486EF05EFC2A
:106858004FF0FF35201D6EF062FC2DF01BFF28461F
:1068680070BDC3F340019B0707D502211E4A1D488E
:106878006EF04CFC6FF07705ECE7A06972F0E2FE71
:106888000646A06972F06EFF054628B10121174A35
:1068980014486EF03BFCDDE7A36F4BB13146204650
:1068A8006EF017FE0546A0B1A06972F083FFD1E72C
:1068B800A06972F0FFFEA0670028EFD101210C4A01
:1068C80008486EF023FCA06972F074FF6FF00B05A6
:1068D800C0E794F86C3043F0020384F86C30B9E7F1
:1068E8009D660A00F0880900C3660A00E9660A0086
:1068F80005670A0038B590F86C3004469B0708D441
:106908000221144A14486EF001FC6FF077052846FE
:1069180038BD6EF0FDFB0021204601F0C1F820B122
:1069280001210E4A0C486EF0F1FBA06972F042FF9B
:10693800054620B101210A4A07486EF0E7FB94F8A2
:106948006C30201D23F0020384F86C306EF0E7FBF6
:10695800DDE700BF21670A00F088090048670A00E0
:1069680066670A002DE9F04385B006460C46904656
:106978006EF0D7FB0546B8F1000F07D030466EF031
:10698800D5FB012810D1B5FA85F56D0901342946E2
:106998003046E2B26EF0B6FD814650B90121234679
:1069A800324A33486DF02CFF0024204605B0BDE87C
:1069B800F0834768B8F1000F09D03868796801ABEF
:1069C80003C33A7A01AF1A7007238DF80530F18DA9
:1069D8007B883046994228BF19466EF0E5FE04468A
:1069E8000028E1D0038A428A4169D21AC36800F1BB
:1069F8000C085B1AD21A3B7839469A4228BF1A46C5
:106A080040466EF01BFBD9F80C90B9F1000F08D185
:106A1800218AF38D9942C8D94046C91A6EF035FBD0
:106A2800C3E7D9F8040083681B6B13B9D9F8009041
:106A3800EBE7294698470028F8D0071F57F8041FA6
:106A48000029F3D008780028F0D0628A238AA2EBC4
:106A5800030C6269E3689B1AACEB0302904294BF93
:106A6800024692B240466EF0E9FAE7E796670A00F6
:106A7800D088090038B50446806F6EF089FA05465B
:106A88006EF03FFA2046294601F052FA044638B122
:106A980004480121044A6DF0AAFE2846FFF774FD58
:106AA800204638BDD0880900BC670A0038B5802167
:106AB8000446806972F021FE054678B101462046F9
:106AC80001F036FA044638B106480121064A6DF04D
:106AD8008EFE2846FFF758FD204638BD6FF00B04A0
:106AE800FAE700BFD0880900DB670A0000232DE918
:106AF800F04F93B005930B7E044633F080060F46A3
:106B080015460AD00121AD4AAD486DF070FE6FF010
:106B18000406304613B0BDE8F08F82B10846FFF78F
:106B280033FD7B7EDA0704D49D07F2D53B7E002B2C
:106B3800EFD1204613B0BDE8F04FFFF79BBF4A7E68
:106B480000F12809900705D5802B09D13846FFF7B1
:106B58001BFDDEE7910700F03884002B40F03584F8
:106B6800D3071ED53B8A082B12D1FA683946136819
:106B78000020A3625368C9F804306EF033FA059018
:106B880080B18F4801218F4A6DF031FE059805E0EC
:106B98008B4801218C4A6DF02AFE3846FFF7F4FC39
:106BA8001EE00597FFF73AF9002394F82850874A22
:106BB80015F0600F8350C5F341131CD0032B40F030
:106BC80064836FF08505FFF729F9804B1B58002B6C
:106BD80000F0A183002D00F0698305980028DDD11D
:106BE80048466EF0D6FB0346A069002B00F02884C7
:106BF800802100F02EBC48466EF0CBFB94F829307B
:106C0800002840F02C81013B0A2BDAD801A252F867
:106C180023F000BF5B6D0000CB6B0000E16D00004E
:106C2800CB6B0000496C0000CB6B0000CB6B000005
:106C3800CB6B0000AF6C0000CB6B0000236D000035
:106C4800A069618D03697F2993F88030B9D8A28D36
:106C5800002AB6D1E28D002AB3D1EE06B1D194F85C
:106C68003020022A02D14FF0FF35ACE71D070BD5C3
:106C7800C9B26EF0C4FB054648B1638D0121544A80
:106C88004F486DF0BDFD9EE7012384F8393094F834
:106C98003030012B05D1638D1BB984F830300025C5
:106CA80091E70123F9E720466EF03BFA628D014631
:106CB800FF2A86D8E38D002B83D194F82830D80694
:106CC8007FF47FAF94F83030002BCCD092B9618D2F
:106CD80094F838308B42E2D02046C9B200F0E0FE8A
:106CE800638D054668B1012100903A4A34486DF039
:106CF80091FD68E72046D2B26EF02AFC0028E6D162
:106D0800B1E7002B14BF02220122052184F83020AC
:106D180020461A466EF091FDC1E705F01F05012DCA
:106D28007FF44FAFE38D002B7FF44BAF628DFF2ACA
:106D38003FF647AFA18DFF293FF643AF94F83030B7
:106D4800022B90D12046D2B2C9B26EF0B1FC0546F2
:106D580039E7E38DA68D002B7FF433AF94F83030FC
:106D6800002B80D0012B02D1002E7FF47CAF15F0D0
:106D78001F0515D0022D92D1B4F82A80B8F1000F62
:106D88008DD1F6B23146204601F03AF9421C05464B
:106D98003FF419AF4246314620466EF000FB12E739
:106DA800002E7FF460AF638D012B7FF478AF94F8E9
:106DB8006C3066F3C30384F86C3070E7FE670A0032
:106DC800D088090036680A001F680A000C00000015
:106DD80058680A007A680A00A38DE28DDEB2002A9C
:106DE8007FF4EFAE628D022A11D105F01F053543FD
:106DF8004FEA13217FF4E5AE0122A0696EF0DFFAB5
:106E080000287FF4DEAE012384F8393047E794F890
:106E1800301000293FF427AF012902D1002B7FF45D
:106E280022AF15F01F050FD0022D7FF438AF002ACE
:106E38007FF435AF3146204601F0C0F8431C0546C3
:106E48003FF4C1AE0122A6E7002B7FF40CAF012A64
:106E58007FF425AF94F86C3043F00803ABE70A2BB6
:106E680063D8DFE813F00B00620062006200620082
:106E780062003A006200DD016200F201E38D022B3C
:106E880053D194F83030002B4FD0012BA18D01D174
:106E980000294AD115F01F050ED0022D17D0002663
:106EA800022120466EF080FC054618B131460C30B0
:106EB8006EF0D5F80595F2E6002936D194F86C30D5
:106EC8009E0806F00206C3F300131E43E8E72046B7
:106ED800C9B26EF08DFC0646E2E7618DED064FEA19
:106EE8001123C9B207D0002320460AA90A936EF0DD
:106EF8009FFA0A9DDEE7013B0E2B16D8DFE813F058
:106F08000F003000380015001500D20036001500BB
:106F18001500150015001500150015000F01204675
:106F28006EF0FFF818B1012818D00025C2E7266FC7
:106F3800002EFAD0B4F82E8033782046984528BF22
:106F4800984641466EF030FC05460028B2D04246CD
:106F5800314605F10C006EF071F8ABE7666FE7E7B4
:106F680000222046FFF7FEFC0546A3E70122F8E7CA
:106F78000A46204603216EF060F980460028D4D0E6
:106F88006EF002FAE58D98F81530B8B998F81460E3
:106F98008DF82930AE428DF8286028BF2E46D8F8E3
:106FA800103031461B882046ADF82A306EF0FCFBC5
:106FB80005460028B9D032460AA9CAE74FF0000AA8
:106FC800B44A8DF81130D8F808308DF810A01A405E
:106FD800B14B9A4255D1102106A828F0C5FE061ECD
:106FE80036DB0AAB102E984628BF1026AB4806AAF7
:106FF800564503F1020334D8B6000236F6B28DF8CE
:107008001060AE4228BF2E46204631466EF0CCFBBB
:107018000546002889D0022EB34628BF4FF0020B40
:107028005A46A6EB0B06C34600F10C0A504604A9C3
:107038006EF004F8730808EB56025A4528D1F00799
:107048007FF538AF504618F803106EF000F831E7B6
:1070580058367FF46AAF0121914A92486DF0C7FB18
:1070680063E712F8011B0AF1010A4FEA111C01F04B
:107078000F0110F80CC0415C03F802CC03F8011CA6
:10708800B6E798F81460D8F810808DF81060B8E763
:1070980050461BF8011BCDE902236DF0E0FFDDE946
:1070A8000223CAE720466EF03CF8D4E91C530028B6
:1070B80008BF1D460A2300268DF8283006232046DF
:1070C800CDF82A60CDF82E608DF829306EF02EF8B4
:1070D80001287FF42AAF002D3FF4ECAE6B882046E0
:1070E800ADF82A302B798DF82C306B798DF82D304E
:1070F800AB798DF82E30EB798DF82F306B7C8DF8CD
:107108003030E68D9DF828309E4228BF1E46314615
:107118006EF04AFB054600287FF44DAFCAE62046CC
:107128006DF0FFFF20B101287FF4FFAE636F00E030
:10713800236F002B3FF4F9AE5B88B3F5007F7FF631
:10714800F4AE594B04F14C060A9300238DF82C3009
:10715800E36C9E4208BF0023BDF82A2093B1597DF5
:107168000F2908D1197D0A44ADF82A209DF82C2052
:1071780001328DF82C20226D9A4201D01B68EBE772
:10718800BDF82A20B4F82E802046904528BF9046A6
:1071980041466EF009FB054600283FF4C6AE9DF84F
:1071A800282000F10C0A424528BF424650460AA949
:1071B8006DF044FF9DF82830434594BFA8EB0308C1
:1071C800A8EB0808B8F1000F3FF474AED4F84CB03F
:1071D800B3453FF46FAEBBF1000F3FF46BAE9BF8C5
:1071E80015300F2B15D19BF814205046424528BF67
:1071F8004246DBF810106DF021FF9BF81430434530
:1072080094BFA8EB0308A8EB0808B8F1000F3FF4F7
:1072180051AE236D5B453FF44DAEDBF800B0DAE7C5
:1072280094F83030002B3FF480AEE18D01297FF4D3
:107238007CAE94F8386020466EF0B6FA0546002811
:107248003FF438AE31460C30FFE605F01F05012D3E
:107258007FF46BAE20466EF069F900283FF465AE06
:10726800A38D4268FF2B3FF660AE12799A42FFF475
:107278005CAEDAB20F2A3FF658AEE18D01297FF4F1
:1072880054AE234493F83A60D5E7204605A96EF03A
:10729800CFF85CE500FF02000003020068B50A00B1
:1072A8009D680A00D0880900050F050075F0DBF815
:1072B8004FF47A76A0FB060C47F61222002306FB51
:1072C80001C1F9F729FF654BD3E8AF1F41F28732B7
:1072D800461A9642624A39D9D3E8EF6F8E4204D1F2
:1072E800C3E8EC0FBCF1000FF6D12FD1D2E8EF3F85
:1072F800C2E8E15F0029F9D123B10221594A5A486D
:107308006DF07EFA0221594A57486DF070FAFEF77F
:1073180085FD574B1D58002D7FF45FAC7B7EE28DB9
:10732800D9071BD548466EF034F8B8B9BAB1294622
:10733800A06972F0CEF90146059000283FF450ACE0
:10734800204613B0BDE8F04F00F0F2BDD2E8EF3FA1
:107358000133C2E8E13F0029D9D0F7E73AB920461E
:10736800FFF7A4FB00287FF43BACFFF7E2BB4846DD
:107378006EF00FF8059D18B92846FFF705F9EEE7F6
:10738800002D3FF42DAC2946204600F0D1FD08B170
:10739800284603E4A069036993F8801011F00401FA
:1073A8007FF4C7AB72F0A9F9054600283FF418AC82
:1073B8000146204600F0BCFD00283FF4BAAB01218D
:1073C8002C4A29486DF013FAE2E752077FF508AC1A
:1073D800002B3FF4BBAB3846FFF7D6F894F83930AA
:1073E800002B3FF496AB94F82930052B0CD1618D16
:1073F800A069C9B26EF003F8054628B1638D012172
:107408001D4A19486DF0FCF994F82930032B11D165
:10741800638D022B0ED1A18D00220E0A3146A06980
:107428006DF0CDFF054628B101213346134A0E48B9
:107438006DF0E6F900232E4684F83930FFF769BB72
:10744800E38D002B3FF4D4AB0599003918BF012117
:10745800C90172F055F8FFF76CBB00BFF057002068
:10746800EC570020BF680A00D0880900D3680A00DA
:107478000C000000FC680A0058680A0020690A002D
:107488000B7810B4062B14D10369D3F89C20EFF3C2
:107498001184202383F31288BFF36F8F00204B6879
:1074A8001860506A60B9C2E9083384F31188BFF3E1
:1074B8006F8F0022002304485DF8044B74F0DBBB97
:1074C80003605362F1E700BFE820002030B589B0BF
:1074D800002200230024CDE906236FF007034FF4B0
:1074E8008062CDE90334CDE90144154B1549009478
:1074F80015482CF0BFFD1549134874F057FE144B7E
:1075080014498B4207D30020134B14498B420CD3E8
:10751800002009B030BD03F11402D2E8EF0FC2E831
:10752800E54F002DF9D11833EBE703F11402D2E847
:10753800EF4FC2E8E50F002DF9D11833E6E700BF99
:10754800C175000058DD0020602D002055AA0A00F2
:10755800102400207024002070240020D024002053
:1075680038B50D466DF0E2FF30B90121BDE838406D
:107578000F4A10486DF03BB9C46804B938BD2B7880
:10758800032B05D0052B0ED0022B08D02468F4E776
:10759800606883685B69002BF8D09847F6E76068F5
:1075A80083689B69F7E760688368DB69F3E700BF76
:1075B80047690A00E08809002DE9FF4120274FF0BC
:1075C800FF334FF0FF32644801A92CF071F8039B98
:1075D8001B69D3F89C40236A93B1EFF3118287F3B8
:1075E8001288BFF36F8F216A29B1606A0B688142E4
:1075F800236208BF636282F31188BFF36F8FC9B932
:107608009DF80430062BDAD0072BD8D801A252F8FF
:1076180023F000BF617600005576000089760000EF
:1076280067760000BD760000AB760000C7750000E5
:10763800517700000B7E20465D06D1F81E2002D14E
:10764800FFF754FAC7E76DF0C1FFC4E70022012134
:1076580020466EF0F2F8B2E700221146F8E794F8F7
:107668006C3043F0040384F86C3094F83030022B0B
:1076780003D1204601A9FFF773FF00220321E7E7A2
:1076880094F86C3023F0040384F86C3094F83030AC
:10769800022B03D1204601A9FFF762FF0022022135
:1076A800D6E794F83030022B89D1204601A9FFF79C
:1076B80057FF84E794F86C30A66923F0040384F834
:1076C8006C30D6F808803369A033D3E8AF3F9A0707
:1076D8001ED53046D8F83C309847D8F824300021D9
:1076E800304698470546D8F840303046984795B117
:1076F8001A4A01211A486DF07AF80022042120461E
:107708006EF09BF8002D3FF45AAF2A4607219FE7F9
:107718004FF0FF35ECE72946204600F0C1F9054651
:1077280008B1104AE5E7A06972F006F8831E5842CE
:10773800584194F86C3084F8305023F0680343EAD9
:10774800401384F86C30D8E70121074A04486DF0EB
:107758004EF80621029A7BE7E820002076690A00A5
:10776800E0880900A4690A00D0690A0038B5024611
:1077780005460C49806972F03DF8044630B1012194
:10778800094A0A486DF033F8204638BD85F83800B4
:10779800284600F043F904460028F5D0A86972F09D
:1077A80058F8F1E789740000E0690A00E0880900E8
:1077B800F8B501231D460C68002C35D063F07F0214
:1077C800D6B202F07F02103224FA02F7FF0716D56C
:1077D800046824FA02F7FF0708D433461348012146
:1077E800134A6DF00DF86FF01500F8BD05FA02F2B6
:1077F80024EA020404600C6824EA02040C60DC40F9
:10780800E6070ED5026822FA03F4E40700D4E5E798
:1078180005FA03F422EA040202600A6822EA040272
:107828000A600133102BC6D10020DEE71089090059
:10783800076A0A002DE9F04F0026536891B0D46812
:107848000A900891069202930E96039674B9039BC8
:10785800029A09339BB293701B0AD370069B167168
:10786800DC68002C40F0C780A346AEE04FF0000A69
:107878006068CDF83CA083681B6B002B00F0AC80DF
:1078880008999847002800F0A7803546C4E903AA5C
:10789800A0F1040959F8043F0BB11A789AB9B54216
:1078A80040F29780E3680F9A1343E3606068836847
:1078B8009B6A002B00F0928098478346002800F0CE
:1078C8009080534A7DE05A780B2A08BF9D70D9F8FA
:1078D80000305A78042A10D1E2680F990A43E2600E
:1078E800DA78002A5CD101229D702369AA401343EB
:1078F80001352361EDB2CDF83CA0D9F800707B7852
:10790800052BC7D16FF0120B4FF001080A9B9B693A
:10791800099379793A790E9B42EA0122ADF836202B
:1079280097F902205FFA88F1002AACBF424641F07D
:1079380080010493B7BF4BB24FFA88F321F080025D
:107948000793A8BF0793049BB8BF103223FA02F02D
:10795800C0072CD40F9B23FA02F20593D30726D431
:10796800BB79FA78099800930DF136030B9171F001
:107978003DFD0B998346D0B9079BB970002B4FF09A
:107988000103BCBF21F0800110318B400498059998
:10799800BDF8362019431843CDE90E01BA8079E7BE
:1079A8006A1E9A700FA90EA8FFF702FFA3E708F155
:1079B8000108B8F1100FACD1BBF1000F3FF46AAF6A
:1079C800144A012114486CF012FF584611B0BDE862
:1079D800F08F6FF0150BF3E7354667E76FF0850B0F
:1079E8006FE7606808996DF0C1FD039B2E4603445C
:1079F800246803932AE7E36804F10C01A3600EA846
:107A0800FFF7D6FE08B924682BE76FF0150BDCE703
:107A1800486A0A00246A0A001089090070B5836957
:107A280005461B69026F93F88030C3F34113022B9C
:107A38000CD0032B0CD0012B0CBF10230823D371BF
:107A4800EE6D3EB96E6DBEB9344611E02023F6E7FF
:107A58004023F4E7324601212846FFF7EBFE0446AF
:107A680040B173685B790B4A01210B486CF0C8FE82
:107A7800204670BD3668E4E7324600212846FFF705
:107A8800D9FE044618B173685B79044AECE7366896
:107A9800D9E700BF6C6A0A00108909008F6A0A00DA
:107AA8002DE9F04105460E466DF03BFB95F8383060
:107AB800804633B328466DF039FD0746F0B10146DC
:107AC80028466DF0A3FD10220446002105F13A0076
:107AD80090F06EF8002385F83830FF683FB984B11C
:107AE80019491A486DF001FD2046BDE8F081786813
:107AF80083685B6A03B198473F68EFE76FF03C041F
:107B0800EEE71EB985F838600024EDE732464146B5
:107B180028466DF0F7FC074690B1024628466DF0FE
:107B28009FFD04460028DFD185F83860FC68002CEA
:107B3800EAD0606883681B6A03B198472468F6E74F
:107B48006FF03C04D0E700BF48670A00C888090006
:107B58002DE9F04105460F461446D2F804806DF031
:107B6800C8FC95F86C30D9070BD5474947486DF0E4
:107B7800BCFC6FF00F07281D6DF0C2FC3846BDE84D
:107B8800F081012F0AD128466DF0D0FA30B940496A
:107B98003E486DF0AAFC6FF08507ECE798F80730CF
:107BA8009A0607D5AB691B6993F880309B0701D407
:107BB8003849EDE71FB1012F06D03749E8E7EB6DEB
:107BC8002BBB05F1540603E06B6DABB905F15C0600
:107BD800002233680BBB002FD5E91C2308BF1346CE
:107BE8005B7C626803F10103DBB25371D5E91C12B7
:107BF80008BF0A46537422E09C4206D1274923480D
:107C08006DF073FC6FF01507B5E71B68DDE79C4264
:107C180001D12349F3E71B68D2E79C4221D12368AD
:107C2800CAB972683360944200D17360002323603C
:107C380063685B7902211B4A14486CF0E1FDA16876
:107C4800B9B128466DF013FB074668B116490F48CD
:107C58006DF04BFC8FE7136073689C4208BF72603D
:107C6800E4E71A461B68B5E7A0686DF08DFB88F855
:107C780006000023236073681BB9C6E90044002787
:107C880079E71C607460FAE7E06A0A00C8880900AE
:107C9800026B0A00BC6A0A00206B0A00406B0A00EB
:107CA8005D6B0A007A6B0A00976B0A00F8B5054607
:107CB80000AF29B301290BD1184C194E2BE063688A
:107CC80028461968F9F782FAB8B11834B442F6D3DD
:107CD8006C4688B06A46134BCDE905354FF40073FE
:107CE800ADF81C30104B42F8103F00234FF4E2511E
:107CF8000E48FCF759FDA54600242046BD46F8BDB0
:107D08000B4C0C4EE2E7636828461968F9F75EFAEF
:107D18000028F2D01834B442F5D3D9E770240020F3
:107D2800D0240020CE6B0A0003000001D888090087
:107D3800102400207024002070B5012501F07F0375
:107D480011F0800F18BF10339D4090F83030044672
:107D5800022B06D001210C4A0C486CF048FD00208B
:107D680070BD90F838606DF0DCF932460146204667
:107D78006DF0C8FB0028F2D0C0680028EFD08368F7
:107D88001D42EDD10068F8E7EC6B0A00D8880900BD
:107D98002DE9F84305460846114616469846FFF76A
:107DA80085FF0446002843D028466DF0D8FB95F897
:107DB8006C30DA0702D5204A012109E0D4F8049092
:107DC80004F11407D7E8AF3FDB070CD502211B4AA3
:107DD8001B486CF00CFD6FF00F04281D2BF03EFDC6
:107DE8002046BDE8F883D9F804301BB1AB4201D076
:107DF800144AE1E74246314628466DF083FBA0B1BC
:107E08000023236003696BB9C0E90344D7E8EF3F57
:107E180043F00103C7E8E23F002AF7D10024C9F87C
:107E28000450DAE71C600461F0E76FF03C04D4E723
:107E38006FF01204D4E700BFE06A0A00116C0A0070
:107E4800D8880900336C0A002DE9F04F83B000AFE1
:107E58007B6097F830304C680E463B608146904610
:107E68006DF05FF9A36801461B6B33B96FF0150419
:107E780020460C37BD46BDE8F08F204698470028BD
:107E8800F4D00024051F06F10C0A55F8041F09B1A7
:107E98000B782BB9002C14BF00246FF03C04E7E7E3
:107EA8004B78042B0ED1002C3CD18B787A68934206
:107EB800EBD1CB783A689342E7D10B79002BD7D036
:107EC8000124E2E7052BE0D1002CDED0B8F1010F48
:107ED80091F802B009D0B8F1020FF1D152465946D3
:107EE800D9F818006DF04AFC04E05246D9F8180099
:107EF8006DF028FC04460028E2D06D468AB06A4638
:107F0800F368CDE907B3062307490990CDE90518B9
:107F180042F8103F00234FF441510448FCF744FC59
:107F2800AD46A5E70024A3E7736C0A000889090099
:107F38002DE9F0410B7E0C465906054637D16BB347
:107F48006DF02FF940B11B4801211B4A6CF04FFC22
:107F58004FF0FF30BDE8F0812846D5F87080268ABA
:107F6800EF8D6DF0DEF8F8B1421E534253419B018C
:107F7800228A9AB1BE42324628BF3A46E98D9142DA
:107F88000CD9B2FBF3F103FB11223AB994F918307A
:107F9800002BBEBF637E43F0080363762146A869C1
:107FA800BDE8F04171F008BB98F80730E0E76FF0E2
:107FB8001500CFE7F8880900AF6C0A0070B50646CF
:107FC80080690C4671F09CFA054638B102212346B7
:107FD800094A0A486CF014FC284670BD012214F0C6
:107FE800800F18BF24F08004736B18BF1034A240B0
:107FF8001A437263F0E700BFC36C0A00F8880900EF
:1080080070B5054680690E4671F0A5FA044638B188
:1080180002213346054A06486CF0F2FB204670BD43
:10802800314605F134006DF07FFBF7E7DA6C0A00A2
:10803800F888090070B50646EFF31181202383F311
:108048001288BFF36F8F1B4D2A6881F31188BFF325
:108058006F8F526892F86C20D20705D4BDE8704043
:10806800202200232BF056BFEFF3118283F31288EE
:10807800BFF36F8F2C682CB1696823688C422B6022
:1080880008BF6B6082F31188BFF36F8F44B16068DB
:1080980004F10801C36998472146074873F088FD31
:1080A8002B6833B13046BDE87040002200232BF026
:1080B800F9BE70BDF45700206020002030B585B0AF
:1080C800CDE90012054600220023144803A92BF02D
:1080D80055FA0246E8B9DDE90001039B5D60083303
:1080E80083E80300EFF31180202383F31288BFF3A2
:1080F8006F8F039B1A600A4A516861B9C2E900335D
:1081080080F31188BFF36F8F0022002305482BF0FE
:10811800C9FE05B030BD0B605360F1E76020002058
:10812800F45700200000002073B5202504698DF85D
:108138000710EFF3118685F31288BFF36F8F0122C2
:10814800206C0DF107016BF031FF86F31188BFF346
:108158006F8F012812D074F023F8C8B10122104B98
:10816800D3E8EF1F002903D1C3E8E02F0028F7D197
:1081780004D102210B4A0C486CF039FB237F2BB148
:108188002022002304F148002BF08CFE02B070BDC1
:10819800A37E002BE2D00021202074F009F9C8E763
:1081A800FC570020046D0A00C088090038B5002477
:1081B80005690E492B6C05F14800C3E90144DC60F0
:1081C800AB6BC3E90144DC6073F092FF05F1780002
:1081D800074973F030FF074905F1280073F02BFFBA
:1081E80028466DF04FFB204638BD00BF21830000B4
:1081F80069840000358500002DE9F34103690646CE
:108208000D46D0F804801C690F7E002A32D00B8AF4
:1082180071323E480BBF022101213D4A3D4A00937D
:108228003B466CF0F7FA30462F7E6DF09FFB874295
:1082380004D1042104F188006DF04CFC30462F7EF7
:108248006DF0A2FB874204D1052104F188006DF08E
:1082580041FC30462F7E6DF07BFB874203D104F151
:108268008C002BF0E3FB2946404602B0BDE8F04104
:108278006DF0BBBA6DF07AFBB84214D12A8AE9686E
:10828800A06B6BF093FE28B1236A1BB104F12800A0
:108298002BF098FD04F1880004216DF01BFC04F11B
:1082A80078002BF08FFD30462F7E6DF06DFB8742F6
:1082B80015D1236A1BB104F128002BF083FD052199
:1082C80004F188006DF006FC237F9BB9002340F67B
:1082D800354204F148002BF0E5FD012323773046B1
:1082E8002F7E6DF035FB8742BDD104F18C002BF059
:1082F8003BFBB8E7236C5A89DB889A42EFD000220F
:10830800002304F148002BF0CDFDE8E7C088090000
:10831800236D0A00476D0A002DE9F04750F8483CE4
:1083280000F140075B68054600213846D3F8009005
:108338006DF008FB002864D0012138466DF002FB7F
:10834800804600285DD155F8083C5A89DB889A4256
:1083580003D115F82D3C002B53D0D7E8EF4F44F04C
:108368002003C7E8E23F002AF7D114F0200448D1DF
:1083780048466DF009FB00228246002322486CF033
:10838800C5FD064650B9384605216DF0A3FB2846C1
:10839800BDE8F047202200232BF084BD80F818A008
:1083A80015F82C3C33B1428AC16855F8080C6BF0BB
:1083B8001DFE0446214606F10C006CF039FE5CB146
:1083C800D9F804006DF064FBB4FBF0F303FB104430
:1083D800B4FA84F84FEA58183146484605F82D8C07
:1083E8006DF0EBF968B10121084A09486CF0FFF912
:1083F8003046FEF7C9F83846BDE8F04705216DF06C
:1084080069BBBDE8F08700BFDC210020686D0A0069
:10841800C088090038B503461B6940685D68AC68C8
:10842800A37A84F8223094F82D3084F82330A37688
:10843800696849B1237C3BB96CF019FF30B101215F
:10844800054A06486CF0D3F9002038BD68686CF01E
:108458009BFF2074F8E700BF7A6D0A00C088090006
:1084680070B550F8782C00F11004526803460021CA
:10847800204615686DF066FA00284DD00121204687
:108488006DF060FA002847D153F8402C686893884B
:10849800918916695B1A9BB2F61A6DF0F9FAB04227
:1084A8003AD8D4E8EF3F43F01002C4E8E12F00299E
:1084B800F7D1DB0606D5BDE870400221174A1848F7
:1084C8006CF095B928466DF051FA00220646002353
:1084D80014486CF01BFD0446F0B1067668686DF030
:1084E800D7FA638A984203D268686DF0D1FA83B2EA
:1084F8002146284663826DF060F968B128466DF020
:1085080035FA034606480121074A6CF079F92046F6
:10851800BDE87040FEF738B870BD00BFA46D0A0012
:10852800C0880900DC210020C46D0A0038B550F865
:10853800083C044633B9BDE8384001212A4A2B4893
:108548006CF055B950F8283C00F160055B680221D1
:108558001A6800238382838328466DF0F3F9B8B143
:1085680054E9023110699847637D1BB104F150004A
:108578002BF028FC052128466DF0E4F998B9637FB3
:108588006BB10022002304F120002BF08BFC0AE0E1
:10859800032128466DF0D6F90028E1D1E4E714F864
:1085A8000D3C002BEDD1022128466DF0CBF938B1F6
:1085B8002369DA885B899A4202D020462BF002FCB4
:1085C800032128466DF0BEF960B1A26993889189AC
:1085D80012695B1A9BB29A4204D02046BDE8384023
:1085E8002BF0F0BB38BD00BFE96D0A00C088090058
:1085F800D3B5002600270446CDE9006705486CF08E
:1086080089FC28B1230658BF0023047658BF03828B
:1086180002B0D0BD102300202DE9F04383B0002321
:108628004FF0010805691C4C1C4E02AF28602B77DF
:1086380085F8203005F12409B442234601D30020EF
:1086480019E095F820201034CAB16C4688B01B6830
:1086580002AA1349C2E905134FF400739383114B1F
:1086680042F8103F104800234FF4E251FCF79CF801
:108678006FF00B00A5460437BD46BDE8F08385F8CA
:10868800208054F8043C4846009354F8101C54E9E0
:1086980003236DF0EBFCCFE7CC420B00DC420B0070
:1086A8004B6E0A0003000001188909001FB5CDE9C7
:1086B800010103924FF0FF324FF0FF3301A9034845
:1086C80073F0D9FA002005B05DF804FBB82000204B
:1086D8001FB500230190CDE902334FF0FF324FF070
:1086E800FF3301A9024873F0C6FA05B05DF804FB30
:1086F800B82000202DE9F041044617460E460068D0
:108708006DF01CFB31463A468046FFF771FFD4F8FE
:108718007B300546DB1B0146C4F87B3020686DF0D2
:108728004CF888B10B4A434601210B486CF068F8B5
:10873800314620466DF0CDFB2846FDF725FF204643
:10874800BDE8F0416DF091BBA37F0133A377BDE88D
:10875800F08100BFC46D0A00188909002DE9F84F9F
:10876800044600686DF0FFFA4FF030090746E37FD2
:10877800012B1ED82368D3F810B0D3F804A09BF8B7
:10878800616009FB06B6243630466DF095FC31462B
:108798000246804650466DF0FCFA9BF81F300546AD
:1087A80033B1A8EB0002314650466DF0F2FA0546A7
:1087B8000DB9BDE8F88F20466DF0A8FA2A460146A3
:1087C80006463846FFF714FF0546014620686CF058
:1087D800F4FF80B101213B46094A0A486CF010F8C1
:1087E8002846FDF7D1FE314620466DF072FBBDE804
:1087F800F84F6DF03ABBE37F0133E377B7E700BF8B
:10880800C46D0A00188909002DE9F04FB94F89B0E5
:108818004FF0FF324FF0FF33B74805A92AF048FF61
:10882800059E069D3469002D40F09080257704F15F
:10883800240694F820309D42C0F2828004F1180387
:10884800D3E8EF2F22F00202C3E8E12F0029F7D185
:10885800D3E8EF1F21F00401C3E8E21F002AF7D193
:1088680004F11803D3E8AF3FDB07D1D5237F022BF0
:1088780000F08E81032B00F0878153BBDDF814A034
:10888800DAF81050EB7F23BB50466DF06CFA814646
:1088980028466DF03BFA4FF40072014606464846FA
:1088A800FFF7A6FE8046014650466CF086FF00287A
:1088B80000F0668101214B46904A91486BF0A0FF79
:1088C8004046FDF761FE314628466DF002FB6DF02B
:1088D800CCFAA37F002B9BD1237F012B40F07D8115
:1088E800302304F1630694F86150304694F862101E
:1088F80003FB054500F060FA24350246314623693A
:10890800284600F077FA0646C4F8840028466DF039
:10891800C9FB814628466DF0CAFB804628466DF0A3
:10892800CBFBE26D3044002A40F03B81002840F048
:10893800338128466DF0E7FB003818BF01202CE191
:1089480030466DF0A6FB0135303672E7DDF81C8045
:10895800D6F804A095F81890B8F1000F21D02B8A0A
:1089680018F1710F6648009308BF02214B4616BFE5
:108978000121644A644A6BF04DFF304695F818802F
:108988006DF0F1F9804540F0EF80E37F013BE3773C
:10899800204669696DF09DFA294650466CF025FF1E
:1089A8005EE730466DF0DFF9484540F09580237F5B
:1089B800D5F80C80B5F810B0002B49D1BBF11F0FCA
:1089C80042D1D8F80030BB423ED1414604F15403AD
:1089D80008F11C0251F8040B914243F8040BF9D139
:1089E8000A881A808A7842219A70552384F873304D
:1089F800532384F8743084F87630A36DE26DC4F89C
:108A080077300023C4F8803094F86030C4F87B20B5
:108A18009A0684F875100FD194F8612094F82030E4
:108A28009A4209D294F86230013B0F2B04D80123F3
:108A380084F87F302377A0E720686DF08AF9022355
:108A480084F87F300423F5E720466DF00EFA94E7AA
:108A5800032B92D1302394F8619003FB0949D4F891
:108A6800803009F124095B44C4F88030BBF1000F61
:108A780016D048466DF020FB90B141465A4648460C
:108A88006DF02CFB804628B902215B461F4A1C4822
:108A98006BF0B6FED4F87B30A3EB0803C4F87B3048
:108AA800D4F88020E36D9A420DD248466DF004FB5D
:108AB80000287FF462AFD4F88020E36D9A4202D296
:108AC80020686DF05CF948466DF01DFB003818BF52
:108AD800012084F87F00B5E7304695F818906DF0CE
:108AE8002DF981457FF449AF237F052B10D184F8F8
:108AF8001C8042E755534243B8200020C46D0A0049
:108B080018890900236D0A00476D0A00626E0A0081
:108B1800022B7FF432AF4FF030092A8AD4F8803024
:108B280094F861801344C4F8803023681969D3F835
:108B380004B091F8613009FB031124310846039110
:108B48006DF0BAFA0399024658466DF022F90028EA
:108B58007FF413AFD4F87B3013B120686DF0F9F8C7
:108B680009FB08402430AFE7304695F818806DF0CF
:108B7800E5F8804502BFA37F03F1FF33A37707E73A
:108B8800EB7F0133EB77A4E62046FFF7E7FDA0E68D
:108B980020466DF0AEF99CE6022084F87F0004239D
:108BA8001AE094F9601040B90029206802DA6DF0E3
:108BB800D0F8BEE66DF0E3F8BBE6002914DA90427F
:108BC80002D8B9F1000F06D120686DF0C2F802236F
:108BD80084F87F30E3E702232377237F022B0ED12B
:108BE80020466DF086F913E6904202D8B8F1000FDE
:108BF80003D120686DF0C3F8E9E70323ECE7032B02
:108C080003D12046FFF7AAFD02E6042B7FF400AE4D
:108C1800A37F2BB101211D4A1D486BF0E8FDF7E544
:108C280020686DF08BF8804620466DF06FF8054699
:108C3800024604F1730304F17F0153F8040B8B42DD
:108C480042F8040BF9D11B782946137040460D22CF
:108C5800FFF7CEFC0646014620686CF0AEFD78B101
:108C68000C4A434601210A486BF0CAFD3046FDF71D
:108C78008BFC294620466DF02CF96DF0F6F8C7E517
:108C8800A37F0133A37705232377C1E5886E0A0004
:108C980018890900C46D0A00802938B50D461446A4
:108CA80021D083290DD019BB80235371832303203E
:108CB800117193710023E07023706570A370043004
:108CC80038BD0223137101235371002393710A23C2
:108CD800D37108224168A0188EF0A1FF064B0E2020
:108CE8001B882382E6E7044B02201B889380E1E778
:108CF8006FF08500E4E700BF7AB40A002DE9F0417F
:108D08008769D0F82480BA4228BF3A46B2FBF8F403
:108D18000646C269234600686BF04BFF0546C0B99A
:108D2800B7FBF8F7A7420BD1002205213068FCF702
:108D380061F828B101210A4A0A486BF058FD01255B
:108D4800F3692344F3613DB10020074BB362BDE8EA
:108D5800F08100240125E7E7706A6043F7E700BF68
:108D6800A96E0A00188909000203000C81420B460B
:108D780007B509D302210D4A0D486BF041FD6FF08C
:108D8800150003B05DF804FB6AB101391144814252
:108D980001D28B4207D90221009305481346054AA0
:108DA8006BF038FDEBE70020EBE700BFC06E0A0070
:108DB80018890900D76E0A000C290346084616D1FF
:108DC8001B78252B12D009D8122B10D8084A42FA42
:108DD80003F313F0010F08BF0620704703F0FD02EC
:108DE800282A03D05A2B08BF0A2070470A20704748
:108DF800F6FFFBFF2DE9F041984690F82C3086B03D
:108E080023F00C0380F82C300023C0E9043383617D
:108E1800062A04460F460B7840F010810BBB4B79AD
:108E28005B0724D490F82C309F070DD402234FF40D
:108E380068521946002584F8283084F8291062857C
:108E4800284606B0BDE8F0816DF092F80028EDD113
:108E5800002319461A46EDE70223052145F202329E
:108E6800E8E7032B36D14E7916F0040604D0022326
:108E780005214FF41052DDE790F82C308DF807608B
:108E880043F0040380F82C307023ADF8043090F8D8
:108E980029300D7903F00F038DF806300A23122DBF
:108EA80028BF12258DF80B30438D2A465BBA404601
:108EB80001A98DF808608DF809608DF80A6003969D
:108EC800ADF81030ADF81260ADF814608EF04AFEBF
:108ED800A662B5E71B2B00F0898009D8122B1AD09F
:108EE8001A2B61D00121B24AB2486BF089FCBEE767
:108EF8001E2BF7D14B795E07B9D40B7913F0030316
:108F080000F09780012BA3D190F82C3043F0010397
:108F180080F82C309CE74B795E07A8D490F82C3069
:108F280043F0040380F82C304A7812F002061FD16F
:108F3800D5078B7822D5B1F8035042461946FFF77A
:108F4800ABFE6DBAADB285420BDAB7F803506DBA15
:108F5800ADB200231A4684F8283084F82960628567
:108F68006EE742462046B978FFF796FE051EF0DA0E
:108F7800022305264FF410520025ECE72BB10221FD
:108F88008D4A8C486BF03CFCF2E7B1F8035041463F
:108F98006DBAADB26DF022F8232DD6D941462046E0
:108FA8006DF01CF82425D4E74D7915F004057FF4FD
:108FB8005EAF90F82C3043F0040380F82C308B78A7
:108FC8003F2B0ED1CE78002ED2D10D790323042D5C
:108FD80028BF042540462A4601A901938EF0C2FD08
:108FE800B7E7022305264FF41052B4E74B79590727
:108FF8003FF53DAF3B791A090CD19A070AD5DB0733
:1090080015D494F82C3003F00303032B3FF424AF5A
:10901800002305E094F82C209707C2F34003F0D50D
:1090280094F82C2063F3410284F82C2010E70123E4
:10903800F6E790F82C2063F30002F5E70A2A7FF49C
:1090480051AF2A2B1AD8222B7FF64CAFA3F123025B
:10905800072A3FF647AF01A151F822F0DB90000044
:10906800ED8E00005D910000ED8E0000ED8E000099
:10907800C5910000ED8E00001D9200005A2B7FF470
:1090880031AF4D7A15F004057FF4F1AE90F82C302D
:1090980043F0040380F82C308B783F2B40F0DD80C0
:1090A800CE78002E40F0D9804FF4C063CDE9013668
:1090B800B1F8075040466DBAADB2082D28BF082553
:1090C80001A92A468EF04EFD3246334684F8282000
:1090D80053E07B7A13F004037FF4C9AE01AEADF818
:1090E8000430B370082390F82C208DF8073042F034
:1090F800040280F82C206CF03BFF0028B5BF4FF02D
:10910800FF3302220322236A8DF80C20A8BF1BBA62
:109118000293636A31461BBA8DF80D30C3F30722F8
:10912800C3F307438DF80F3094F82C308DF80E20D8
:1091380043F0040384F82C30B7F8075040466DBA62
:10914800ADB20C2D28BF0C252A468EF00BFD00234E
:10915800A36275E67E7A16F004067FF488AE90F86E
:109168002C3043F004039D0780F82C3009D40226E4
:109178004FF46853002584F8286084F829606385D3
:109188005EE66CF0F5FE0028F1D1236A03B1013BDD
:1091980094F82C10626A1BBA12BA41F0040184F8E0
:1091A8002C100825C8F80030C8F804200023E2E78E
:1091B8001E6F0A0018890900016F0A007B7A580798
:1091C8003FF555AE94F82C30D7F8026043F004030D
:1091D8009907B7F8075084F82C307FF527AE20465A
:1091E8006CF0C6FE00287FF421AE6DBA36BAADB277
:1091F8002A463146206AFFF7B9FD20B1022305212E
:109208004FF4045216E6174B2361636AE6616B4319
:10921800A3611DE67B7A5A073FF529AE90F82C30FA
:10922800D7F8026043F00803B7F8075080F82C30ED
:109238009B077FF5FBAD6CF09BFE00287FF4F6AD35
:109248006DBA36BAADB22A463146206AFFF78EFDAE
:109258000028D3D1044B6361D7E7022205264FF4D7
:10926800105333E747600700058D000010B5046907
:109278000346204640F8143B0122002172F02FFEDD
:1092880004F12C00024972F0D6FE002010BD00BF88
:109298002594000038B503461B6940685C681B6963
:1092A80025685A681AB19A680AB1DA683AB913484F
:1092B8000121134A6BF09BFA6FF0150038BD10338B
:1092C800D3E8EF1F41F00101C3E8E21F002AF7D1FC
:1092D800216909B90020F1E72B7A002BFAD16BF04C
:1092E800C6FF28B10121074A04486BF080FAF1E76C
:1092F80020696CF049F82872ECE700BF0089090082
:10930800396F0A007A6D0A0038B504694068006848
:1093180004F11005D5E8AF5FED071FD40BB15D6808
:109328003DB9104A104801216BF061FA6FF0150041
:1093380038BD90F820501DB1DD680DB90B4AF1E732
:1093480085791DB19D690DB9094AEBE7C4E9021297
:1093580063600274120A42740020E9E76FF0770034
:10936800E6E700BF636F0A0000890900826F0A0000
:10937800A16F0A002DE9F347D0F804A006698846D2
:1093880015467768DAF8044006F11003D3E8AF3FD2
:109398009B073BD5236960685B68D3F800906BF046
:1093A800C0FE00220023012829460CBF99F81B9013
:1093B80099F81490DAF80C00CDE9002342466BF0D6
:1093C800A9FD054650B90121124A13486BF00FFA5E
:1093D8006FF00B04204602B0BDE8F087014680F824
:1093E800189020466CF0E9F9044618B12846FDF7B4
:1093F800CBF8EFE7FB69002BECD14FF0FF324FF0D1
:10940800FF3306F114002AF0EBFAE3E76FF00C04DF
:10941800E0E700BFC26F0A000089090070B550F884
:109428002C3C5C6865681C38D0E8AF3F9B0725D5A5
:109438002B6968685B681E686BF073FE0022012860
:109448004FF00003A0680CBF96F8296096F82260D8
:109458006BF05CFD044630B9094A0121BDE8704053
:1094680008486BF0C4B90146067628466CF0A5F9A1
:1094780020B12046FDF788F8034AEEE770BD00BF2B
:10948800DD6F0A0000890900F76F0A0070B50B78D4
:1094980092B006460C4607AD032B31D8DFE803F03F
:1094A800022A2C2E19492846F7F79AFE0595637863
:1094B800174A0493A3781E210393E3780AA802931A
:1094C800237910AD019363790093A37965F014FDB6
:1094D80032460AAB1C4603CCAC42106051602346AE
:1094E80002F10802F6D1206810603046A388938004
:1094F80012B070BD0749D6E70749D4E70749D2E754
:109508000A212846064A65F0F7FCCFE72C700A00C6
:109518004E700A0033700A003A700A0044700A005C
:10952800E2910A000E4B402928BF402170B51D4624
:109538000C4C4618B04203F1020304D1002305F88D
:109548001130074870BD02781209A25C03F8022C9A
:1095580010F8012B02F00F02A25C03F8012CE9E7D6
:10956800ABD30020C1B50A0010B50024094B86B062
:1095780009480393CDE9044472F0B3FD03AB0093AB
:109588004FF440620A23054903482AF021FC20468B
:1095980006B010BD78700A00202F002058E7002080
:1095A800014601482AF054BC202F002001460148FA
:1095B8002AF07EBC202F00200146014872F066BDCB
:1095C800202F00202DE9F74306468946174698467E
:1095D8003C4DD5E8AF3FDA0722D548B901213A4AD0
:1095E8003A486BF004F96FF0010003B0BDE8F0836E
:1095F80001A96BF020FB022804462BD1024634490E
:1096080030468EF0DDFA0028EDD1D5E8AF3FC3F340
:10961800C0061B0706D52F4A21462C486BF0E7F8F1
:109628000020E2E7A5F18804072221464046B84712
:1096380006280AD80121284A24486BF0D8F845F8AA
:10964800886CE671C4F80360EAE70723B0FBF3F01F
:10965800E071E5E7042818D10246204930468EF02B
:10966800AFFA04460028BED11C22404605F1A001ED
:10967800B847031E05DA0121194A14486BF0C0F8EF
:10968800CEE72B4483F8A040CAE70A28ABD10246AC
:10969800144930468EF094FA0028A4D1B9F1020F8B
:1096A80007D00A480121104A6BF0A1F86FF01500A5
:1096B8009BE74A46404605F1BE01B84700EAE0701C
:1096C80093E700BF0802002081700A00C8870900DC
:1096D80041700A00A2700A00C6700A00B1760A003A
:1096E800EB700A001D710A0028710A002DE9F04389
:1096F80089B0DDF840909D795E791F7993F803C0B1
:1097080093F802E093F801800C461B78B9F1000F3A
:1097180015D0CDE90639CDE904E81346CDE9027C38
:10972800CDE900560D4A65F0E7FB002813DBA0429F
:109738002CBF6FF01500002009B0BDE8F083CDE91B
:109748000583CDE903CE1346CDE90167044A0095A8
:1097580065F0D2FBE9E76FF01500EDE75F710A00ED
:1097680083710A0010B5FBF74BFD044628B10121AF
:109778000346034A03486BF043F8204610BD00BF78
:10978800A4710A00C887090070B504461E4615462C
:109798008CB0AAB129B10A4602A804216AF011FACC
:1097A80002A900912B462246242103A8FFF79EFF19
:1097B80070B93146109A03A8FBF79EFB0CB070BD38
:1097C80003462421044A03A865F096FB2328F0D910
:1097D8006FF01500F2E700BFC9710A0007B50B4B1F
:1097E8000B48DA79C2EBC202009200221146FFF759
:1097F800CBFF034638B10121064A074803B05DF89C
:1098080004EB6AF0FDBF03B05DF804FB80010020A3
:1098180041700A00CF710A00C887090030B50446B4
:1098280015468DB09AB129B10A4602A804216AF0FA
:10983800C8F902A900912B462246242103A8FFF764
:1098480055FF60B903A86BF0CEF90DB030BD0346E3
:109858002421044A03A865F04FFB2328F2D96FF0AE
:109868001500F2E7C9710A0007B5009313460A46C6
:1098780001460348FFF788FF03B05DF804FB00BF0B
:10988800218F0A000A4601460148FFF7C7BF00BFFB
:10989800218F0A0007B5009313460A46014603487C
:1098A800FFF772FF03B05DF804FB00BF1B8F0A00CF
:1098B8000A4601460148FFF7B1BF00BF1B8F0A00E7
:1098C80007B5009313460A4601460348FFF75CFFB5
:1098D80003B05DF804FB00BF4C8D0A000A46014640
:1098E8000148FFF79BBF00BF4C8D0A0007B5002257
:1098F8000346009103481146FFF746FF03B05DF8A1
:1099080004FB00BF138F0A0007B50022034600912D
:1099180003481146FFF738FF03B05DF804FB00BFAA
:10992800B1760A0007B500220346009103481146A4
:10993800FFF72AFF03B05DF804FB00BF1D710A00A2
:1099480008B502482AF03EFA002008BD5C0800204D
:10995800F8B51E4DD5E8AF3F13F0010F2F4632D0B2
:1099680095F8A040A5F188063CB91C22184906F5CF
:1099780094708EF054F986F84441F3798BB902F06B
:109988004BF8044630B10121124A13486AF02FFF00
:109998002046F8BDF37923B902F04EF804460028B2
:1099A800F1D1D5E8AF3F5A0701D400F0CBFED7E894
:1099B800EF3F23F40062C7E8E12F0029F7D11B0528
:1099C80001D5FFF7BDFF0024E2E700BF0802002031
:1099D800EA710A00F1710A00C887090007B5009307
:1099E80013460A4601460348FFF7CEFE03B05DF86A
:1099F80004FB00BF52940A000A4601460148FFF7DB
:109A08000DBF00BF52940A0030B50378012B11D066
:109A1800022B21D06BB90A46144B03F1100453F8FA
:109A2800045BA34242F8045BF9D143881A0A8A709E
:109A3800CB7030BD0A460D4B03F1100453F8045B9C
:109A4800A34242F8045BF9D143681A0C180E4A7015
:109A58000870C3F30722EAE700F11003013913F88D
:109A68000129984201F8012FF9D1E2E7D2B50A009D
:109A780010B56CF0ABFD72F093FB044608B92AF000
:109A8800F5FD064BD3E8AF3F0BB10A2098471CB948
:109A9800BDE810402AF0FEBD10BD00BFC064002024
:109AA80038B5044608486BF031FA054648B1631EDC
:109AB800DBB21F2B96BF054A0021D15C0C306BF03E
:109AC800C6FA284638BD00BF8C220020E2B50A003D
:109AD8000F2810B50CD80D280CD90A486BF016FAC7
:109AE800044618B104210C306BF0B1FA204610BDC1
:109AF8001328F2D009B10448F0E70220BDE810406D
:109B0800FFF7CEBF3C23002008220020C3681B7843
:109B18000221024A02486CF0F7BD00BF33720A0006
:109B280090870900F8B506460F4604F01DFB044669
:109B380090B9394630460BF003F80546F0B9394676
:109B4800304608F0D9FF164B1B6823B153F80C496F
:109B580004B10C3CB3B9F8BD83781321012B4FF045
:109B6800000312BF1D46D0F8A450C0F8A4306DF011
:109B7800F8F9204603F06EFE002DDAD028466FF083
:109B880083FADCE79B6813B13946304698472CB115
:109B9800E26802B10C3A23461446DBE72246FAE7AC
:109BA800C865002010B5002486B003AB00934FF4BD
:109BB80080624FF0FF3305490548CDE90344059419
:109BC8002AF006F9204606B010BD00BF58F3002061
:109BD8002030002038B5C4682378ABB9B4F80150F8
:109BE8000F21284603F09CFFE278044688B90D4B04
:109BF800194633F8024B44B96FEA05536FEA135319
:109C080021F81030084B1A5438BD01300528F0D11E
:109C1800FAE70273012103F069FE2046BDE83840E7
:109C280003F018BE18D100202CD4002070B5C368EA
:109C38001D787DBBB3F801600F21304603F070FF3B
:109C4800044638B901213346BDE87040124A13482A
:109C58006CF05ABD294603F049FEA378012B04D0C5
:109C68002046BDE8704003F0F5BD201D6CF035FDC1
:109C7800C307F5D50321204603F038FE032002F080
:109C880025FF03460028EBD00221054A03486CF063
:109C98003BFDE5E770BD00BF5B720A0090870900D5
:109CA80081720A0010B5C3680121B3F8014020464B
:109CB80003F036FF38B901212346BDE81040044AB5
:109CC80004486CF021BDBDE8104003F0C3BD00BFDF
:109CD800A7720A009087090010B5C36801211C8883
:109CE800204603F01DFF38B901212346BDE8104086
:109CF800034A04486CF008BDBDE8104003F0AABD53
:109D0800A7720A009087090010B501210C306BF08A
:109D1800DCF903780121BDE81040024A02486CF0E2
:109D2800F3BC00BFCB720A0090870900014610B54A
:109D380008486BF002F90849084872F0A7F9031EB1
:109D480006DABDE810400121054A06486CF0DCBC83
:109D580010BD00BF840200207C08002020310020B4
:109D6800ED720A00908709000121024A02486CF04E
:109D7800B7BC00BF0A730A009087090070B5C568B0
:109D88000121B5F80160304603F0CAFE044638B92F
:109D980001213346BDE870400B4A0C486CF0B4BC56
:109DA8002B783BB9D5F80330C0F89930D5F807308F
:109DB800C0F89D30201D4FF400316CF09AFC20460D
:109DC800BDE8704003F046BDA7720A0090870900FD
:109DD80008B502F031FE064B18466CF07EFC00F028
:109DE8000B00D3E8EF2FC3E8E10F0029F9D108BD34
:109DF800080200200B46B0B50D8A00AF044629467C
:109E0800D868FFF78FFB8AB06A460A4BCDE907503E
:109E1800CDE9053440F20243ADF82430064B42F850
:109E2800103F00234FF432510448FAF7BDFCBD46F9
:109E3800B0BD00BF24730A00050000019087090027
:109E48002DE9F84FD0F80C90018A99F8004000AF3E
:109E5800A30001338B4260D96D468AB06A46CDE9CA
:109E6800073105232E48CDE9050442F8103F0023A9
:109E78004FF421512B48FAF797FCAD46BD46BDE893
:109E8800F88F01212B46284A26486CF03DFC013604
:109E980099F800309E42F1DA09EB8603B3F80150D5
:109EA8000F212846B3F8038003F03AFE0446002841
:109EB800E7D000F1C00AB8F1000F06D0656945B9CE
:109EC80001211A4A17486CF00BFC204603F0C2FC2B
:109ED800DDE7A2692B6895422046636108BFA3614C
:109EE80003F0D8FB29F040FDC5F800B0236A8BB910
:109EF800C4E90755DAE8EF3F013BCAE8E23F002A28
:109F0800F8D10021204608F1FF3803F0CDFB1FFAF5
:109F180088F8D0E71D602562ECE70026B346B7E76E
:109F280046730A009087090071730A008D730A004E
:109F380080B500AF8AB06A46094BCDE90530094BB8
:109F4800079340F20133ADF82030074B42F8103F39
:109F580000234FF412510548FAF726FCBD4680BD90
:109F6800A4730A00E8A30A0004000001908709000E
:109F780037B50446084602EBC3039A4202D16FF094
:109F88005E0010E0114611F8085BA54211D1038A62
:109F98005178994209D908480121084A00946AF081
:109FA80039FC6FF0150003B030BD536898470020A6
:109FB800F9E70A46E1E700BF90870900C0730A0085
:109FC8002DE9F0470C462AF051FBE5682B78022B67
:109FD80072D0042B07D001213B4A3C486CF094FB1B
:109FE8006FF015040EE0B4F81080B8F1020F0ED827
:109FF8004346374A354801216CF086FB2046FCF77A
:10A00800C3FA00242AF046FB2046BDE8F0876878AA
:10A018003E280CD1B8F1030F02D12E4A4346E9E796
:10A02800EB78012B01D00A2B46D1032704E06CF012
:10A0380041FB0746F8073FD504F10C0601213046DD
:10A04800D4F814A06BF039F8022130466BF03DF8D3
:10A05800814600783E2807D1E3681B78012B01D0A0
:10A068000A2B06D1032614E06CF024FBC107064630
:10A078000FD441F28A13184A1849194869F028FB85
:10A08800002383F31188BFF36F8F0323184602DF81
:10A098000226144A0623214699F800006CF055FB65
:10A0A800B2070DD56369A5EB0A0513FA85F5E560D6
:10A0B800A4F81080BB07A4D52046FFF737FEA0E719
:10A0C8002046FCF761FAF5E788740A0090870900D2
:10A0D800E2730A00FE730A001E740A0052740A0032
:10A0E8006B740A000C90090010B5012104460C306D
:10A0F8006AF0EBFF2146BDE810400223014A0078D0
:10A108006CF023BB3C90090073B53E486AF02AFF07
:10A118000446002873D000F10C0528466AF0DDFFDC
:10A128000228034603D0042847D0374A03E0238A8D
:10A13800032B05D8354A012135486CF0E5FA13E0C0
:10A14800042128466AF0C1FFFF2342880688237647
:10A15800238AC6F30B009A42608309D0012100923A
:10A168002B482C4A6AF056FB2046FCF70DFA12E001
:10A178000F2103F0D5FC054610B9638B264ADAE7B0
:10A1880003F002FD21462076320B284603F0DEFA62
:10A19800284603F05FFB214BD3F804317BB32049F9
:10A1A800204871F073FF031E29DA01211E4A18485E
:10A1B80002B0BDE870406CF0A7BA284602216AF0E8
:10A1C80084FF054600783E2812D06CF073FA10F030
:10A1D80002060DD140F6BC43144A1549154869F0EA
:10A1E80077FA86F31188BFF36F8F0323184602DFCF
:10A1F80006232146104A28786CF0A7FAB4E702B083
:10A2080070BD00BF8402002031750A009C740A00EA
:10A2180090870900BD740A00E1740A0080010020DB
:10A228007C08002020310020ED720A001E740A000C
:10A2380003750A006B740A004C90090010B50121DF
:10A2480004460C306AF041FF2146BDE810400D235A
:10A25800014A00786CF079BA7C900900F8B50121C0
:10A26800044600AF0C306AF030FF06780023214620
:10A278003046114AFFF77CFE5F301AD1258AE06824
:10A288002946FFF74FF96C468AB06A460B4BCDE971
:10A298000750CDE9053640F20243ADF82430084BAB
:10A2A80042F8103F00234FF432510648FAF77CFA7F
:10A2B800A546BD46F8BD00BFE490090045750A00F3
:10A2C80005000001908709002DE9F74F002380461B
:10A2D80089461746DFF810A1DAE8EF4FCAE8E23FEF
:10A2E800002AF9D1264644B9012143463A4A3B4857
:10A2F80003B0BDE8F04F6CF007BA2046FCF7A4F8AD
:10A308004FF00C0B364D0BFB0050438843451BD0D8
:10A318002046FCF799F80BFB005043880121009375
:10A32800304A43462D486AF075FADAE8EF3FCAE842
:10A33800E26F002AF9D1002B4BD01E46304603B0FD
:10A34800BDE8F04FFCF720B9A74208D020466AF0D4
:10A35800D8FD3A8AF96804F10C006AF06FFE2046CD
:10A36800FCF772F80C2707FB00504368ABB1B9F152
:10A37800000F12D12046FCF767F8012107FB0050B7
:10A388004268536803F01F00814010685B0900EBC6
:10A398008300137ACBB16CF0ACF92046FCF754F883
:10A3A8000C2707FB00508368002BC7D02046FCF71A
:10A3B8004BF8784305F800902046FCF745F807FB72
:10A3C8000055A86829F0D0FAB8E7C9436CF0A3F99A
:10A3D800E3E703B0BDE8F08F77750A0090870900BE
:10A3E800C46400209F750A008002002073B5C56808
:10A3F8000121B5F80160304603F092FB044640B9EC
:10A40800012133463D4A3E4802B0BDE870406CF039
:10A418007BB92B78061D1A2B19D1C378012B50D183
:10A428004FF4804130466CF064F942040FD4D4F8FC
:10A438008C3069460093D4F894302046019304F098
:10A44800EBFB204602B0BDE8704003F003BA2B785E
:10A45800BBBB40F2E242B5F803302A495343C4F883
:10A468008830B5F80520A4F89020B5F80720A4F89E
:10A478009220A3F5EA520C3A8A4204D90221224AD0
:10A488001F486CF041F9B4F89030B3F5FA7F04D363
:10A4980002211E4A1A486CF037F940F67641B4F8A2
:10A4A8009230A3F10A0292B28A4204D90221184AD0
:10A4B80013486CF029F96FF4805130466CF02BF991
:10A4C80014E030466CF009F9C304F4D52B78202B3E
:10A4D800F1D194F89830002BEDD0013B84F89830F6
:10A4E8000C4A002304F1400029F0DCFC2B78002BF7
:10A4F800A7D1204603F01EFDA3E700BFA7720A00FC
:10A508009087090095F03C00D2750A00F9750A0099
:10A5180020760A005A62020010B5C1E900239DF8AE
:10A5280008300C460B72FBF78FFF0C22024B02FB24
:10A5380000335C6010BD00BFC4640020F8B502465B
:10A548000B4610486AF0E2FC0446C0B104210C3006
:10A558006AF063FD2046FBF777FF0C2700260A4DBB
:10A5680007FB005046802046FBF76EFF07FB0050B4
:10A5780086602046FBF768FF07FB00556E602046A3
:10A58800F8BD00BF60220020C46400200138C0B2BA
:10A5980002289ABF014B185C002070472CB60A00AD
:10A5A80037B50C468DF8070000F0FF05A0B929B1B2
:10A5B800072220460A498DF003FB40B900200949CB
:10A5C8000DF107020AF004FA002003B030BD21465D
:10A5D8002846FFF7A7FAF7E76FF01500F5E700BF81
:10A5E800AEB50A001567070029289ABF014B185C09
:10A5F8000920704702B60A0070B5C3680F21B3F886
:10A6080001601D78304603F08BFA044638B9012101
:10A618003346BDE87040184A18486CF075B865B103
:10A628002846FFF7E1FF29460246204603F03AFD97
:10A638002046BDE8704003F00DB98378012B07D19F
:10A648000AF076F820466CF01DF8002808BF0525AA
:10A658002846FFF7C9FF29460246204603F022FD97
:10A66800002DE5D00121064A04486CF039F805218F
:10A6780020466CF076FCDBE75B720A0090870900E5
:10A688004C760A002DE9F041C6680F21B6F8017032
:10A698003578384603F044FA044638B901213B4678
:10A6A800BDE8F0411E4A1F486CF02EB865B1284637
:10A6B800FFF79AFF29460246204603F0F3FC20469E
:10A6C800BDE8F04103F0C6B8F278C37A934205D1E9
:10A6D8000221154A13486CF017F8F0E78378C27224
:10A6E800012B08D10AB10AF023F820466BF0CAFF03
:10A6F800002808BF05252846FFF776FF29460246A9
:10A70800204603F0CFFC002DD9D00121074A054887
:10A718006BF0E6FF052120466CF023FCCFE700BF75
:10A728005B720A009087090072760A004C760A006C
:10A73800034B0146D3F8240182689268104700BF92
:10A748008001002008B5042103486BF0D2FFBDE862
:10A75800084002F071B900BF0802002008B503489C
:10A768006BF0BBFFC0F3800008BD00BF08020020EB
:10A7780038B50546F6F73CFD1C2804461BD8294683
:10A788000E48F6F723FDA0B1224629460B488DF066
:10A79800E9F900220A482146031900F5947083F864
:10A7A8002821FFF7B1F820B10221064A06486BF0CC
:10A7B80097FF002038BD6FF00B00FBE7A8020020D0
:10A7C80080010020A1760A009087090000487047A0
:10A7D800A8020020014BB3F8460170478001002011
:10A7E80037B50F4DADF80600B5F84631834203D1B1
:10A7F8000024204603B030BD02210DF10600FFF70A
:10A8080091F8044630B101210346064A06486BF028
:10A818007BFFEEE7BDF80630A5F84631E8E700BF54
:10A8280080010020B6760A00908709000149024895
:10A8380071F02CBC6C0800202030002070B5054653
:10A848000C4639B1CB684A699B1A032B0ED86FF0B6
:10A85800150509E04FF0FF304FF0FF31FFF76EFEAE
:10A86800044618B96FF06805284670BD2046FBF706
:10A87800EBFD0C22164BA61802FB003303213046D1
:10A888005D806AF009FC0580238A0121033B8370FF
:10A8980030466AF009FC40F635439D420FD1204608
:10A8A800FFF746FF05460028DED001210346094A86
:10A8B80009486BF029FF2046FBF766FED4E72146DE
:10A8C800064871F0D5FA0025FFF7B0FFCCE700BFC6
:10A8D800C4640020E7760A00908709008C020020F3
:10A8E8002DE9F04786B0804691460C4600AF71B915
:10A8F8004FF0FF304FF0FF31FFF720FE044660B9FC
:10A908006FF0680528461837BD46BDE8F087887A95
:10A91800FBF792FD3C4B83426FD101220021384660
:10A9280071F0DDFA2046FBF78FFD0C23DFF800A15C
:10A9380003FB00A0876020466AF02AFB01464046D8
:10A94800FFF77CFF054618B12046FBF71DFED9E747
:10A95800002338462D4A29F043F8064690B140F2C4
:10A96800E3132B4A2B492C4868F0B2FE3246414685
:10A978002A4868F0ADFE85F31188BFF36F8F032373
:10A98800184602DF2046FBF75FFD0C2358431AF8F0
:10A99800006066B36D468AB06A46214B0796CDE9DA
:10A9A8000538204B089340F20243ADF824301E4B83
:10A9B80042F8103F00234FF432511C48F9F7F4FED7
:10A9C8002046AD46093EFBF7DFFD092E0CD8DFE82F
:10A9D80006F0050B0B08170B0B0B0B146FF06E052D
:10A9E80090E76FF00C058DE76FF004058AE7B9F181
:10A9F800000FA9D0C9F8004084E76FF0150581E77A
:10AA08006FF00B057EE700BF60220020B4C404008D
:10AA18001E740A0009770A006B740A0012770A008C
:10AA280057770A00E8A30A0005000001908709008B
:10AA3800C464002073B506460D4642F22F0000217B
:10AA480001AAFFF74DFF044638B10121144A154801
:10AA58006BF046FE204602B070BD0198C368B3F89B
:10AA680001203280B3F803302B80FBF78DFD33884B
:10AA7800A3F11B02E02A04D902210B4A09486BF012
:10AA880043FE44F248112B88A3F5A47292B28A427D
:10AA9800E0D90221054A03486BF036FEDAE700BF29
:10AAA80076770A009087090096770A00BB770A0034
:10AAB8002DE9F04385B004460DF10301002001F0B3
:10AAC80029F8054600287CD14FF0FF304FF0FF31C0
:10AAD800FFF734FD0746002877D000F10C080A215B
:10AAE80040466AF0A5FA0646056045600581384D7E
:10AAF800023095F8DA3095F8DB209A4294BF04F1D9
:10AB0800700104F17E016BF0EDFD9DF80330737068
:10AB1800AB6813F002091DD101231021404673725E
:10AB28006AF086FAAA890280EA894280B4F88C2001
:10AB38008280B4F88E20C280B4F890200281B4F8E4
:10AB4800922080F80C90428180F80D9080F80E9049
:10AB580080F80F90AB68DB071CD5737A102143F09F
:10AB68000403404673726AF063FA2A8A02806A8A8A
:10AB78004280B4F88C208280B4F88E20C280B4F869
:10AB880090200281B4F8922042810022027342731D
:10AB98008273C2730F4B3846019307230293012334
:10ABA8008DF80C30FBF750FC0C220B4B394602FB9E
:10ABB800003301AA5A6042F243000022FFF790FED8
:10ABC8000546284605B0BDE8F0836FF06805F8E74C
:10ABD8008001002008020020C46400203C2870B5D1
:10ABE800054644D002283ED100210246084603F01B
:10ABF80047FB044680B901211D4A1E486BF070FDD1
:10AC0800032001F063FF034688B3BDE870400221CA
:10AC1800194A18486BF078BD04306BF05EFDC30725
:10AC280007D50321204602F061FE204602F012FEFD
:10AC3800E6E704F1400071F067FA10F00C0607D15E
:10AC48000E4A29460B486BF04BFD31462573E9E760
:10AC58002046FFF72DFF0028E7D00121084A0548C4
:10AC68006BF03EFDE1E7BDE87040FFF761B970BDEC
:10AC7800DE770A009087090081720A00FC770A00D3
:10AC880022780A0030B54FF0FF304FF0FF3185B021
:10AC9800FFF754FC0446B0B10C4B00250193072381
:10ACA8008DF80C500293FBF7CFFB0C22084B214682
:10ACB80002FB003301AA5A6042F20E002A46FFF74F
:10ACC8000FFE05B030BD6FF06800FAE708020020FB
:10ACD800C46400202DE9F0478CB0764AB0F80180B2
:10ACE80005460023104600AF48F4704132F8024B85
:10ACF800A14258D1002220F813206F4A12F803907D
:10AD080000F07CFDEB782E1D012B08BF6B4B304605
:10AD180014BF002493F822406BF054FC31460028FD
:10AD280047D007F108006BF042FCD5F81130C7F89E
:10AD38000130B5F81530A7F8053001233B70E878E5
:10AD4800002843D1022207F1080103F099FA0446CA
:10AD5800EB7823B96FF0800159486BF0DCFC002CCC
:10AD680049D107F1100531462846FEF78FFB6E469C
:10AD780088B06A46534BCDE905354FF40073ADF8FA
:10AD88001C30514B42F8103F4FF4E2514F482346D4
:10AD9800F9F70AFD1321B54640466BF011FD30372F
:10ADA800BD46BDE8F0870133052B9FD14FF0000960
:10ADB800A6E720466BF0A0FE014607F108006BF0FD
:10ADC80091FC314638466BF08DFCB8E7012810D16C
:10ADD800DFF8E8A006229AF8220007F1080103F03C
:10ADE8004FFA04460028B3D1052239499AF82200BF
:10ADF800ABE70024ACE7204640F2E242B5F8013068
:10AE080007F1080120F8703B6BF06CFCB5F81730BF
:10AE18005343C4F88830B5F81930A4F89030B5F821
:10AE28001B30A4F892300023EA782373012AE270D9
:10AE38002ED1394604F177006BF054FCD5F80B306D
:10AE4800C4F87F30B5F80F3084F87E20A4F883303A
:10AE58000721204602F04AFDB9F1000F05D0012173
:10AE6800204684F80C9002F041FD204602F0C8FE0E
:10AE7800E3784BB9032001F029FE034620B10221F3
:10AE8800144A12486BF040FC204602F0E3FC86E7C7
:10AE9800002ADDD1394604F17E006BF023FC217ACB
:10AEA800064BC1EBC101194404F177006BF01AFCA1
:10AEB800CEE700BF18D100202CD40020800100204C
:10AEC800080200203E780A0003000001908709006C
:10AED800A7B50A0081720A0000B5C16889B0087870
:10AEE80020B109B05DF804EBFFF778BEB1F8013086
:10AEF8008DF80000ADF80130CB7801A88DF803304B
:10AF0800B1F80B300431ADF81730B1F80930ADF8AD
:10AF18001930B1F80B30ADF81B304B7B8DF81D3074
:10AF28006BF0E0FB084B68461A689B88CDF80B204D
:10AF3800ADF80F30CDF81120ADF81530FFF7CAFE87
:10AF480009B05DF804FB00BFBBB50A0010B5F6F701
:10AF5800B7FA034B1B6813B1BDE81040184710BD82
:10AF6800E86400202DE9F341344D0646D5F8240164
:10AF780070F06AFD50B90121314A32486BF0B0FBDC
:10AF88006FF01204204602B0BDE8F0816FF00201B4
:10AF980005F188006BF0BFFB01216BF0AAFBC3072A
:10AFA80048D4FEF7DFFB04460028EBD1264B1E6091
:10AFB800012205F1E800114670F091FF234F05F5D5
:10AFC800867070F017FF384671F08BF838466FF0CE
:10AFD80007034FF400621E49009428F0F9FED7F8E1
:10AFE800E0001C4971F0E2F8D5F824010769D7F8A8
:10AFF8000080B8F1000F15D1174B3B6083681B68C0
:10B008009847044628B986B902B0BDE8F041F6F77A
:10B0180057BAC7F8008001212346104A09486BF047
:10B0280073FBAFE76FF07704F5E705F1780028F0D8
:10B03800C9FEA7E76FF07704A4E700BF80010020EE
:10B04800BA790A0090870900E864002020310020BE
:10B0580058F70020D2790A00C99F0000DB790A005E
:10B06800F0B5C56801212F8887B0BCB2204602F030
:10B0780057FD064640B901212346274A274807B00D
:10B08800BDE8F0406BF040BB02ACD5F80220D5F823
:10B0980006300194698900916DF040FE48B34FF085
:10B0A800FF304FF0FF31FFF749FA054648B9012153
:10B0B8001B4A1A486BF014FB304602F0CBFB07B072
:10B0C800F0BD12210C3069F0B3FF0346224623F885
:10B0D800027B144603CC596006A98C4218602246AC
:10B0E80003F10803F5D1294642F21A00FFF7A6FB3F
:10B0F800E2E74FF0FF304FF0FF31FFF71FFA044649
:10B108000028D4D002210C3069F092FF2146078034
:10B1180042F21B00EAE700BFA7720A009087090005
:10B12800F7790A0073B5C368D9789A781E8842EA15
:10B138000122ADF8002059791A79B4B242EA012205
:10B14800ADF80220D9799A79204642EA0122ADF871
:10B1580004201A7A5B7A012142EA0323ADF806300B
:10B1680002F0DEFC054658B901211D4823461D4A58
:10B178006BF0CAFA022120466BF0A9FB02B070BD41
:10B18800694602F023FF38B91E2120466BF09FFB69
:10B19800284602F05FFBF1E74FF0FF304FF0FF3138
:10B1A800FFF7CCF904460028F2D00E210C3069F0E4
:10B1B8003FFF00230680C0F80A30BDF80030214662
:10B1C8004380BDF802308380BDF80430C380BDF8E9
:10B1D8000630038142F22000FFF730FBD8E700BFBA
:10B1E80090870900A7720A0038B5042104460C307C
:10B1F80069F06BFF034640885D7818B122461978DC
:10B20800FFF762F835B1044828F0AEFBBDE83840D6
:10B21800FFF70CBB38BD00BF68020020B0B504467C
:10B22800032100AF0C3069F050FFE2680346117843
:10B2380040F63542B0F80100904217D16C468AB00A
:10B248006A46114BCDE90531104B079340F20133A3
:10B25800ADF820300E4B42F8103F00234FF4125146
:10B268000C48F9F7A1FAA546BD46B0BD1D7810B146
:10B278002246FFF729F8002DF6D0074828F074FB7E
:10B28800FFF7D4FAF0E700BF0E7A0A00E8A30A0035
:10B2980004000001908709006802002038B529F0F1
:10B2A800E5F9314DD5F80C31002B5AD00022002396
:10B2B80005F1E80028F094FB002852D10022002371
:10B2C80005F5867028F01AFB044668B940F6CC43A9
:10B2D800264A2749274868F0FBF984F31188BFF309
:10B2E8006F8F0323184602DFD5F800317BB1224A5D
:10B2F800012122486BF0F4F90022214BD3E8EF0F2B
:10B30800C3E8E12F0029F9D108B1FBF73DF9204640
:10B3180069F03EFEC5F800012046FFF709FA03462A
:10B32800C8B10121174A15486BF0EEF9164828F004
:10B338001BFB2046FBF788F80C22144B02FB00335A
:10B34800588818B122461F21FEF7BEFF2046FBF79A
:10B358001BF9FFF76BFAFFF769FABDE8384029F0E7
:10B3680099B902F05DFCF8E7800100201E740A001C
:10B3780027720A006B740A00467A0A00908709004F
:10B3880080020020E7760A0068020020C4640020DA
:10B3980070B54FF0FF320D464FF0FF3300210646DF
:10B3A800FEF796FB044660B91A230A4A0A490B4875
:10B3B80068F08EF984F31188BFF36F8F0323184662
:10B3C80002DF022104F10C0069F032FE06704570BC
:10B3D800204670BDAE7A0A0027720A006B740A0014
:10B3E800F8B506460024094DEF79E3B29F4202D82A
:10B3F8006FF0010007E0294630466BF0B2FA0735D6
:10B40800631C08B12046F8BD1C46EEE78001002009
:10B4180037B504460D46B9B1284616496BF0A1FA6E
:10B4280090B929461448C4EBC40420446BF092FA3E
:10B4380012486BF08CFA430703D5FEF781FA6BF0DC
:10B4480059F8002003B030BD68466BF0A2F8002818
:10B45800F8D16846FFF7C4FF0028F5DA064BC4EBBD
:10B46800C400694618446BF075FA002DE0D0014617
:10B478002846DBE7AEB50A0080010020080200205C
:10B4880070B5174E0622314605468CF099FB10B36D
:10B498004FF0FF304FF0FF31FFF750F80446E0B1AE
:10B4A800062229460C3069F0C9FD2146002242F2E5
:10B4B8000500FFF715FA044648B110F10D0F04D145
:10B4C8000221084A08486BF054FA204670BD2868E3
:10B4D8003060AB88B3800024F7E76FF06804F4E7C6
:10B4E8009C010020E47A0A00A0870900064BD3E8F3
:10B4F800EFCF4CF4806CC3E8E2CF002AF7D1037A8F
:10B5080019430172704700BF080200202DE9F3417A
:10B51800002104460222084602F0B2FE054648B160
:10B5280020460121FFF7E2FF284602B0BDE8F041BE
:10B5380002F090B98DF8000069464E4800F0ACFE64
:10B548009DF8003033B101212046FFF7CFFF02B04C
:10B55800BDE8F08148486BF0FAF98106C0F340175E
:10B5680008D545486BF0F3F9420603D5012120467A
:10B57800FFF7BCFF0021414800F08EFE17B1002004
:10B5880001F070FA3E4D95F8DB309BB100206BF06E
:10B598002FFA78B102213B4A3B486BF0EAF917B120
:10B5A800012001F05FFA0021384802B0BDE8F041FF
:10B5B80000F072BE95F8DB2095F8DA309A4218D17F
:10B5C8000221334A30486BF0D4F9002242F22900B4
:10B5D8001146FFF785F910B101212E4ADCE795F8ED
:10B5E800DB30013385F8DB30237A43F00403237220
:10B5F800D5E7224604F10108414612F82E0B6BF0FC
:10B60800BAF9064610B1244A01210EE095F8DB305C
:10B61800013385F8DB30237A43F00403237295F86D
:10B628005B305B0708D402211C4A17486BF0A1F96C
:10B6380001206BF0DDF9B2E7414668466BF08AF904
:10B6480001234FF0FF304FF0FF318DF80730FEF740
:10B6580075FF044660B1082269460C3069F0EEFCBB
:10B668003246214642F24E00FFF73AF90028DFD071
:10B678000B4AC9E7E16A070008020020B16A07001F
:10B6880080010020F37A0A00A08709002B6A0700CE
:10B69800187B0A00497B0A00697B0A00897B0A003B
:10B6A800B37B0A002DE9F74300210446022208462D
:10B6B80002F0E6FD054648B120460221FFF716FFD5
:10B6C800284603B0BDE8F04302F0C4B88DF807007F
:10B6D8000DF10701404800F0DFFD9DF8073033B158
:10B6E80002212046FFF702FF03B0BDE8F0833B4884
:10B6F8006BF02DF98206C0F3401808D537486BF077
:10B7080026F9430603D502212046FFF7EFFE002164
:10B71800334800F0C1FDB8F1000F02D0002001F05D
:10B72800A1F900206BF064F92E4D0646C0B1012145
:10B7380003462D4A2D4869F063F895F8DB3013B1BC
:10B7480001206BF055F9B8F1000F02D0012001F08B
:10B7580089F90021264803B0BDE8F04300F09CBDFC
:10B7680095F8DB3095F8DA209A420CD2013B85F83F
:10B77800DB30237A024623F0040302201D4923729A
:10B7880009F048F9D9E74FF0FF304FF0FF31FEF7E5
:10B79800D5FE04F10109074668B107210C3069F0AC
:10B7A80047FC49466BF0D6F83246394642F2280043
:10B7B800FFF796F828B101210F4A0C486BF0D9F829
:10B7C800BBE795F8DB30013B85F8DB30237A23F0C3
:10B7D80004032372B1E700BFE16A070008020020F2
:10B7E800B16A070080010020CE7B0A00A08709000B
:10B7F8002B6A0700E3690700FB7B0A00084BD3E8C4
:10B80800EF2F22F48061C3E8E01F0028F7D1530529
:10B8180004D500220220034909F0FCB8704700BF94
:10B8280008020020296C0700002307B50549CDE967
:10B8380000036A46022009F0EDF8019803B05DF8AC
:10B8480004FB00BF556A0700034610B470B10B49EA
:10B8580091F8DA4091F8DB200CB1944209D2013218
:10B8680081F8DB201A7A42F004021A725DF8044B60
:10B8780070475DF8044BFFF749BE00BF8001002008
:10B88800034610B4A0B10C4C94F8DA1094F8DB20FD
:10B8980031B101318A4204DC5DF8044BFFF702BF85
:10B8A80012B1013A84F8DB201A7A22F004021A72E3
:10B8B8005DF8044B704700BF8001002038B50D4685
:10B8C8000649CC7938B12B689C4228BF1C46C4EB8A
:10B8D800C4028CF047F92C6038BD00BF80010020FD
:10B8E80070B5044611BB20B325496BF03AF800BB8C
:10B8F8002046FFF775FD00283BDA237853B9214825
:10B90800C279002A35D121466BF024F80123C3718E
:10B91800104670BD012B04D1A37903F0C003C02BDE
:10B9280007D00121184A19486BF023F86FF0150069
:10B93800EFE7144DEB79012B1ED005F188006BF071
:10B9480006F8C30707D4002CF0D020460C496BF04A
:10B9580008F80028EAD1EE792146731C3046EB71CD
:10B96800FFF756FD08B93046D3E7EB79013BEB7199
:10B97800CFE76FF07700CCE76FF00B00C9E700BFA7
:10B98800AEB50A0080010020207C0A00A0870900CB
:10B998002DE9F341044640B91A4A02211A486AF0CF
:10B9A800E8FF002002B0BDE8F081002141F2090063
:10B9B80001AAFEF795FF054608B1144AEDE7019E76
:10B9C8000622D6F80C80124908F1010738468CF097
:10B9D800F7F828B1062238460E498CF0F1F818B964
:10B9E8003046FAF7D1FDDCE7D8F801303046C4F824
:10B9F8000130BB882570A4F80530FAF7C5FD012091
:10BA0800D0E700BF4E7C0A00A0870900677C0A00C7
:10BA1800BBB50A00B5B50A0007B56846FFF7B8FF19
:10BA2800044BD87118B169460020FFF7F1FC03B048
:10BA38005DF804FB800100202DE9F041304E88B00C
:10BA4800F179002954D196F8764014F0010411D107
:10BA58002C4A02212C486AF08CFF0024F471162528
:10BA680000240127F379E0B283422BD8002B3FD082
:10BA780000203AE06A464FF60940FEF731FF08B168
:10BA8800224AE6E7DDF800C0DCF80C5095F80180A2
:10BA9800B8F1000F0ED0AB1C02AA12351746186871
:10BAA8005968083303C7AB423A46F7D1186838607B
:10BAB8009B88BB806046FAF767FDB8F1000FCDD1CF
:10BAC800134AC6E708AB05FB003353F8182C33F8C4
:10BAD800143C6946CDF80120ADF805308DF80070AA
:10BAE800FFF796FC01340028BCD008B0BDE8F0810F
:10BAF8000021084608B0BDE8F041FFF7F1BE00BFDD
:10BB080080010020857C0A00A0870900B17C0A001A
:10BB1800D17C0A0038B50C4661B108480578012D7A
:10BB280005D10130FFF7ACFC00B9257038BD002005
:10BB38000870FBE76FF01500F8E700BF80010020F0
:10BB48002DE9F0411D460E461746034648B145B15A
:10BB58000A0311D54C0708D50121284A28486AF05C
:10BB680008FF6FF01500BDE8F0816BF036F800288B
:10BB7800F9D101232B70F6E7B107047824D02149C5
:10BB88002FB1B20603D591F89020500632D5C4EBF8
:10BB9800C40411F80480B8F1010F09D10134184622
:10BBA80021446AF0B5FF0028DDD185F8008002E065
:10BBB800B8F1000FF9D02FB1B30642BF2B7843F08C
:10BBC80002032B700020CEE7720710D50D49C4EB95
:10BBD800C4040F5D012F07D1013421446AF098FF96
:10BBE8000028C0D12F70E7E7002FE5D1FAE76AF007
:10BBF800F4FFBEE76FF08500B5E700BFFA7C0A00E6
:10BC0800A08709008001002070B500F10F060446E6
:10BC18000D46072230460C498BF0D2FF03462078A8
:10BC280073B90522094902F02BFB044658B1057384
:10BC3800002101F05BFE2046BDE8704001F00ABE1D
:10BC480006223146EFE770BDAEB50A00A7B50A0077
:10BC5800F8B504690646456844B140F203432B40F1
:10BC680039D005F48263B3F5806F34D015F480635E
:10BC780002D115F4F84F2ED1184F3078FB79834252
:10BC880029D9C0EBC0000722154938448BF098FF2A
:10BC9800A8B115F0030306D197F82320082A02D883
:10BCA800B2689F2A17D915F0300F09D09CB1EB065E
:10BCB80008D405F46035B5F5603018BF0120F8BD2B
:10BCC800002CF6D1D6E902239A4204D81F2A02D9B9
:10BCD800B3F1807FEDD30020F1E700BF80010020A1
:10BCE800AEB50A0038B50E4D28466AF0B8FF10F018
:10BCF800010412D1A5F118031846582221468BF0E9
:10BD080057FF0346D5E8EF2F42F00102C5E8E12FBF
:10BD18000029F7D118465C7038BD0020FCE700BF49
:10BD280038320020F8B5044614F80F7B154B064648
:10BD38000D4607222046144983F822708BF040FFF5
:10BD480070B93846114902F0E3F9044610B96FF0AA
:10BD58000B00F8BD052101F0C9FD00202C60F8E7B3
:10BD68002146384602F024FA40B92146307802F0DC
:10BD7800CFF904460028EAD00621ECE76FF0150059
:10BD8800E7E700BF80010020AEB50A00A7B50A00AA
:10BD98002DE9F04F91B015460390506800221446E3
:10BDA8000691824212D1FB2C18D89F4BB3F8D83099
:10BDB8009C421ED99D480093022123469C4A68F064
:10BDC80029FD6FF0200011B0BDE8F08F296802341A
:10BDD80001EBC2014B7801321C44E2E7039B0821C6
:10BDE80003F118006AF03EFF0028DED06FF00A0069
:10BDF800E9E7FB2C6ED8039B0B2103F118006AF0CE
:10BE080031FF10B91F2C28BF1F244FF0FF304FF00F
:10BE1800FF31FEF793FB04F104080746002800F001
:10BE2800FF8041460C3069F003F94FF000090646DF
:10BE3800424600218BF0BCFE4946D5F8008006F149
:10BE4800040B6B6899450FD3039BF1705B78002254
:10BE5800337003233946737001230698B37011B009
:10BE6800BDE8F04FFEF73CBD98F80120881C131878
:10BE78009C4298F800C013D2BCF1090FA4EB000251
:10BE880001D1002A0ADC694801216A4A68F0AFFC3E
:10BE98003846FAF779FB6FF0150094E74FF0080C75
:10BEA8005FFA82FA0AF101030BF801300131C9B2D5
:10BEB8000BF801C0C3B2D8F80410584404938BF0AF
:10BEC80051FE049B09F101099A445FFA8AF108F1CD
:10BED8000808B6E7002110220CA88BF069FE00279D
:10BEE800012340F272600B933B4669680A958B42C6
:10BEF80007D100240123A046A34605935FB938461D
:10BF080061E72A68023702EBC30252781744874276
:10BF1800C1D80133EBE7FB2F4FF0FF304FF0FF3173
:10BF2800BA4628BF4FF0FB0AFEF708FB0AF10406E1
:10BF38000490002874D031460C3069F079F8039BDE
:10BF480081465B78002603704FF000035FFA8AF29F
:10BF580083700792031D55F83B2005EBCB0102EBDC
:10BF6800C80252780232944209D14A6808F101089D
:10BF7800904509BF00240024A0460BF1010BBBF13A
:10BF8800010F12D055F83B204FEAC80112EBC80C3C
:10BF98000BD09819FCB901249CF8012001329A555C
:10BFA8000136F6B2079AB242D5D8059BBF1B002BC3
:10BFB80031D0002F0CBF03230123002204990698D7
:10BFC80089F8036089F80130FEF78AFC00287FF4BD
:10BFD800FAAE059092E7012C05D1525C0136022495
:10BFE8000270F6B2DEE79CF80120AAEB0601121BEC
:10BFF80002328A4228BF0A46DCF804C0A11E614406
:10C00800099308928BF0AEFD089A099B14443244B8
:10C01800A4B2D6B2C6E7B7FA87F35B095B00CCE7F0
:10C028006FF06800CFE600BF800100202887090074
:10C038001F7D0A004D7D0A002DE9F3470F690D4663
:10C04800496890463A1E18BF01224C02064601650F
:10C0580005D5EB787F33DBB2932B00F204813046B1
:10C068000DF10303FFF76CFD0446002840F0E8805B
:10C0780006F10F03002F00F0E7802A6911684FF0DE
:10C08800FF30C6F80F109188998092794FF0FF31F0
:10C098009A71FEF753FA8146002800F0E7801921CB
:10C0A8000C3068F0C5FF0446002119228BF080FD92
:10C0B80073782370AB68E370C3F307221B0C2271FB
:10C0C8006371EB68A371C3F307221B0C2372E2713F
:10C0D8006A6812F4004F14BF06230723D00348BF31
:10C0E80003F00503910348BF03F0FB0363729DF857
:10C0F8000330A3726B685A0254BF7F2395F903304B
:10C10800E374012323756B6803F44063B3F5806F10
:10C1180014BF01230223A3756B68DB0442BF03230A
:10C128002375A3756A68C2F3802383F001031B019A
:10C1380050049BB248BF43F04003910448BF43F00A
:10C148002003D20544BF012222766A6890077DD079
:10C1580043F0010A1FB9510501D443F0030A9005C1
:10C1680002D4B8F1000F03D04AF0020A1FFA8AFA83
:10C17800002F6DD0D1062A6948BF4AF00403116820
:10C1880058BF4AF00C03C4F80B1091889BB2A4F86E
:10C198000F10927962746A7801AFE275AA784946FD
:10C1A8006275A4F801303A4642F23600FEF798FB71
:10C1B8000446002844D1019BDB6893F90130B37031
:10C1C800D7E8EF0FC7E8E34F002BF9D108B1FAF72A
:10C1D800DBF906F11807D7E8EF3F43F00203C7E899
:10C1E800E23F002AF7D16FF0100138466AF041FDAE
:10C1F800C2062FD46A68092112F0030218BF01226F
:10C2080038466AF041FD0A213846CAF340026AF00E
:10C218003BFD2A790C213846C2F380026AF034FDCE
:10C228006A790B213846C2F380026AF02DFD9DF829
:10C2380003200321531E5A4238465A416AF024FD0E
:10C24800204602B0BDE8F0870A4A17E79A4686E713
:10C258005346A0E7304606F109016AF059FC002868
:10C26800C8D00446ECE76FF01504E9E76FF06804FE
:10C27800E6E700BFAEB50A0008B520B904486AF081
:10C28800EEFCC30701D4002008BD0248FCE700BF4C
:10C298003832002020320020034610B504486AF0E6
:10C2A800DEFCC20703D5BDE810400248184710BDA0
:10C2B800383200202032002010B5054CA06930B17A
:10C2C8006FF0010118306AF0D4FC0023A36110BD9F
:10C2D8008001002010B5164B9C693CB90121154A14
:10C2E800154868F084FA0024204610BD20466AF0FC
:10C2F80051FD04F11802082110466AF0B3FC10B988
:10C30800FFF7DAFFEFE7092110466AF0ABFC18B136
:10C3180000212046FFF778FC0022204611466AF0EB
:10C32800F4FC04460028DFD1FFF7C6FFDCE700BFB6
:10C3380080010020667D0A002887090010B50A4B95
:10C3480020389B6983420AD1FFF7C4FF034648B1EE
:10C35800BDE810400221054A054868F051BA6AF064
:10C368001CFDF3E710BD00BF800100209D7D0A0081
:10C37800288709002DE9F04FDFF888B10646DBF879
:10C3880018400F469046994685B0002C40F09E8094
:10C39800FFF7A8FC0546CBF81800002800F09980A4
:10C3A8000BF18800D6F810A0ADF808408DF80A40C7
:10C3B80003946AF054FC410774D573685A0574D421
:10C3C80032690AB19B0770D03046FFF741FC00285C
:10C3D8006BD005F1180B082158466AF043FC002879
:10C3E80066D143486AF03BFC440501D5FFF706FADD
:10C3F8003378B9F1000218BF0122314628462B7064
:10C40800FFF71AFE044660B9BAF1000F0CD10E9B73
:10C418004246009339464B4628466AF0E9FC0446F2
:10C4280080B1FFF749FF33E07368D8060AD4802348
:10C43800ADF80830DBE8EF3F43F08003CBE8E23F9C
:10C44800002AF7D17368990716D10121284602AA54
:10C458006AF05BFC0446B8B10121264A264868F018
:10C46800C6F9039E002EDCD03046002101F03EFACA
:10C47800304601F0EFF9D4E7284603A9FFF752FC4C
:10C4880004460028E1D0CCE7039808B101F0E2F9AE
:10C498003946002340F2011098450CD1204605B0DA
:10C4A800BDE8F08F6FF00A04BBE76FF01504B8E73A
:10C4B8006FF07704B5E70A88824204D14A6812B15E
:10C4C8001278D20708D401330831E5E76FF0770412
:10C4D800E4E76FF00B04E1E72035284607496FF0E1
:10C4E80007FE00232846064A27F014FDD6E700BFBA
:10C4F80008020020827D0A002887090045C3000041
:10C508001C4E0E00800100202DE9F341C6687078AA
:10C51800FFF7B2FE044638B90121364A364802B060
:10C52800BDE8F04168F063B904F1180875886AF04D
:10C5380031FC6FF4807140466AF09BFB33782F4FD3
:10C548001BBB2846012101F0EBFA054650BB6FF0F2
:10C55800800140466AF08DFB03060ED520466AF03E
:10C5680055FBFFF74BF963683BB11B682BB1327978
:10C5780020468DF8042001A99847BB699C4235D113
:10C5880002B0BDE8F041FFF797BE092140466AF0C6
:10C5980069FB18B120463178FFF736FB3378002B5A
:10C5A800D5D1CEE7236D00F17E0213F4002F12D00F
:10C5B800A368C0F87E30A3899380A37B93716368D6
:10C5C8002BB15B681BB12046019501A99847284605
:10C5D80001F040F9BBE7037AC3EBC303F918FB5832
:10C5E800C0F87E308B8893808B79E7E702B0BDE88E
:10C5F800F08100BFBC7D0A00288709008001002067
:10C608007FB5C5682878FFF737FE044638B9012199
:10C61800134A144804B0BDE8704068F0E8B84368AD
:10C628008BB19B687BB10135284669F0CBFF02AE20
:10C63800294650B1304669F0BAFF636820469B68C6
:10C64800019601A9984704B070BD20786AF054FAA1
:10C658000346006802909A889B79B280B371ECE730
:10C66800BC7D0A0028870900034B1A7A012A04BFF7
:10C6780002221A72704700BF31D4002008B5094859
:10C688006FF044FD031E04DA0121074A074868F0E9
:10C69800B7F80022064B99689A801960054B1A7200
:10C6A80008BD00BFC8020020D07D0A00C08709006D
:10C6B8008C08002031D40020F0B505460F464FF015
:10C6C800FF304FF0FF3187B01646FDF737FF0446BD
:10C6D800C0B106210C3068F0ABFC468000264770DC
:10C6E800057006714671094A204603A9052300957D
:10C6F800FDF712FF3246214642F24200FEF7F0F8FB
:10C7080007B0F0BD6FF06800FAE700BF080200202C
:10C7180038B50546407A0C46FDF738FF2073A87AED
:10C72800FDF734FF607395F90C30A37195F90D305E
:10C738006371EB7A2371EB8963812B88103BDBB241
:10C748000B2B8EBF0523054AD35CE3712B8883F03E
:10C75800100303F01F03238138BD00BF2FB60A0062
:10C7680008B50C4B0246400903EB80006AF06CFBED
:10C7780002F01F0340FA03F313F0010006D122B9B7
:10C7880005486AF061FB40F3C01008BD6FF0770000
:10C79800FBE700BFEC640020080200202DE9F04709
:10C7A80088B0002200238E4826F0E6FF06460028BF
:10C7B80040F0CB808B486AF047FB10F0010F894DA1
:10C7C8007ED02B1D93E8070008AB03E907008648D5
:10C7D8006AF03AFBC0F3401382486AF035FB04461E
:10C7E800002800F0A3808BB10C22804905A88BF0AB
:10C7F800E7F90446002800F0A480002211461046FC
:10C80800FFF75AFF0446002840F09B8076486AF0FC
:10C818001BFB410501D5FEF7F1FF9DF815502A07CE
:10C8280057BF9DF8143000278DF80430BDF8163036
:10C838005FBF01AFADF80530BDF81830ADF807306F
:10C8480015F0040500F0C880BDF81C200AB9BDF831
:10C858001620BDF81E300BB9BDF818309DF814101D
:10C86800ADF80D208DF80C10ADF80F3003AD002F8A
:10C878006FD03B78012B71D0002D6AD10025BDF80F
:10C888001A3006F0010043B1574BD3E8EF1F41F0CF
:10C898004001C3E8E21F002AF7D10DF103016AF055
:10C8A800CFF9044600284CD14FF0FF304FF0FF314C
:10C8B800FDF744FE8046002852D16FF0680440E03E
:10C8C80049486AF0C1FA10F0800F494A0ED09089A1
:10C8D800D18913694FF48072ADF81600ADF81420B1
:10C8E800ADF81810ADF81A60079370E7414C05AB26
:10C8F8002068616803C3A068186092F891303948CD
:10C908001F0744BF05238DF815306AF09DFA840788
:10C9180006D53023ADF818306023ADF8163056E749
:10C9280030486AF091FA4007F3D450E74BB1024619
:10C938000146FFF7C1FE044618B92C4B2861C3E92C
:10C948000100274826F08AFF2646304608B0BDE891
:10C95800F0872E78731E5E425E4190E71E468EE792
:10C9680000F10C090321484668F062FB9DF803308A
:10C978009DF815A00370CAF34003064684704370FF
:10C9880037B10123052283703946484668F056FBC3
:10C9980045B1B378052243F0040329464846B370ED
:10C9A80068F04CFB0022414642F24100FDF798FF37
:10C9B80004460028C5D10120BDF81A200AF001015B
:10C9C800FFF77AFE04460028BBD1084B08AA12E9F3
:10C9D800070083E80700B4E7002F7FF44AAF4DE76C
:10C9E80008650020EC64002008020020FC64002098
:10C9F80080010020108A0900002347F6122210B592
:10CA0800064827F087FA031E06DABDE81040012120
:10CA1800034A044867F0F4BE10BD00BFC8020020F6
:10CA2800FD7D0A00C08709000022024B1A60FFF74B
:10CA380025BE00BF3865002010B5442200210848F3
:10CA48008BF0B6F8064B03F11C001C466FF053F947
:10CA580004F130006FF04FF9BDE81040FFF7E4BF74
:10CA6800EC6400200022044B801A597C18BF012076
:10CA780001F00101FFF720BEEC640020032870B527
:10CA8800054603D1BDE87040FFF788BEFFF768FE92
:10CA98000446B0B9012605F01F039E400A4B6D09F4
:10CAA80003EB8505D5E8EF3F3343C5E8E23F002AAD
:10CAB800F8D1FFF773FE044618B1F14328466AF02F
:10CAC800C6F9204670BD00BFEC640020032808B5F5
:10CAD8000AD0012100F01F039940054B4009C943C2
:10CAE80003EB80006AF0B3F9BDE80840FFF756BED3
:10CAF800EC6400202DE9F74F05465E486AF0A4F97A
:10CB080000F001085B486AF09FF90E461446994602
:10CB18008246B8F1000F03D00B895A0700F1A680AE
:10CB2800284669F04FFD6F46002868D029466846B8
:10CB380069F03DFDB8F1000F02D11AF0040F28D1B9
:10CB48004D4BD3F800B0BBF1000F13D02268A36897
:10CB5800B4F804A0A4F80490A2EB030838462346CE
:10CB6800F27996F90510D847A368A4F804A013FA37
:10CB780088F32360414B37601A6842B152F808893C
:10CB8800B8F1000F01D0A8F10808002A47D1002306
:10CB98003360384833896AF057F910F0010665D1D7
:10CBA800DB0763D503223946304601F069FB0446AA
:10CBB80000285BD00220FFF789FF2B682046C4F8C5
:10CBC8007E30AB88A4F88230AB7984F8843069F081
:10CBD800F5FD002843D01F2331462373204600F07B
:10CBE80085FE204600F036FEFFF7D8FD03460028F4
:10CBF8003CD00221224A234867F002FE36E02B7817
:10CC0800FF2B07D1204B186800909A889B79BA802F
:10CC1800BB718FE7294669F06FFF0346F3E7136896
:10CC28008BB12168A368B4F804B0A4F80490A1EB10
:10CC3800030A3046136821469847A368A4F804B04D
:10CC480013FA8AF32360B8F1000F06D0D8F8083039
:10CC580003B1083B4246984697E74346FAE7204621
:10CC6800022100F043FE204600F0F4FD03B0BDE8C9
:10CC7800F08F00BFEC64002038650020306500208C
:10CC880081720A00C0870900AEB50A0010B50020FD
:10CC9800FFF71CFF58B16FF0ADFA0020FFF716FF41
:10CCA800034620B10221124A124867F0A9FD6FF02D
:10CCB800400111486AF0CBF86FF480710E486AF0B1
:10CCC800C6F8FEF79BFD0D4B1B6823B153F80849C6
:10CCD80004B1083C03B910BD5B6803B198472CB197
:10CCE800A26802B1083A23461446F3E72246FAE757
:10CCF8002E7E0A00C0870900080200203065002047
:10CD08002DE9F04F00F10C0989B00746484668F054
:10CD1800E4F906465D486AF097F800F001035B48BD
:10CD280003936AF091F85A4DC0F38003DFF874A1B9
:10CD380002939EB1039B53B13B8A172B11D8012153
:10CD4800544A554809B0BDE8F04F67F050BD2B7AFA
:10CD58000BB1FFF793FC029B002BEDD109B0BDE8A6
:10CD6800F08F1821484668F0B0F93A8AC37DB0F8C8
:10CD780000B09342CBF3411804460BF0100B0FD9C7
:10CD8800454800920221454A67F044FD384668F05C
:10CD9800B8F8BBF1000FE1D102223D4B1A72DDE772
:10CDA800BBF1000F0DD004A9FFF7B2FC4A46E37DA2
:10CDB80004A9A01CFFF79EFE4846E17D68F07DF9B6
:10CDC80029E095F808B0BBF1000F37D0C27AEB79AB
:10CDD8009A4205D1811C072228468AF0F1FE48B301
:10CDE800B8F1000F02D1204604A9DDE7BBF1010F1D
:10CDF80027D102212A4A284867F0F9FCDCE72B7A78
:10CE0800022B3DD05046F96868F018F9B8F1010FC7
:10CE180004D1FFF7F1FD013EF6B28AE7204604A9E6
:10CE2800FFF776FC5246BAF8043004A9A01CFFF7B5
:10CE380061FE28E0B8F1020F18D124E0B8F1000F24
:10CE4800D1D0B8F1020F1ED0BBF1020F01D1FFF70C
:10CE580015FCD4F80220E37A2A60E288EB710123FA
:10CE6800AA80227A2B72AA71FFF7C6FDE27DBAF872
:10CE78000430BAF8061013448B42C0DD02232B722B
:10CE8800B8F1010F98D0FFF7F9FB95E7EC640020A3
:10CE980031D40020577E0A00C0870900707E0A003E
:10CEA8009A7E0A008C0800202DE9F04F00F10C074B
:10CEB80085B00646384668F010F905462A4869F0F4
:10CEC800C3FF00F00109284869F0BEFF4FF0010ACE
:10CED800DFF8A0B0C0F3800815B905B0BDE8F08F41
:10CEE800B9F1000F02D1B8F1000FF6D0338A082B40
:10CEF80007D801211D4A1E4805B0BDE8F04F67F06C
:10CF080076BC0921384668F0E0F8037A328A0133A2
:10CF18009A420446EDD37F23ADF80CA08DF8063075
:10CF2800037A694603445B7A01308DF80530FF23A4
:10CF38008DF804300023ADF80A3010F8012C013DBB
:10CF4800042A98BF1BF802308DF80720ADF8083086
:10CF5800C3793A46FFF7CEFD217A3846013168F0A9
:10CF6800ACF8EDB2B8E700BFEC640020577E0A00C9
:10CF7800C08709003BB60A00F8B50546224869F0A3
:10CF880063FF43070F463CD52A78012A03D96FF07F
:10CF980015042046F8BD6B780F2BF8D843F6FC74BF
:10CFA8006888031F9BB2A342F1D8A9880B1F9BB2C4
:10CFB800A342ECD88842EAD37AB900220023134866
:10CFC80026F0DAFB04460028E3D1FFF7C9FB044644
:10CFD80040B10E4826F042FCDBE769F015FE002858
:10CFE800EBD1D4E728686968094E0A4B03C6A868DC
:10CFF8001F6030602046FFF741FD044606F124001B
:10D00800E8E76FF00A04C4E7080200201C65002066
:10D01800F06400203865002008B5FFF705FD002200
:10D028000A4B6FF040010A481A6069F010FF430686
:10D0380006D56FF48071064869F009FFFEF7DEFB3C
:10D04800BDE808400020FFF741BD00BF386500205B
:10D05800080200200A4A00F10803116831B981600A
:10D06800516839B9C2E90033002070478B4204D0B7
:10D078000968F3E70B605360F6E76FF0100070473C
:10D088003065002008B5034869F0DEFE00F00100B5
:10D0980008BD00BFEC64002070B59AB014220021CE
:10D0A80004A88AF085FD47F21213ADF80C304FF44E
:10D0B800807344F20102ADF80E30364B01A903A883
:10D0C800CDE905235FF04CFC034618B3324A012131
:10D0D800324867F095FB1F25314BD3E8EF1F21F04D
:10D0E8000101C3E8E21F002AF7D12E4E27F0BEFA4D
:10D0F800346804B1043C002D2B4D18BF0025002CCA
:10D1080041D023680BB1284698476468002C3AD070
:10D11800043CF6E702AB4122019809A989F0DEFB3D
:10D12800034608B1214AD2E7214A0DF125030DF142
:10D13800650153F8040B8B4242F8040BF9D102AB9A
:10D1480020221C49019889F071FB034608B11A4A4C
:10D15800BDE7019889F022FB054610B1174A03463E
:10D16800B5E71349104869F07DFE1548203169F08C
:10D1780079FE144BD3E8EF1F41F01001C3E8E21F1A
:10D18800002AA9D0F6E70023C6E9003327F082FA7F
:10D198001AB070BD00000209BF7F0A00808709002D
:10D1A8003C650020446500207FD50020DD7F0A0013
:10D1B8003FD500201FD5002000800A0024800A00E7
:10D1C8009FD500200802002030B5A7B01422002106
:10D1D80008A88AF0EDFC04233D22002116A8159327
:10D1E8008AF0E6FC47F21213ADF81C304FF4807356
:10D1F80044F20102ADF81E30284B2949CDE9092334
:10D2080007A805AB202289F093FB0346E0B1254A25
:10D218000121254867F0F4FA6FF0040427F026FA94
:10D22800224B1D6865B100201860214BD3E8EF1F21
:10D2380021F00201C3E8E21F002AF7D144B3A8474E
:10D2480027F028FA27B030BD1A4B0DF155021946C0
:10D2580003F1400053F8044B834242F8044BF9D1E0
:10D2680006AB029320230D48CDE9001315AA4123EC
:10D27800059989F030FD034608B10F4AC8E70598BB
:10D2880089F08CFA04460028C8D00C4A0346BFE748
:10D298000DA8084969F0E6FD0DA8D0E700000209CD
:10D2A8001FD5002044800A008087090040650020BF
:10D2B8003C6500203FD500207A800A0096800A004D
:10D2C800402208B503498AF07BFCB0FA80F0400997
:10D2D80008BD00BF40B60A0010B598B00446142235
:10D2E800002102A88AF064FC44F21213ADF804305D
:10D2F8004FF480734FF48042ADF80630144B21464A
:10D30800CDE9032304230DF11D008DF81C3069F0CD
:10D31800A9FD04F120010DF13D0069F0A3FD6B4664
:10D32800412207A901A889F003FB044601A889F056
:10D33800F8FD2CB9009889F031FA012018B010BD19
:10D34800044823460121044A67F05AFA0020F5E709
:10D358000000020980870900B3800A0010B5002880
:10D3680034D01D4A136823B1043B984231D05B681E
:10D37800F9E71A4BD3E8AF1F890707D518480221E8
:10D38800184A67F034FA6FF00F0010BD1468011DD9
:10D3980044605068116000B95160D3E8EF2F42F043
:10D3A8000101C3E8E01F0028F7D1D30701D5002009
:10D3B800EBE70D4BD3E8EF1F21F01001C3E8E21FA4
:10D3C800002AF7D10948FCF7F7F8F0E76FF01500E5
:10D3D800DBE76FF07700D8E7446500203C65002064
:10D3E80080870900D7800A0008020020A8080020CA
:10D3F800044BD3E8AF3F13F0100F034808BF0020D9
:10D40800704700BF080200207FD5002070B5054690
:10D41800194803688B4228D0184BD3E8AF3FDA0687
:10D4280026D5036813B16FF00F0070BD144AD2E817
:10D43800AF3FDB07F7D4D2E8EF3F43F00204C2E87E
:10D44800E64F002EF7D113F00204ECD10160294613
:10D458000C4869F007FD0C4805F1200169F002FD50
:10D468000A48FCF7A9F82046DFE76FF07700DCE709
:10D478006FF07C00D9E700BF40650020080200205B
:10D488003C6500203FD500205FD50020980800208B
:10D4980070B505460B4B1C6844B154F81C3C1C3C49
:10D4A80013B12846297B9847E469F5E7064C074EEF
:10D4B800B44200D370BD236813B12846297B98472E
:10D4C8002034F5E7C0650020D886090018870900D0
:10D4D80010B50446F8F7B8FF044901EB00112046DF
:10D4E80069F0B1F8BDE81040FDF7A0B94C6500201F
:10D4F800002270B50446D1E901560748C1E9012266
:10D508006EF0B6FC3DB1314620462B46BDE8704072
:10D518006FF06D02184770BD6C21002030B5051DF5
:10D5280004464FF48061284685B069F0C5FC400583
:10D5380033D4284669F0BBFC810321D5E17871B367
:10D54800637B072B29D1224B93F890309B0624D577
:10D5580069F009F908B30DF10E0103A8FDF76AFA9D
:10D56800D8B92046BDF80E20BDF80C1069F067F94F
:10D57800034690B10121174A174869F09BFC0CE05B
:10D58800204669F041F9034620B10121134A1248A7
:10D5980069F090FC637B072BD0D005B030BD0C4BF5
:10D5A80093F89130DA0706D4022319460C4A0A4840
:10D5B80069F080FCC4E7022320461A46009169F00E
:10D5C8005DF903460028BBD00121064AEFE700BFFA
:10D5D8008001002056810A004087090005810A0061
:10D5E80026810A003F810A0070B505460022002303
:10D5F8000E4826F0F5F9B8B90D4B1C6834B154F84B
:10D60800143C1C3C03B19847E469F7E7094C0A4EFF
:10D61800B44204D32846BDE8704026F0D3BBA368C3
:10D6280003B198472034F3E770BD00BF48210020BC
:10D63800C0650020D8860900188709002DE9F04147
:10D64800044620270025EFF3118287F31288BFF3E1
:10D658006F8FE16929B1206A0B688142E36108BFD5
:10D66800236282F31188BFF36F8F71B1D1E901682A
:10D678000748C1E901556EF0FBFB1EB10022414687
:10D688002046B047FDF7D2F8DDE7BDE8F08100BFDE
:10D698006C2100200348B0F8BC30C030002B08BF14
:10D6A800002070478001002030B50446F8F7B6FB2B
:10D6B8000D460D4A0D498BB00858D2F8E010884243
:10D6C80005D120460BB0BDE83040FFF7B7BF243482
:10D6D800214610466EF0DAFC1DB1694620466EF010
:10D6E800E5FC0BB030BD00BF9051002008000000E1
:10D6F80038B5002204468A4202D10024204638BDAB
:10D70800012004F1C803D3E8EF5F002D04D1C3E87A
:10D71800EC0FBCF1000FF6D102D0D0340244EAE796
:10D72800002CEAD0C822002120468AF041FA04F1F0
:10D73800400004496EF0DCFC034904F124006EF05B
:10D748007AFCDBE7DDE50000E36E0700F7B5164677
:10D758000D4601210446FFF7A7FF012E23D0022E14
:10D7680052D123693BB135480121354A67F03FF86A
:10D77800204669F0D0FB25612269138A012B5AD90A
:10D78800D2681288043292B2934254D343D9012109
:10D7980000922A482B4A67F03DF8204603B0BDE8BE
:10D7A800F04069F0B8BB206940B9274A31462348A0
:10D7B80067F01DF8204669F0AEFB01E02A8A2AB915
:10D7C800284603B0BDE8F040F8F7DEBE018A438A78
:10D7D80047695B1AC168C91B5B1A9A420CD91B4A74
:10D7E8003146164867F003F800222046216901F007
:10D7F800E7F900232361E3E7E9680C3067F01EFCD2
:10D808002846F8F7C1FEB7E701213346104A0B480E
:10D8180069F050FBCEE7002204F11003D3E8EF1FB4
:10D82800C3E8E02F0028F9D10122204603B0BDE863
:10D83800F04001F0C5B903B0F0BD00BF4087090052
:10D8480072810A00F2810A008F810A00AD810A0004
:10D85800D4810A0008B500F1C803D3E8EF2F013AD4
:10D86800C3E8E12F0029F8D1AAB90B4B984212D38B
:10D8780003F5826290420ED2C01AD023B0FBF3F2B5
:10D8880003FB120038B9054826F06EF8BDE80840D9
:10D89800034826F097BA08BD7832002048210020B6
:10D8A800C808002010B5044669F044FB26F0DEFEE7
:10D8B8000C4B04F1BC01D3F8DC3043B90A4869F0D9
:10D8C800DBFA26F0E7FEBDE81040FCF7AFBF99424F
:10D8D80001D01B68F1E726F0DDFE2046FFF7BAFF0E
:10D8E800F1E700BF800100205C020020F8B5457B0D
:10D8F80004468D420E4600AF1CD1082D98BF694BD7
:10D908006C4688B094BF53F82530674B6A46674920
:10D91800CDE905134FF40073ADF81C30644B42F8A1
:10D92800103F00234FF4E4516248F6F73DFFA54647
:10D93800BD46F8BD4173DDB1022D1CD0637B082BB9
:10D9480000F2AD8001A252F823F000BFB3D9000065
:10D958004DDA00001DDA000039D9000039D900007D
:10D9680039D9000039D900008DD9000039D9000013
:10D9780069F0E0FAE2E78378012BDFD140306EF0FE
:10D98800C5FBDBE70023C4E90D33E378012BCFD1D6
:10D99800A378494A012B04BF032384F89830002355
:10D9A80004F1400026F07EFAC2E7082DC0D8DFE86F
:10D9B80005F02A0521172626212A2A0004F1400508
:10D9C80028466EF0A3FB01212046FFF76DFE204696
:10D9D80069F0A1FA00220023284626F09BFAA7E75F
:10D9E8000220FFF773F8034620B10221334A314879
:10D9F80069F060FA237B13B12046FFF749FD204602
:10DA0800FFF728FF94E733462D4A0221294869F099
:10DA180051FA8DE7A378012B8AD12A4B9D8A002DD4
:10DA280086D00A2340F2E730002147F612265D43EC
:10DA38004FF47A720023E5FB0601F3F76DFB02460B
:10DA48000B46ADE7237B3E2B0FD16D4688B06A4667
:10DA58001D4BCDE90534032342F8103F00234FF452
:10DA6800C4511448F6F7A0FEAD46164D05F1C006A0
:10DA7800616911B9FCF7DAFE5AE7A2690B689142AD
:10DA880008BFA36120466361FFF732FDB5F8BC30DB
:10DA9800002B14BF3046002025F066FFE8E70B4A4C
:10DAA8003346B2E7F89009000D820A0017820A008F
:10DAB80003000001408709005A62020028820A0018
:10DAC80059820A008001002070820A0097820A00A9
:10DAD8002DE9F04706460F46904600254FF0D0093D
:10DAE800DFF828A009FB05A069F024FA044620B154
:10DAF80083781E4206D1FFF7ADFE0135052DF1D121
:10DB0800BDE8F0874146B8472046F4E77832002060
:10DB1800002201200149FFF7DBBF00BFD76E0700D5
:10DB28002DE9F04105460E460027DFF858804046AB
:10DB380069F000FA044658B1437B012B02D0073B39
:10DB4800012B03D82388AB420BD02046FFF782FE77
:10DB58000137052F08F1D008E9D100242046BDE897
:10DB6800F081A3781E42F9D102212B46034A0448CA
:10DB780069F0A0F92046FFF76DFEEEE7B3820A00D0
:10DB88004087090078320020034BC01A034B00116C
:10DB98005843C0B2704700BF78320020C54EECC46D
:10DBA80070B51C46144305460E460DD0F8F736F9F5
:10DBB8000E49D1F8E0400E4909588C4206D102219D
:10DBC8000C4A0D4866F013FE002213460B49002D3F
:10DBD80014BF2846084667F099F9044618B1711D24
:10DBE8000C3067F01AFA204670BD00BF9051002033
:10DBF80008000000CA820A0040870900842100202A
:10DC080010B50446054826F0DDF8204600F0D2FE9F
:10DC18002046BDE81040FFF73BBC00BFB808002015
:10DC28002DE9F04F002387B000AFFB607B61B94B53
:10DC38005A8B3AB1B84DD5F8DC403CB91C37BD46D3
:10DC4800BDE8F08F1B68002BF4D1F7E754F8BC3916
:10DC580003B1BC3B0026B14901E01C461346B5F8A8
:10DC6800BC20002A00F05481D5F8C8204AB904F134
:10DC7800BC06002BE2D0D3F8BC20002AEDD0BC3A79
:10DC8800EBE70A68002AF2D0D4F8A820002AEED0E0
:10DC9800D4F8AC20002AEAD0D4F8B020002AE6D084
:10DCA800637B072B6AD120469047002866D004F191
:10DCB800C00069F0FCF8022860DC204669F03AF9F7
:10DCC80004460028BAD0637B072B40F01E8120460B
:10DCD800D4F8A830B5F8BC1007F11002984781466F
:10DCE800002800F00581B5F8BC203B699A4208D3AA
:10DCF8000146D4F8AC60204607F1140307F10C0282
:10DD0800B0477B69D7F80C803B60B9F81030002B1E
:10DD180000F0F5804846D7F810A068F0AAFC7860B3
:10DD2800002840F0EF80B5F8BC30DFF800B2002BD7
:10DD380014BF584600200022002325F051FE78B970
:10DD480000220023754825F0D9FD064600283BD15E
:10DD5800B5F8BC30002B18BF5E46304625F004FEEF
:10DD68006FF00B054846F8F70FFCB8F1000F00F00C
:10DD7800AA802A4620463968C047A4E0D4F8BC30B7
:10DD880004F1BC02C6B9D5F8E010C5F8DC308A4207
:10DD980001D1C5F8E03000232046C4F8BC30D4F8DF
:10DDA800B030984700288ED0637B072B40F0AD80B9
:10DDB8002046FFF777FD86E73360D5F8E0309A42D2
:10DDC80008BFC5F8E060E6E73B68C0F804808360F8
:10DDD800B5F8BCB00022DA454FF000034FF000015F
:10DDE8004C4898BF1FFA8AFBF8F750FB804650B1A1
:10DDF800F8F72AFB4A4B5A4603EB001349464046BC
:10DE080068F0FCFB8046B5F8BC3094F8C4909A459D
:10DE180084BF01237B607B689CBF09F102095FFA1C
:10DE280089F984F8C43004F1C00ADAE8EF3F013315
:10DE3800CAE8E23F002AF8D104F1140B31465846EB
:10DE480069F01AF8A378012B56D108F10C030421C4
:10DE580018467B6067F020F9228809F0FD0942EA3C
:10DE680009320280B8F810207B68043A4280022107
:10DE7800184667F019F94046FCF75AFC8146002815
:10DE880043D0DAE8EF3F013BCAE8E23F002AF8D185
:10DE98003146584669F024F8224A4B460121224867
:10DEA80069F008F84046F8F76FFB20463146FFF75F
:10DEB8001FFBB5F8BC301D48002B08BF002025F01B
:10DEC80053FD6FF004056E4688B0194A0423CDE966
:10DED80005256A46079442F8103F4FF4015112484D
:10DEE8000023F6F761FC1321B546204669F039F89E
:10DEF8002046FFF7AFFCA1E66FF01509C1E76FF008
:10DF080079052FE76FF004052CE7FCF78FFCEFE7A6
:10DF18009368FFDE34220020800100206C2100205D
:10DF28004C650020E7760A0040870900400200207F
:10DF3800F3820A0040F2E2432DE9F041D0F888600C
:10DF48000446B6FBF3F6031D184668F0B0FF8204DA
:10DF5800B6B213D5B4F88C20B2420FD8B4F88E20DC
:10DF6800B2420BD3D4E92412914207D1D3E8EF1F70
:10DF780021F40051C3E8E21F002AF7D1104B1D68B5
:10DF880065B155F80C7C1C3D37B131462046B4F8D4
:10DF98009230B4F89020B847ED69F1E7094DDFF801
:10DFA8002880454501D3BDE8F0812F6937B1314656
:10DFB8002046B4F89230B4F89020B8472035F0E7FE
:10DFC800C0650020D8860900188709002DE9F041AE
:10DFD800074608460D4668F0C8FB064618B90026ED
:10DFE8003046BDE8F081144B1C6884B154F8103CED
:10DFF8001C3C0BB9E469F8E72946384698470028DD
:10E00800EDD0284668F0B1FB0028F3D1E7E70B4CC8
:10E01800DFF82C804445E3D2E3680BB92034F9E7F4
:10E028002946384698470028D9D0284668F09DFBED
:10E038000028F3D1D3E700BFC0650020D8860900C7
:10E04800188709002DE9F041C37804468BB900F11F
:10E058007E06114B1D687DB11C3D04F170076B698C
:10E068001BB13A46314620469847ED6925B11C3D1B
:10E07800F5E700F17706ECE7084D094F04F1700861
:10E08800BD4201D3BDE8F0816B691BB14246314600
:10E09800204698472035F3E7C0650020D886090058
:10E0A80018870900F8B5437A04468372164669F062
:10E0B8002AF9144B1D684DB155F8043C1C3D1BB1A1
:10E0C80032462046617A9847ED69F4E70E4D0F4FC6
:10E0D800BD420DD3A6B9637A012B11D9A378012BC0
:10E0E8000ED1207A04F17001BDE8F84006F030BF87
:10E0F800AB691BB132462046617A98472035E7E77D
:10E10800F8BD00BFC0650020D8860900188709003F
:10E1180038B505460C460F480521FFF7E9FAC0B1A6
:10E12800057223680367A388A0F87430A37980F880
:10E1380076300123437283728370074BC0F8A8308E
:10E14800064BC0F8AC30064BC0F8B030054BC0F8F1
:10E158008C3038BD78320020BDE80000A16E070081
:10E16800956E0700180028002DE9F04107468846FB
:10E1780000250E4E304668F0DDFE044620B1837857
:10E18800012B0AD0FFF766FB0135052D06F1D006F5
:10E19800F0D100242046BDE8F0814246394668F0B7
:10E1A800D4FF0028F6D12046ECE700BF78320020E3
:10E1B800F0B589B000AF0D46FFF7D6FF044618B397
:10E1C80029463846FBF762F9637B6D46082B98BFF2
:10E1D8000F4A8AB094BF52F823300E4B6A46CDE9F5
:10E1E80007730D4B0D4909930D4BCDE9051442F802
:10E1F800103F00234FF442510A48F6F7D5FA20465B
:10E20800AD46FFF727FB01202437BD46F0BD00BF10
:10E21800F89009000D820A000103020416830A001F
:10E22800050000024087090038B50446134868F025
:10E238003EFE420702D46FF00A0038BD084668F077
:10E2480094FA10B96FF01500F7E7FEF71BFF0028E6
:10E25800F1D10A4868F02BFE0306C0F3C0150AD4B2
:10E2680068F0D2FC0028EDD021462846FFF7A0FF31
:10E278000028E2D0E6E76FF07700DEE7080200202A
:10E288002DE9F04706460F46904600254FF0D00985
:10E29800DFF844A009FB05A068F04CFE044620B155
:10E2A8008378012B06D0FFF7D5FA0135052DF1D17A
:10E2B80000240DE037B13A46314668F046FF08B908
:10E2C8002046F0E7637B4345FAD1237AB342F7D17E
:10E2D8002046BDE8F08700BF7832002070B58B7803
:10E2E8000646012B0C4692B042D191F8703007AD2A
:10E2F800032B37D8DFE803F0023032341E492846B2
:10E30800F2F76EFF059594F871301E21049394F886
:10E3180072301A4A039394F873300AA8029394F857
:10E328007430019394F87530009394F8763060F067
:10E33800E3FD32460AAB10AD1C4603CCAC4210607C
:10E348005160234602F10802F6D120681060304679
:10E35800A388938012B070BD0949D0E70949CEE778
:10E368000949CCE70A212846084A60F0C5FDC9E7F3
:10E3780000238DF82830DCE72C700A004E700A0064
:10E3880033700A003A700A0044700A00E2910A00E9
:10E39800002210B5837804460B70C3784B70037A5B
:10E3A8008B70437B81F82320023BDBB2062B8EBFA8
:10E3B80013462848C35C204681F82030A378012BF7
:10E3C80014BF0023637A81F8213068F050FE81F889
:10E3D8002200A378012B3AD104F170038B60237AD1
:10E3E8001D4AC3EBC30313444B60E27804F177037F
:10E3F80004F17E0012BB1A460346C1E9032340F22A
:10E40800E242D4F888304B61B3FBF2F30B83B4F8E3
:10E4180090304B83B4F892308B83D4F8A4302BB16E
:10E428005B7CDA0644BF012381F82330D4F8A4309A
:10E4380013B15B7C9B0603D4002010BD0246DCE7C9
:10E4480091F8233043F0020381F82330F4E76FF0AA
:10E458001500F2E780B60A00800100202DE9F0419E
:10E4680004460F4615469846002B6ED01B6823B10C
:10E478000221394A394866F0BAF929462046FFF799
:10E48800D3FE064600283FD12046294668F033FED1
:10E49800044600285CD097E80F00314D05F1080CC0
:10E4A8008CE80F00AB8A002B08BF4FF49673AB8241
:10E4B8002B8A03B9AB892B826B8A03B9EB8929486C
:10E4C8006B8268F0F4FC430501D5FDF797F995F8E0
:10E4D800DB2095F8DA309A4219D903212046FFF754
:10E4E80005FA0220FEF7CAFA054658B10220FEF7DF
:10E4F800EDFA20460021FFF7F9F92046FFF7AAF9BF
:10E508002E4601E0C8F800403046BDE8F0810221FF
:10E518002046FFF7EBF9204668F050F90546002839
:10E52800F0D0002120462173FFF7E0F92046FFF7DD
:10E5380091F90320FEF7A2FA03460028E0D0022151
:10E54800094A064868F0B6FCDAE76FF01506DBE71B
:10E558006FF00B06D8E700BF4F830A004087090019
:10E56800800100200802002081720A0038B50446A4
:10E5780008460D4668F0F9F838B3154B93F8903013
:10E58800990707D4E37873B129462046BDE8384097
:10E5980000F042BB94F899309A07F3D5201D68F033
:10E5A80086FC4304EED42946204668F0F4FD58B9A9
:10E5B8002B88A4F88C306B88A4F88E30AB88A4F82C
:10E5C8009430EB88A4F8963038BD6FF01500FBE75F
:10E5D80080010020F7B510F8333C0446A0F140064E
:10E5E8000BBB304668F032FE3C4B1D684DB155F808
:10E5F800183C1C3D1BB1304614F8341C9847ED6993
:10E60800F4E7374D374FBD4205D3304603B0BDE878
:10E61800F040FFF71FB96B681BB1304614F8341C83
:10E6280098472035EFE710F83E3C012B53D110F8FE
:10E638003D3C8BB9FCF726FB69304CD102212A4AB4
:10E648002A4866F0D4F840F239120023204603B075
:10E65800BDE8F04025F05EBCA0F13C05D5E8EF3FF1
:10E6680023F40052C5E8E12F0029F7D199041FD5FA
:10E67800E36C69460093636D30460193FFF776FFBC
:10E68800034678B9D5E8EF3F23F48053C5E8E23F65
:10E69800002AF7D14FF40061284603B0BDE8F040E6
:10E6A80068F00ABC124A0221104868F003FCF1E73E
:10E6B8004FF428130F4A69463046CDE90023FFF787
:10E6C80055FF034628B94FF48051284668F0F4FBFB
:10E6D800E0E7094AE7E703B0F0BD00BFC0650020E6
:10E6E800D88609001887090084830A004087090032
:10E6F800B7830A0018002800DC830A0008B568B14F
:10E70800094B00F10C011A6822B9074868F0B4FBFC
:10E71800104605E0914204D01268F5E76FF0150045
:10E7280008BD6FF07700FBE7C86500202DE9F041D0
:10E738001C486DF05FFB1C491A486DF099FB1B499A
:10E7480018486DF095FB1A4916486DF091FB69F071
:10E75800E6F904F0B3FA044600BB06F097F804465D
:10E76800E0B968F032FE2646A046124F384668F0F7
:10E77800E1FB054668B1043068F099FBC30705D58D
:10E788000321284685F80880FFF7B0F82846FFF7E8
:10E7980061F80136052E07F1D007E7D12046BDE81C
:10E7A800F08100BF6C2100209C650020A865002036
:10E7B800B46500207832002003460121014A02484E
:10E7C80066F01EB882840A00B087090080B500AFE1
:10E7D80088B06A46074BCDE90530032342F8103F5D
:10E7E80000234FF4C2510448F5F7DEFF6FF00B0029
:10E7F800BD4680BDAA840A00B087090070B5002212
:10E808005026094D06FB02F35C19EB583BB1013267
:10E81800052AF7D1FFF7DAFF6FF00B0003E018467F
:10E82800024A62600C6070BDD46500204491090002
:10E8380070B5044652EA030008D0F7F7EFFA074D1F
:10E84800074ED5F8E0503058854201D100221346D2
:10E858002046BDE870400431FFF7A2B9905100206E
:10E868000800000038B5054618462B68DBB15B7B0D
:10E87800072B18D10B7A012B07D001210B4A0C4822
:10E8880065F0BEFF6FF0150038BDCB7A072BF9D9BC
:10E89800C8618A6105F130006DF0EAFA284668F02F
:10E8A800ACFC0020F0E76FF07F00EDE7D1840A00B0
:10E8B800B08709002DE9F84F88469146D0F8B44052
:10E8C80000AF44B1483C236B63B92068B43068F0AA
:10E8D800B3FCA46CF5E7FBF7A9FF00263046BD465C
:10E8E800BDE8F88F04F1300A50466DF0E6FA0546A7
:10E8F8000028F0D067F0BDFE80B16C4688B06A464B
:10E90800294BCDE90535032342F8103F00234FF486
:10E91800C2512648F5F748FFA546DEE7284666F0C7
:10E9280037FBE56C06469DB9A38C058A403B9BB234
:10E938003F2B03D8238D9D4228BF1D46042106F195
:10E948000C0066F0A9FB0580A38C04354380E564C0
:10E9580045451FD8B6F810B0AB4506D100220023B4
:10E96800504624F0CBFFF7F70FFEA38CA3F140022B
:10E978003F2A06D8AB451ABF002213460C4AF3615A
:10E98800B2612068B43068F057FC236B13B120469D
:10E9980068F033FCE36C98452CBF0021A3EB080119
:10E9A800C9F80030E16499E7E9840A00B0870900F2
:10E9B80085730700F7B504460026234D234FBD4253
:10E9C80001D303B0F0BD2988204668F0CEFC6B68FF
:10E9D800019001A920469847002830DB019B2A882E
:10E9E8009A829A8403F11002D2E8EF1FC2E8E06F1E
:10E9F8000028F9D19E64DE649E60A16B03F10802D1
:10EA0800F9B9C4E90D221C60DE6003F130006DF035
:10EA1800F1F9019843681B6803B19847019B1033CB
:10EA2800D3E8EF1F41F00101C3E8E21F002AF7D144
:10EA380001984368DB6913B100F110019847083564
:10EA4800BDE70A60A263DEE7C0860900D886090030
:10EA58007FB50D460646042105F10C0066F035FB2E
:10EA68002A8A43880446934208D000931346444AAE
:10EA78000121444865F0CEFE04B070BD417839B933
:10EA88000121414A3F4804B0BDE8704065F0AFBE7F
:10EA98000278122A22D0132A1AD0012AECD0022195
:10EAA80013463848394A65F0ABFE617802220120E6
:10EAB800356868F040FC04460028DDD002210C309F
:10EAC80066F0B6FA0023214603704370284624E016
:10EAD800022BD1D0022200922D4AC9E7082B03D07D
:10EAE800082200922B4AC3E73468637B072B02D0C5
:10EAF8000221294AC6E7E378A3B10222012068F07F
:10EB08001AFC05460028B7D002210C3066F090FAAE
:10EB18000023294603704370204604B0BDE87040C6
:10EB280068F039BCEB6813201A88ADF808205A88B9
:10EB3800ADF80A209A88ADF80C20DB880222ADF8DF
:10EB48000E3068F0F8FB0546002895D002A920464B
:10EB5800FFF73CFA0646022105F10C0066F068FA58
:10EB680086F00103DBB203802946204668F013FCD7
:10EB7800002E81D0204602A968F00DFB7CE700BF7B
:10EB880001850A00B087090022850A00AE850A00BF
:10EB980043850A006E850A00A0850A0008B50B8A1D
:10EBA800032B06D80121044A044865F020FE002002
:10EBB80008BDFFF74DFFFAE7D6850A00B0870900C0
:10EBC80038B50B8A0546032B0C4609D801210F4A94
:10EBD8000F4865F00CFE2046BDE83840F7F7D4BC76
:10EBE800042104F10C0066F070FA4188284668F0A8
:10EBF800E3FB30B9074A0B460548022165F000FEE1
:10EC0800E9E7436821465B699847E4E7F4850A0029
:10EC1800B087090011860A0070B5134A0C461378AC
:10EC28000646013313F0FF010ABF01230B461946BC
:10EC380013701220082268F07EFB054688B108216F
:10EC48000C3066F0F5F922882946028062884280F5
:10EC5800A2888280E288C2803046BDE8704068F0B1
:10EC68009ABB6FF00B0070BDBFD5002023281FD8BA
:10EC78001A2804D8431E182B0ED906207047A0F175
:10EC88001B03082B1ED8DFE803F0051D1B231D19E5
:10EC9800251D05000320704701230F4A83401A40B1
:10ECA800C2B90E4A1A40002A0CBF0620012070473C
:10ECB80000F07F03522B05D10020704701207047D8
:10ECC8000520704710F0400F14BF00200620704741
:10ECD8000420704702207047AAAA8A0254554501A9
:10ECE8002DE9F74F064608460C46F7F7ADFB182303
:10ECF80043432D4F0546FA1891680191E16806F1E2
:10ED08005400D0E8AF0FC0070AD40121274A284889
:10ED180068F07EFB6FF01509484603B0BDE8F08F38
:10ED2800E068007810710022FA500B78D22B0FD1CE
:10ED38003368214618686AF05EF8814640B10121BF
:10ED48001C4A1B4868F064FB2046F7F71DFCE3E704
:10ED5800182303FB0573D4F80C80D4F814B0B4F866
:10ED680010A09E60002321461A46301DFFF77AFD49
:10ED780081460028D0D010F1690F04D101210E4A34
:10ED88000B4868F045FB6269A8EB0B0812FA88F299
:10ED9800E26018225543019B7A19A4F810A09360E9
:10EDA80047F80590B8E700BF6C6700204D860A0059
:10EDB8003087090067860A007A860A0008B5EFF3EB
:10EDC8001181202383F31288BFF36F8F0023036020
:10EDD8000F4B5A68C2B9C3E9000081F31188BFF329
:10EDE8006F8F0C4824F0EEFF031E0CDA01210A4A4B
:10EDF8000A4865F005FD002383F31188BFF36F8F80
:10EE08000323184602DF08BD10605860E5E700BF1D
:10EE180064670020000900209D860A0030870900E9
:10EE2800094B011F9A680948914204BF00229A6061
:10EE38001A6A914204BF00221A629A6B914204BF77
:10EE480000229A636CF0B4BE6C6700202820002072
:10EE58000121024A024868F0DBBA00BFC6860A00F0
:10EE68003087090010B5044600F15003D3E8EF1FBE
:10EE780041F00101C3E8E21F002AF7D1201F68F022
:10EE8800F0FA04F1740004496DF032F92068BDE825
:10EE9800104003F06BBD00BFA9FE000073B50E461D
:10EEA800438D418B01328B4228BF0B469A4205465F
:10EEB80009D9022100921D481D4A65F0ABFC0024C7
:10EEC800204602B070BD3046FFF7D0FE6FF0140345
:10EED800034113F0010310D0F6F7A0FF154B1958A2
:10EEE800154BD3F8E03099421DD0144B1B685A1AC1
:10EEF80018BF4FF0FF32134600E0114A00211148B5
:10EF0800FFF796FC04460028DAD0F7F79DFA182296
:10EF18000D4B012102FB003304F10C009D6066F0EB
:10EF280087F80670CCE70022E5E700BF30870900C4
:10EF3800E3860A000800000090510020B467002012
:10EF48001C4E0E00B02100206C67002070B50446EE
:10EF580001F10C000D4666F0C8F8266801462B8AB8
:10EF6800EA68306869F0E0FC1E2100222046FFF7BD
:10EF780095FF014630B90121044A054868F048FA6E
:10EF8800002070BD204668F05EFAF9E708870A009D
:10EF980030870900F0B51D4603680E46003904465F
:10EFA80018BF012187B01868174669F0CEFC40B930
:10EFB80004F1540068F086FB002846D0002007B012
:10EFC800F0BD002D43D018220021684688F0F0FDDE
:10EFD8006FB1002213212046FFF760FF019030B97E
:10EFE8001C4801211C4A68F013FA1120E7E723683E
:10EFF80029461B68284600930023ADF812300C9B65
:10F00800164A0393BDF834308DF80860ADF8103017
:10F0180001238DF814306B4668F0FCFA9DF8143023
:10F0280063B1002FCAD00198F7F7AEFA2A463146E5
:10F0380020469DF8143068F050FBBFE7019900297D
:10F04800BCD0204668F0FFF9B8E71220B7E70120E6
:10F05800B5E700BF3087090025870A00D374070089
:10F068002DE9F3410B8A04460D4643B90121294A8B
:10F07800294868F0CDF9002002B0BDE8F0810768A2
:10F08800012105F10C0066F020F87B7B0646072B72
:10F09800F1D154F8043C002BEDD0002203781F4F27
:10F0A800043C17F832004FEAC208984207EBC20145
:10F0B80014D12A8A4878904226D90121009316480B
:10F0C8001346174A65F0A6FB04234744BA78012A79
:10F0D800D1D1002BCFD00022317811E001321C2A87
:10F0E800DFD1104A02210C4865F08AFB31780846C6
:10F0F800FFF7BCFD2122C24012F00102BBD106235A
:10F10800204668F0EAFAB6E74B6820462946984751
:10F118000346DAE73E870A00308709006C91090048
:10F1280073870A0059870A00F8B5124A0746002370
:10F1380011480D4665F0EAFE044638B901212B4610
:10F148000E4A0F4865F05CFB2046F8BD00F10C063E
:10F158000921304665F061FF2046F7F775F9182256
:10F16800084B012102FB003330469F6065F060FFC9
:10F178000570E9E71C4E0E00B021002082840A00C9
:10F18800308709006C6700202DE9F0410E8A04469B
:10F19800043EF6B2022E08468CB001D0102E64D17F
:10F1A80004210C3065F091FF0DF1080805884788A7
:10F1B800011D3246404667F0CCF9002857D0A5B368
:10F1C80000268FB3AF4230D34FF42053404601A9F5
:10F1D8008DF80460ADF8063067F08EF948BB14224C
:10F1E800002107A888F0E4FC11212046FFF79CFFC6
:10F1F8000990002837D001210C30CDE9074865F087
:10F2080017FF00230A90394603701A4A0B932846C1
:10F2180007AB68F0FFF9DDE909131B78FBB908466D
:10F22800F7F7B2F90A2301E03D4601232A461021E7
:10F238000EE042F60103404607A98DF81C60ADF8C0
:10F248001E3067F059F90028C9D010232A461946FC
:10F25800204668F042FA00200CB0BDE8F081204654
:10F2680068F0F1F8F7E71120F6E70420F4E70E203C
:10F27800F2E700BFD5F700002DE9FF410368044617
:10F288000D461868012169F060FB40B904F154008B
:10F2980068F018FAA0BB122004B0BDE8F081102273
:10F2A8000021684688F084FC21212046FFF73CFFB6
:10F2B800029038B34FF00108009405F10C072B8A2F
:10F2C800012B04D82046029968F0BDF818E03846AA
:10F2D80065F00BFF6B4601460B4A06468DF80C801D
:10F2E80068F098F99DF80C30002BE8D00298F7F7F1
:10F2F8004BF93246202120469DF80C3068F0EDF994
:10F308000020C9E71120C7E7457907002DE9FF412B
:10F31800036804460D461868012169F016FB40B9D8
:10F3280004F1540068F0CEF9A0BB122004B0BDE887
:10F33800F08110220021684688F03AFC0F2120460F
:10F34800FFF7F2FE029038B34FF00108009405F180
:10F358000C072B8A012B04D82046029968F073F811
:10F3680018E0384665F0C1FE6B4601460B4A064672
:10F378008DF80C8068F04EF99DF80C30002BE8D021
:10F388000298F7F701F932460E2120469DF80C3015
:10F3980068F0A3F90020C9E71120C7E7C979070079
:10F3A800F0B51D46036804460E4685B0012118686D
:10F3B800174669F0CAFA38B904F1540068F082F9BE
:10F3C80050BB122005B0F0BD65B31022002168467D
:10F3D80088F0EEFB39462046FFF7A6FE029018B3E8
:10F3E800BDF828302946ADF80430012328468DF8A9
:10F3F8000C300E4A6B46009468F00CF99DF80C30FE
:10F4080002995BB10846F7F7BFF82A46314620460D
:10F418009DF80C3068F061F90020D3E7204668F0C9
:10F4280012F8F9E70120CDE71120CBE7C9790700E9
:10F438002DE9F0410E8A0446043EF6B2022E084633
:10F448008CB001D0102E76D104210C3065F03DFE31
:10F458000DF1040805884788011D3246404667F0CB
:10F4680078F8002869D085B377B3BD422DD801213B
:10F47800606869F06AFA064678BB42F602038DF8BE
:10F48800000069464046ADF8023067F035F820B311
:10F4980042F60303404606A98DF81860ADF81A3005
:10F4A80067F02AF8C8B1012D03D14FF6FF739F42C8
:10F4B80013D004F1540068F005F9002814BF0020A7
:10F4C80012200CB0BDE8F0813D4601232A460821F0
:10F4D800204668F002F90020F3E7182200210DEB1E
:10F4E800020088F065FB09212046FFF71DFE089001
:10F4F800F8B101210C30CDE9064865F099FD0023EB
:10F50800099003700A2339468DF82C30284606AB3B
:10F518000B4A68F07FF89DF82C3008992BB1084603
:10F52800F7F732F89DF82C30D0E7204667F08BFFCC
:10F53800D1E71120C5E70420C3E70E20C1E700BFCB
:10F548008DF800002DE9F0430F460446062187B0E8
:10F5580007F10C0065F0B9FD0588EDB1B0F802803F
:10F56800B8F1000F17D0454516D8002382888DF8CA
:10F5780000308DF804304FF42053684601A9D7F8BD
:10F588000C90ADF80220ADF8063066F0B5FF0646DF
:10F5980060B10A2301E0454601232A460621204698
:10F5A80068F09BF8002007B0BDE8F08301461422FC
:10F5B80001A83F7C88F0FCFA07212046FFF7B4FD3C
:10F5C8000290D8B10A2341468DF81530284601AB80
:10F5D8000B4ACDE9036901948DF8147068F01AF8A4
:10F5E8009DF8153002992BB10846F6F7CDFF9DF826
:10F5F8001530D2E7204667F026FFD3E71120D2E77F
:10F6080079F600007FB5CB6804461D888DB15E8809
:10F6180076B1B5420DD810220021684688F0C8FAA4
:10F6280005212046FFF780FD019058B9112007E019
:10F63800354601232A460421204668F04EF800206A
:10F6480004B070BD6B4631462846084A009467F0FE
:10F65800E1FFDDE9011323B90846F6F795FF0A2310
:10F66800E8E7204667F0EFFEE9E700BF45750700C9
:10F678002DE9F04342F60103002591B0D2F800804D
:10F6880006460F4600680BA9D8F8049014468DF872
:10F698002C50ADF82E3066F02FFF00286DD04FF4B7
:10F6A800205330680BA98DF82C50ADF82E3066F039
:10F6B80023FF38B1A3681BB15A88BA4200D25F80D1
:10F6C800012010E06168084667F08AFEB8F82A2031
:10F6D800B8F81A309A4294BFC0EB0200C0EB03009E
:10F6E800032803D8002011B0BDE8F083084665F070
:10F6F80056FC05466168084667F072FE6B8A2A8ADE
:10F70800A3EB020C6B69EA68D21AACEB0203B8F8F7
:10F718002AC0B8F81A20944594BFC0EB0C00C0EB7F
:10F728000200834228BF03466BB9887AF6F784FE45
:10F738000022002365F0EAFB05460028D2D00146E6
:10F74800606865F03DFC002300933146D6F80480DC
:10F758001023484602AAC047061E0EDB227CE0683A
:10F76800964227D001460BA866F0F3FE40B9237CE9
:10F77800134A0221134865F043F80023A3609FE76A
:10F78800F2B202A906A866F0E4FE10B90E4A3346A2
:10F79800EFE706A90BA866F0AFFE0028EDD100231D
:10F7A8000421637405F10C0065F042FCA060078039
:10F7B800A36884E7324602A988F002FAEDE700BFA1
:10F7C80092870A0030870900B1870A002DE9FF41B6
:10F7D8004FF000084FF4205305460E46006802A972
:10F7E800144617688DF80880ADF80A3066F084FE74
:10F7F800A0B142F60103286803A98DF80C80ADF882
:10F808000E3066F079FE48B123691BB15A88B242BE
:10F8180000D25E80012004B0BDE8F08161682868EC
:10F8280066F06AFE10B100232361F3E7E368A0687D
:10F838001A786AB1B7F81AC0798D038A8C4594BFD3
:10F84800C3EB0C03C3EB0103934201DA0020E2E7A8
:10F8580004210C3065F0ECFB206106802369294601
:10F868005E80074B0194009338460023A26867F036
:10F87800DCFF0028EADB2069003818BF0120CAE74E
:10F88800FD7507002DE9F3471768054689460068A6
:10F8980051681446D7F804A066F02EFE804600286A
:10F8A8004BD195222946504668F0B0FE0646207591
:10F8B80040B1E3681B780BB184F81480002002B0D3
:10F8C800BDE8F0872946504669F078F810B9082352
:10F8D8002375F3E7A068267565F061FB02210C30FB
:10F8E80065F0A6FB164B2061A0F8009000930194E8
:10F8F800334629463846A26867F097FF002807DA9A
:10F9080010F1FF0F32BF0E204042C0B22075D5E77C
:10F918002369002BD2D0A06867F062FD7B8D7A8BBB
:10F928009A4294BFC0EB0200C0EB0300E3681B7867
:10F93800984294BF00200120C1E70120BFE700BF23
:10F94800F97307002DE9F04182B000AF04468846FC
:10F958000022002339463B4823F010FE0546B0B18B
:10F968006D4688B06A46384BCDE90534032342F822
:10F97800103F00234FF4C2513448F4F715FFAD4649
:10F988006FF00B0630460837BD46BDE8F081F6F744
:10F9980045FA2F4B29461A582E4B38681A602C22E4
:10F9A80088F006F93B6800221C603C680023C4E923
:10F9B8000155C4E909552848391D7D6023F0DEFD4D
:10F9C800064688B123686C4688B06A462349CDE963
:10F9D8000513032342F8103F4FF4C4512B461B482C
:10F9E800F4F7E2FEA546CBE70146B022786888F036
:10F9F800DFF878681A4B83605C306CF0FBF97B6841
:10FA08005433D3E8EF2FC3E8E16F0029F9D17B68BD
:10FA18001C60636A7D681BB904F10C006CF0EAF99C
:10FA2800626A05F1A803C5F8A820A26A636202B950
:10FA3800A36217227B685A855A830433C8F80030BA
:10FA4800A0E700BF0C200020D0870A0030870900FB
:10FA580008000000B467002028200020F5870A006D
:10FA6800D808002008B5437B072B06D002210C4A92
:10FA78000C4867F0CDFC002008BD042167F09CFC11
:10FA880010B9094A0121F3E700F15003D3E8AF3F69
:10FA9800DB0701D4054AF5E750F8040CECE700BF92
:10FAA800A0850A00308709001A880A004D860A00D6
:10FAB8002DE9F04F85B000AFB860EFF3118820232F
:10FAC80083F31288BFF36F8F584C204667F07EFC93
:10FAD8002668054688F31188BFF36F8F00285FD02A
:10FAE800F6F7B2FC182202FB00F35149C81851F886
:10FAF80003A003690021D0E90248FB6090F8049054
:10FB0800B0F806B088F054F8A87AF6F795FC696959
:10FB1800034659B16A7AD00706D45A6A2846126849
:10FB28007B60926890477B6800226A612946184684
:10FB38006CF0B1F9B9F1000F0DD064B1236853B17D
:10FB48001B6843B1BAF1000F2ED001215346394A40
:10FB5800394864F055FE1EB30020B9686CF096FA77
:10FB680000281DDA6C468AB06A46344B0593344B3C
:10FB7800CDE906304FF40073ADF82030314B42F830
:10FB8800103F00234FF411512B48F4F70DFE0023CA
:10FB9800A54683F31188BFF36F8F0323184602DF4E
:10FBA8001437BD46BDE8F08F201D67F039FF484681
:10FBB800FFF75CF80528CED801A353F820F000BF62
:10FBC8000DFC0000E1FB00005FFB00000DFC0000E5
:10FBD8005FFB0000E1FB000004F15403D3E8AF3FF2
:10FBE800DA0705D40121184A134867F011FCB2E777
:10FBF800A36D002BAFD00023144A04F1780024F041
:10FC080089F9A8E754F8543B1D68D4E8AF3FDB07EF
:10FC1800E8D5B8F1000F9ED0002403E02846F96823
:10FC2800C0470134A3B29B45F8D894E76467002025
:10FC38006C67002035880A003087090054880A005C
:10FC48008BB60A00040000014D860A001C4E0E0007
:10FC5800F8B50F461646FFF705FFB0B1446A2046CF
:10FC68001CB150F8A84904B1A83C731C194638B116
:10FC7800428B458DAA4228BF2A469A4207D264B9C8
:10FC880002210A4A0A4864F0BBFD0020F8BD32464A
:10FC98003946BDE8F840FFF701B9D4F8A85005B1D6
:10FCA800A83D20460B462C46E2E700BF6F880A00B5
:10FCB8003087090007B50B4600210246F6F7AEF873
:10FCC80001910E4909580E480068884204D00D4831
:10FCD800D0F8E000884201D10022134601A90A4861
:10FCE80023F04CFC014638B91C22019887F060FFCC
:10FCF800019803B05DF804FB0020FAE70800000053
:10FD0800B4670020905100204420002010B5002244
:10FD1800044600F10803D3E8EF0FC3E8E12F0029F8
:10FD2800F9D108B1F6F730FC2146BDE8104001488A
:10FD38006BF03EBF442000202DE9F743044678309D
:10FD48000F4690461E466CF0E1F9A06D50B90221AD
:10FD5800144A154867F05CFB204603B0BDE8F04341
:10FD680000F086B8114B98424FF0000317D0456851
:10FD78004360A06DD0F81890FFF7C8FF00232068F3
:10FD8800A36567F07EFE3DB12068CDF8009043463C
:10FD98003A4631460068A84703B0BDE8F0831D46DF
:10FDA800ECE700BF8A880A0030870900B86700209E
:10FDB800F7B550F8044C0546002C55D000F1A401C5
:10FDC80004F1240067F065FC2E1F05F15807002296
:10FDD8000023384623F092FD024658BB6B6D2BB1C9
:10FDE80001466FF067033046FFF7A6FF002345F88A
:10FDF800043C05F15003D3E8EF1F21F00101C3E8EB
:10FE0800E21F002AF7D1636A73BB04F10C060022D3
:10FE18000023304623F072FD78B9666886B921461A
:10FE2800124826606BF0C4FE286803B0BDE8F040B5
:10FE380002F0BABEF6F7A8FBC9E7F6F7A5FBE6E7B6
:10FE4800A26833689642636008BFA36077683FB1D1
:10FE5800B3696FF067010093002320681A46B8471A
:10FE68003046FFF753FFD8E703B0F0BD0C20002061
:10FE780010B504460430FFF79BFF1321606867F054
:10FE880070F8034630B1BDE810400121024A03482A
:10FE980064F0B6BC10BD00BFA1880A003087090015
:10FEA800F0B589B0044654F8783D00AF3846196873
:10FEB800FEF714FA6E4688B06A460B4BCDE9053753
:10FEC8004FF40073ADF81C30084B42F8103F002384
:10FED8004FF4E2510648F4F767FC2046B546FFF7B1
:10FEE800C7FF2437BD46F0BDBF880A0003000001E4
:10FEF8003087090070B550F8043C0446061F002BF3
:10FF08003BD039B1436D002B37D01B7CDA0734D591
:10FF180005231CE00568284602F090FD6B7A012B4A
:10FF28002BD0646D4CB3237CDB0726D5E368002B0C
:10FF3800EED030466269617CFEF7B0FF054668B9CD
:10FF4800637C01210D4A0E4864F05AFC0E230022FE
:10FF58003046BDE870401146FFF7EEBEE368D4E9CD
:10FF68000512984718B12846F6F70EFBEEE7294622
:10FF78003046FEF7B5FE0028F5D170BDEB880A00C3
:10FF88003087090038B5836D044623B3164A934277
:10FF980021D0CB68DD78F5B1052D406815D00F2D3F
:10FFA8001AD1437A012B17D8022167F06DF808B1EE
:10FFB800103011D104F178006CF0A8F8A26D137C10
:10FFC80043F001031374002038BD437A032B03D890
:10FFD800064AD15CE9E70E2500222B461146204649
:10FFE800FFF7AAFEEFE700BFB867002087B60A0050
:08FFF80010B50C4608B301B37B
:020000021000EC
:10000000FFF734FDE8B1436A3BB153F8A82902B1C8
:10001000A83A996D8C4206D062B90430214667F047
:100020003CFB204602E02046064A9A65BDE81040A7
:10003000FFF770BED2F8A81001B1A83913460A46DE
:10004000E7E710BDB8670020F8B51D460F46164615
:10005000F6F7FEF91823044C03FB00400123C0E926
:100060000376C3800575F8BD6C67002008B586F07F
:10007000D4FD38B101210346034A044867F066FE07
:100080006FF0040008BD00BF12890A0088870900CC
:1000900010B51846144607491022A047041E07DA77
:1000A00001212346044A054867F050FE204610BD52
:1000B0000024FBE72837002028890A0088870900E8
:1000C000F8B506460F460024094D15F8013CB34229
:1000D00007D12946384667F08FFE10B10548204405
:1000E000F8BD1034802C05F11005EED10020F7E7A3
:1000F0004D6800204C680020F8B506460F460024E5
:10010000094D15F8013CB34204D12946384667F041
:1001100073FE30B90C34602C05F10C05F1D10020D0
:10012000F8BD02482044FBE78936002088360020CD
:10013000F8B506460F460024094D15F8013CB342B8
:1001400007D13946284667F057FE10B105482044CC
:10015000F8BD0C34602C05F10C05EED10020F7E75A
:1001600037D1002036D1002038B50C4619466BB186
:1001700003F114055B698AB9E268A360954200D176
:10018000E36000230D681A464B61A847A3685BB97A
:10019000601C0649BDE8384067F066BE1360E3683E
:1001A0009D4208BFE260ECE738BD00BFAEB50A0073
:1001B00070B5204B144682689A420FD1A568C66874
:1001C00075B922793046216867F01EFE024628B1D3
:1001D0001949013067F048FE15701581012070BD86
:1001E000E0680028FBD02B888B420AD0F6D2E0686A
:1001F000A36801380433E060003818BF0120A36011
:10020000EDE7256822792946304667F0FDFD024674
:1002100060B93046084967F0F7FD02460028E6D08D
:100220002946013067F020FE23791370A3685B88AC
:100230001381DCE7C1060100AEB50A00102110B53C
:100240000648F9F757FB034630B1BDE810400121DD
:10025000034A044867F07ABD10BD00BF183700207C
:1002600049890A0088870900F8B5054600260B4C25
:100270002746621C65B91046094967F0BDFD28B9DB
:100280000136082E04F11004F2D100273846F8BDDB
:100290002846217866F05DFFF1E700BF4C6800203A
:1002A000AEB50A00F8B506464C1C01F13305671ED1
:1002B00066B12246304614F8011C66F04AFF18B9B0
:1002C0000A34AC42F3D100273846F8BD2046024933
:1002D00067F092FDF3E700BFAEB50A00F8B505463A
:1002E00000260B4C2746621C65B91046094967F089
:1002F00083FD28B90136082E04F11004F2D100273D
:100300003846F8BD2846217866F023FFF1E700BFA4
:10031000E0680020AEB50A002DE9F04106460F4620
:10032000904666F046FA50B339463046FFF7E4FE91
:10033000054678B90446134A104667F004FDC0B973
:100340000C225443104A601C3946104467F08CFD5F
:10035000A5181655012105F1080001FA08F167F00A
:100360006DFDBDE8F04147F612220023074823F057
:10037000D5BD0134082C02F10C02DDD1EAE7BDE85D
:10038000F08100BF9036002088360020E83600203B
:100390000246014610B5042311F8010B0832F9F7A3
:1003A00067FA034630B1BDE810400121024A034814
:1003B00067F0CCBC10BD00BF6F890A0088870900B8
:1003C000022110B5094867F039FD084007D10849F6
:1003D000084A0B88084CA24202D300B10B8010BD22
:1003E0005068083203449BB20120F4E7CC68002037
:1003F00096D10020188709002887090008B5012137
:10040000024A034867F083FD002008BD8B890A007B
:100410008887090038B514460E4B82680D469A420B
:1004200015D122792168C06867F0EEFC78B1D4F864
:10043000C8302F2B03D9FFF7E1FF002038BD04EBB4
:1004400083021581018901335181C4F8C83001202C
:10045000F4E700BFC106010008B50121034A0448C2
:1004600067F055FD6FF0150008BD00BFDF890A0079
:100470008887090070B50B4B164682689A420ED1E8
:10048000C5686C1C33352046316867F0B5FC18B17F
:100490002046716867F0E8FC0A34AC42F3D10120D1
:1004A00070BD00BFC106010008B513468168074A48
:1004B000914209D11A791968C06867F0A5FC18B192
:1004C0000023036043600381012008BDC1060100D1
:1004D00040F239120023014823F020BDB03700203C
:1004E00008B50421084867F0A9FC6FF0020106482E
:1004F00067F0AFFC044867F026FCC30701D5FFF79F
:10050000E7FF002008BD00BFE0370020024608B525
:100510000749013067F0A8FC00230C3202F8043CC4
:10052000D2E8EF1FC2E8E03F0028F9D108BD00BFC4
:10053000AEB50A002DE9F04385B00E4690469946C7
:10054000044600AF58B90121344A354867F0DFFC52
:100550006FF0150528461437BD46BDE8F08307F156
:10056000080165F0A7FF0546A0B16D4688B06A4650
:100570002C4BCDE905344FF40073ADF81C302A4BF9
:1005800042F8103F00234FF4E2512548F4F710F9E8
:10059000AD46DDE72046391D64F051FB786858B15F
:1005A0000A2229465EF04AFD034628B101211F4A6E
:1005B0001B4867F0CBFBCBE7002007F10801FFF7F2
:1005C000B7FD044620BB002EC4D01949FFF7B0FD8B
:1005D000044638B90121174A114867F098FC6FF0BA
:1005E0000B05B7E7002307F1080100F8013B67F0AE
:1005F0003BFC04F1080104224846C047041EA9DA66
:10060000012123460C4A064867F0A0FB2546A1E7D6
:10061000002EEED10660466086609BE781700A007E
:1006200088870900EB890A0003000001078A0A0095
:10063000AEB50A00228A0A0028890A002DE9F0478F
:1006400006460D461D48002190461F469DF820A0F5
:10065000DDF82490FFF732FB044688B1456080F84E
:1006600011A0C0F81490C760C0F818804A465146DF
:100670003046FFF7F1FA054638B92046FFF74AFB46
:100680006FF00B052846BDE8F087002201231146D4
:10069000FFF7DAFC2846A56042464946B8470546BA
:1006A00018B12046FFF736FBECE72146304667F0ED
:1006B000C2FA05460028E5D0F3E700BF1C4E0E0045
:1006C0002DE9F0471F46BDF8203006468846D1F890
:1006D0000C90002B4ED17B1E012B4ED8012F49468A
:1006E0000CBF15781588FFF7DDFD0446B8B915B9BC
:1006F0003846BDE8F0874946FFF7D4FD044638B9CF
:100700001F4802211F4A67F002FC6FF01000F0E75B
:1007100006F17001013067F0A7FB337A2370D9F836
:100720003830DBB9B4F808A02581B9F83230AB42D3
:1007300003D04946404667F0ECFBAA4505D00022AD
:10074000307A06F17001FFF7E7FD002DD0D10E4998
:10075000601C67F089FB25702581C9E72A46414660
:10076000304698470028C4DB01380128DAD96FF0F9
:100770000D00BEE76FF00600BBE76FF00C00B8E7B6
:1007800088870900448A0A00AEB50A002DE9F041C5
:1007900080460F4616461D46FFF7CAFC044680B940
:1007A0001749FFF7C5FC044630B9BDE8F041012107
:1007B000144A154867F0ABBB394600F8018B67F067
:1007C00053FB238973B9628972B9268165812146F9
:1007D00011F8010B65F0EDFF80B12046BDE8F04156
:1007E000FFF7D6BD9E4204D36289AA4206D29E423A
:1007F000ECD263892681AB42E9D2E7E7BDE8F0811C
:10080000AEB50A005E8A0A008887090010B5FFF7B6
:100810008FFC044678B1014611F8010BF9F736F860
:10082000034620B10121044A044867F08FFA0023EF
:1008300023606360A36010BD7D8A0A008887090079
:100840002DE9F047284B1646826807469A422DD17B
:10085000C5686B8E53B34FF000086C1C05F1330A6A
:1008600006F17009B4F807309BB12246304614F8FF
:10087000011C66F06EFCE0B9214614F8010CFDF78E
:1008800077FC30B1437B072B08BF48F00108FCF729
:10089000E5FF0A345445E5D1B8F1000F06D16B6B82
:1008A000A5F8328013B14146384698470120BDE88B
:1008B000F0874946307A65F07CFF78B90B4B9D4252
:1008C00002D1304667F042FD2046094967F0CCFA74
:1008D000002304F8013CA4F80730DAE74946204633
:1008E00067F0C2FAD5E700BFC10601003809002051
:1008F000AEB50A0073B50C460546082104F1100098
:10090000164667F09BFA122304223146CDE90032E5
:1009100028462246024BFFF791FE02B070BD00BF91
:100920009983070038B505460C460F48012167F04A
:1009300085FA10F0010F0D4B0AD11D835C830A4824
:1009400067F001FA830709D4BDE83840FFF7C0BD5E
:10095000198B5A8BA94202D89442EFD838BD9442E1
:100960001D83ECD9EAE700BFE03700209037002074
:100970002DE9F0419846BDF818300646012B174680
:1009800036D84344012B454635DCFFF76DFC044661
:1009900068B9FFF769FC044648B90221194A1A48A8
:1009A00067F0B5FA6FF010052846BDE8F081B8F1A0
:1009B000000F11D00023217A21FA03F2D00703D5CA
:1009C0003A78DA40D20719D50133032BF4D13B78BA
:1009D00003F007031943217206F17001601C67F0F0
:1009E00043FA337A01212046237067F0FAFCDBE7F3
:1009F0006FF00605D8E76FF00C05D5E76FF012052C
:100A0000D2E700BF9A8A0A008887090010B56FF004
:100A1000020104460E4867F01CFA0D4867F093F98E
:100A2000C20704D5002200230A4823F077FA2046A3
:100A300067F037F958B12046FFF716FC38B1037A52
:100A4000DB0704D5BDE81040012167F0CABC10BD2A
:100A5000E0370020B037002070B56FF0080117486C
:100A600067F0F7F940F2391200231548F8F7A2FDB4
:100A70000026144C651C2846134967F0BDF9B0B92F
:100A8000237ADB0713D52946FDF772FB054620B113
:100A900067F009F92846FCF7E1FE6FF0020104F166
:100AA0000C0067F0D6F90021204667F09AFC013669
:100AB000082E04F11004DDD170BD00BFE037002026
:100AC000383700204C680020AEB50A002DE9F0430D
:100AD00085B0894616469846044600AF58B90121AC
:100AE000414A424867F013FA6FF01505284614375B
:100AF000BD46BDE8F08307F1080165F0DBFC054663
:100B0000A0B16D4688B06A46394BCDE905344FF443
:100B10000073ADF81C30374B42F8103F00234FF400
:100B2000E2513248F3F744FEAD46DDE72046391D79
:100B300064F085F8786858B10A2229465EF07EFA9A
:100B4000034628B101212C4A284867F0FFF8CBE77B
:100B5000002007F10801FFF7B3FA044690B9FFF748
:100B600083FB044638B90121244A204867F0CFF9B5
:100B70006FF00B05BAE7002307F1080100F8013B0D
:100B800067F072F9B9F1000F2AD0022239464046C7
:100B9000B047061E07DA01213346194A134867F0A9
:100BA000D5F83546A2E73B78022E237209D0022100
:100BB000144A0E4867F0ABF90021204667F011FC9B
:100BC00094E77B78012B05D90F4A3146074867F037
:100BD000BDF8F1E7204603F0010167F0F2FB85E77D
:100BE0002046FFF793FC81E781700A00888709009F
:100BF000EB890A0003000001078A0A00C68A0A007E
:100C000028890A00E88A0A003C8B0A0037B50446A6
:100C10000D46FFF755FA0246D0B1037A0C308DF835
:100C2000043067F090F810F0010318BF01238DF82D
:100C30000530022301AA29462046F8F72FFE034675
:100C400020B10121034A044867F080F803B030BDA9
:100C50000346F0E78D8B0A008887090070B50025F0
:100C60000A4C661C0A49304667F0C6F8014630B99E
:100C7000204667F0A6FB31462078FFF7C7FF013515
:100C8000082D04F11004ECD170BD00BF4C680020A9
:100C9000AEB50A0008B50121114867F0CFF8C307C7
:100CA0001CD4FFF78DFB0F490F486BF025FA00238A
:100CB00040F239120C48F8F777FC0C490C486BF0FD
:100CC0001BFA02210B4867F0B9F80B480B496BF08F
:100CD00013FABDE808400A48FDF714BD08BD00BF7F
:100CE000CC6800201585070038370020C91801009E
:100CF000B0370020E0370020E8360020A585070047
:100D00001009002003462DE9F04148B1008A38B9A6
:100D100001244FF0140C1149DFF844E0714501D370
:100D2000BDE8F081D1E90076BB4204D30CFB06722A
:100D3000143A93420ED93444A2B214460831EDE776
:100D40000CFB0578434507D001356219AE4292B2DB
:100D5000F6D1F2E70025F8E71046E1E71887090029
:100D6000288709002DE9F74F99464FF6FF73BDF824
:100D700030400746002C08BF1C46444B90461B8859
:100D80000091834252D2424B1D68002D43D04FF058
:100D9000140B083DAE682EB156F8083C1B8ABB42C6
:100DA00003D900266B689E4243D3AD68002D32D034
:100DB000083DEFE773682B44BB4234D29DB208363E
:100DC000344B9E42F6D3DEE74046D15865F098FB9F
:100DD000A0B101350AF1010AADB273685345EED9ED
:100DE000009B9D4217D8BD42F3D3142303FB0AF3A3
:100DF000326802EB030BB8F1000FE5D1B9F1000F37
:100E00000CD1013CA4B2294658460E9A0D9B984736
:100E10000CB10028DDD103B0BDE8F08FDBF80C3059
:100E20009945D6D1EDE74FF0000AD6E701251A4ED5
:100E3000C6E70BFB06F22968009801EB020ABAF834
:100E400010309842E7D39F4218D8B8F1000F0DD167
:100E5000B9F1000F14D1013C1946A4B250460E9AC4
:100E60000D9B9847002CD6D040B9D4E7404689580E
:100E7000019365F045FB019B0028E9D0013691E71D
:100E8000DAF80C209145F9D1E5E700BF96D10020B2
:100E9000D0680020288709001887090010B59EB087
:100EA00010220021684686F087FE142200210DEBF7
:100EB000020086F081FE4FF41053ADF8103080230D
:100EC0001022ADF812304FF48063284C6946CDE90A
:100ED00006340DEB02001CAB85F02EFD034630B14D
:100EE000234A0121234866F031FF1EB010BD0146A0
:100EF00048220AA886F060FE22461C990AA885F0BE
:100F000089FE034660B101211B4A1A4866F01EFFA4
:100F10001C9885F047FC03460028E6D0174AE0E716
:100F20004FF6FF710120164A0AAB67F0E8FA10226B
:100F3000144904AB0AA885F08BFE04461C9885F082
:100F400031FC14B1104A2346CBE708220D4B03F1C4
:100F50001001187811F8014D013A03F8014B08709F
:100F6000F7D10821094866F069FFBEE70002C00317
:100F7000B68B0A0088870900DF8B0A00FD8B0A0008
:100F8000517D070018370020138C0A00E03700203D
:100F90002DE9F04118490446A1F1300015461E46DE
:100FA000BDF818706BF0CDF8144866F0CCFE010760
:100FB00005D4FFF773FFFFF751FEFFF73FF9204617
:100FC000FFF752F968B1037ADA070AD500F10C0489
:100FD000204666F0B8FEC30703D40221204666F01F
:100FE0002DFF10233A46069331462846BDE8F041CE
:100FF000034B67F0E8B800BF68370020E0370020F7
:101000001837002010B51B4866F09DFEC0F3C000E5
:1010100080F0010408B9FFF741FF164866F093FE1F
:101020000346144866F08FFEDA0622D5830606D5FD
:10103000FCB1FFF713FEBDE81040FFF7FFB8202119
:101040000C4866F0FBFE10220B49881886F0BCFDA8
:1010500048B90A486BF05EF8BDE810406FF0010136
:10106000044866F0F6BE4FF6FF710120FFF75AFC08
:10107000DFE710BDE037002018370020B037002030
:1010800008B51021034866F0D9FEFFF7BBFF00202A
:1010900008BD00BFE03700202DE9F3470446624851
:1010A00066F051FEC10713D4FFF78AF923680025C3
:1010B00018684FF4C05369468DF80050ADF80230FF
:1010C00065F01EFA60B96FF0770002B0BDE8F087F6
:1010D000564866F038FE4207E6D46FF01500F4E794
:1010E000236801A9186841F601038DF80450ADF892
:1010F000063065F005FA0028E5D04D4D23F0BAFA28
:101100002B6826689BB9002E65D1002204F10803E4
:10111000A2606A68002A68D1C5E90033424866F0D7
:1011200012FEC30771D423F0B9FA0020CDE76B6833
:10113000002B77D053E90232142101FB023333F83C
:10114000047C002E4FD1002FDFD023681E8ABE42C0
:10115000DBD829680029E1D00022A1F10803186832
:10116000008AB0424AD904F10803002A40D09168AD
:10117000A1600029CDD09360D0E7F37C318A23F0C1
:101180008003F37489B9791CDBB289B243F0800320
:101190003182F3740F4609F1FF3914361FFA89F9C9
:1011A000B9F1000FE9D14746CDE78F42F2D301AB49
:1011B0000846204ACDF804A067F0A1F9019B43B18D
:1011C000338A01211C4A1D4866F0C0FD23F066FAEF
:1011D00083E73946DEE79846194A17884FF0000A38
:1011E000B4F80490DCE7B846F8E713606B6095E765
:1011F0006A68A1602B60002A90D1F7E79868002800
:101200008CD01A46A0F10803A9E71421D4E90023E1
:1012100001FB0323108A33F8041CFFF783FBFFF75D
:101220001BFC80E71B68FFDECC680020E037002055
:10123000D0680020E77C0700298C0A008887090015
:1012400096D100202DE9F04FB9B000AF0C46904682
:1012500038493A46D7F80801994663F0CCFC40B9C2
:10126000FFF7FAF86FF015052846E437BD46BDE8EC
:10127000F08F3E68391D304663F0E1FC3EB9012134
:101280002D4A2E4866F043FE6FF015043FE0786863
:1012900000BB4FF0000B07F1080A5146304687F8B3
:1012A00014B065F007F9054608B36C4688B06A4685
:1012B000234BCDE905364FF40073ADF81C30214BBC
:1012C00042F8103F4FF4E2515B461C48F3F770FAC6
:1012D000A546D9E70A2200215DF0B0FE03460028AA
:1012E000D7D00121184A154866F030FDCCE7C7F881
:1012F00010A0E4B1C022484607F12001C047041EF7
:1013000007DA01212346114A0C4866F01FFD2546E5
:10131000AAE7A40807F12003C7E906344FF6FF71D6
:1013200001200B4A07F1100367F0E9F89CE7234618
:10133000F2E700BF4A8C0A0081700A008887090022
:10134000EB890A0003000001078A0A0028890A00C5
:10135000B1010100002330B5B5B001918DF808004E
:101360003393044601AB0D4601204FF6FF710B4A43
:1013700067F0C5F8339B73B19B0003AA294620464A
:10138000F8F7A2FA034620B10121054A054866F0A4
:10139000DDFC35B030BD1A46F0E700BF1504010092
:1013A000518C0A00888709002DE9F34100F170088B
:1013B000CDE9001204460F46007A4146154665F015
:1013C000F8F906466B464FF6FF710120214A67F097
:1013D00096F81EB14146207AFFF7BCFF3946207AC5
:1013E000FEF76EFE40B12946013066F03DFD1EB1AC
:1013F0004146207AFFF70AFC94F8088039464046B7
:10140000FEF796FE0446C8B129464046FEF790FE18
:10141000C8B1844217D02289638952EA030106D0F9
:101420000589418995420CD8994200D24381002315
:1014300023606360A3600EB1FEF7AAFF02B0BDE8AF
:10144000F0810281F0E7601C294666F00DFD204620
:10145000F1E700BF7504010014212DE9F04F0646A5
:10146000036885B01A8A0192426801FB023333F89F
:10147000043C029323F0FEF83C4806F1080166F0B4
:101480004AFF8046002866D123F008F96FF001007A
:1014900005B0BDE8F08F1422336802FB0535344AED
:1014A000AB6893423BD14FF0000AEB68A3F832A03F
:1014B0005C1C03F1330B20462E4966F09DFC074669
:1014C00050BB214614F8010CFCF752FE034658B9F4
:1014D000214614F8010C65F06CF9A8B1214614F806
:1014E000010CFFF737FF0FE0427B072A31D100F1F3
:1014F00070013A46007A0393FEF70EFF039B1846ED
:10150000FCF7ACF9002FE3D120461A4966F0ACFC99
:1015100004F801ACA4F807A00A345C45CBD195F9D6
:101520001330002B05DA2B6923F000431B0C1B043E
:101530002B6109F1010973681FFA89F5AB42AAD83A
:101540000D4866F000FCC30708D423F0A7F800207C
:101550009EE74746D3E74FF00009ECE7DDE90101DC
:10156000FFF7E0F9FFF778FAEFE700BFD068002057
:10157000C1060100AEB50A00CC680020002307B503
:101580000193FFF7BFFB411C89B20846034A01AB38
:1015900066F0B5FF019803B05DF804FBDB8207003D
:1015A0002DE9F04387B0437B8046072B0C46154658
:1015B00002AF40F0A68000233B7342F6030320688D
:1015C00007F10C01FB8164F09BFF0646002834D133
:1015D000D4F80490B9F1000F05D101214B4A4C48D1
:1015E00066F095FC8DE001232146009007F108028A
:1015F000C847031E11DA6D4688B002AAD3610423DE
:101600004449C2E9051442F8103F4FF401513346F2
:101610003F48F3F7CDF8AD4673E0012B05D001212B
:101620003D4A3B4866F092FB6BE03B7A13F0300F8B
:1016300067D02046FFF7A2FF0446002320683B73D3
:1016400042F6021307F10C01FB8164F059FF18B157
:101650002046FFF793FF0446002642F60219206851
:1016600039463E70A7F8029064F04AFF18BB002389
:1016700020683B7342F6021307F10C01FB8164F012
:101680003FFF064600283CD1D4F80490B9F1000F82
:10169000A3D0022300902146404607F10C02C84720
:1016A000031EA8DB022BBAD1BB8905EA0300003870
:1016B00018BF012026E042F603032068391D3E7161
:1016C000FB8064F01DFF0028D1D04FF42053206828
:1016D00007F108013E727B8164F012FF0028C6D03A
:1016E00042F60103206807F10C013E73FB8164F0B0
:1016F00007FF0028BBD02046FFF740FF0446002824
:10170000ADD100201437BD46BDE8F0836F8C0A00D0
:1017100088870900838C0A00A98C0A002DE9F84308
:101720001546894694226968064666F073FF80462E
:10173000002841D1022230466968FFF731FF0028B6
:101740003DD000211F48AF8AFEF7B8FA02370446A1
:1017500080B11D211C4B47613A464174C0F80C8092
:10176000436085613046FEF777FA074638B9204670
:10177000FEF7D0FA6FF00B052846BDE8F883012389
:1017800042464146FEF760FCA98A07F10C0002318F
:1017900063F052FC20F8029BAA8A296986F0E6F9D8
:1017A00021463046A76066F046FA05460028E3D099
:1017B0002046FEF7AFFADFE74FF0FF35DCE76FF0CA
:1017C0001505D9E71C4E0E00ED7C070070B50546E7
:1017D0008AB03A4866F0B7FA42070C4667D515B1A9
:1017E0006B7B072B66D1666830460596FFF78AFA51
:1017F0002268ADF81800002A2FD005A902913049BF
:1018000000230191012100914FF6FF710593FFF72D
:10181000A9FA059E1EB96FF001000AB070BD66609E
:10182000002330688DF8103042F6030304A9ADF8A8
:10183000123064F065FE40B90598C3689B799B0639
:1018400008D566F015FEADF81800059866F0B7FEED
:10185000606028B96FF01500DFE70028E0D1DAE713
:10186000BDF818003DB10123014622462846A37564
:10187000FFF754FFD1E76FF07F0307930223ADF822
:10188000203042F60213ADF8123005ABA575029375
:101890000C4B4FF6FF710193012304AA00932B46D2
:1018A00009948DF81050FFF75DFA0798B5E76FF0CF
:1018B0000A00B2E76FF07F00AFE700BF0802002028
:1018C0001B7D0700391B010073B5044650F8083C26
:1018D00000F130056FF00101A0F1200628460193C8
:1018E00066F0B7FA0D4B002044F81C3C0C4B314617
:1018F00044F8183C01AB44F8103C042324F8080CCD
:1019000024F8060C24F80C3CFFF760FF18B90221FC
:10191000284666F093FA02B070BD00BF88920900B5
:101920000D0A01002DE9F84F90463D4B82680546AF
:101930009A4200AF70D1D0F80C90D8F8004009F16D
:10194000010609F1330AB6F80730F3B132462046F2
:1019500016F8011C65F0FDFBB8B14FF495722946ED
:10196000204666F057FE30B3032812D1EB4688B00C
:101970006A462C4BCDE9053542F8100F00234FF491
:10198000C4512948F2F714FFDD460A365645DAD12C
:1019900042E0052820460CBF4FF0030B4FF0020B2E
:1019A00065F0A7FB834506D998F804305B45ECD277
:1019B00088F804B0E9E74946284666F0AAFA1B4BC6
:1019C000994529D1207A04F17001FEF7B1FB054653
:1019D00010B303890BB94389F3B12046FCF7D8F85B
:1019E0002A89134B134923F820206A8903EB8003CB
:1019F0005A80182202FB00110B6104230E4A204674
:101A00004A600E4A8B828A60FFF7E0FE20B1012116
:101A10000B4A054866F07BFA0120BD46BDE8F88F09
:101A2000C1060100C28C0A0088870900380900201D
:101A300022D10020D467002088920900FF8307008C
:101A4000D68C0A0070B504468AB0384866F07BF937
:101A500042070D4663D514B1637B072B62D16E68D4
:101A600030460596FFF74EF92A68ADF81800002AAF
:101A70002FD005A902912E49002301910121009147
:101A80004FF6FF710593FFF76DF9059E1EB96FF0D4
:101A900001000AB070BD6E60002330688DF8103010
:101AA00042F6030304A9ADF8123064F029FD40B9F1
:101AB0000598C3689B79DB0608D566F0D9FCADF8BC
:101AC0001800059866F07BFD686028B96FF0150076
:101AD000DFE70028E0D1DAE7BDF818002CB10146B5
:101AE0002A46204666F0D1FDD3E76FF07F0342F629
:101AF000021207930123ADF8122005AA02920D4AA3
:101B0000ADF82030CDE900324FF6FF71234604AA2C
:101B100009958DF81040FFF725F90798B9E76FF0A0
:101B20000A00B6E76FF07F00B3E700BF08020020AD
:101B30001B7D0700391B01002DE9F84F14463F4B70
:101B4000826880469A4238D1D0F80C903C4B994537
:101B50001BD100263B4D28463B4966F04DF978B92C
:101B60000722294615F8010CFCF78EFB40BB2369C0
:101B700029461A6915F8010C53881288FEF706FEEB
:101B80000136082E05F10C05E5D109F1010709F12F
:101B9000330AB7F80720A3899A420BD1394617F8C0
:101BA000010CFCF7E5FA064620B1437B072B0AD06F
:101BB000FBF754FE0A375745EBD14FF0010B2AE0F3
:101BC000FBF74CFEDCE7D9F83C3023B1414698479F
:101BD00008B93046ECE794224146304666F01AFDDB
:101BE00083460028F5D1A389022B17D1B7F8073017
:101BF0009A0720D530462269A188FFF78FFD054658
:101C000018B92269937D013393753046FBF726FEA0
:101C1000002DA560CEDA5846BDE8F88F012B0AD119
:101C2000B7F80730DB0706D530462269A18866F091
:101C30002CFD0546E9E75D46E7E700BFC106010068
:101C40003809002037D10020AEB50A0073B5437BB8
:101C50000446072B0D461AD1061D4FF4803130463D
:101C600066F0ECF8C30315D402232046CDE9003317
:101C70002A460A4B0A49FEF7E1FC044620B16FF4FC
:101C80008031304666F0E5F8204602B070BD6FF056
:101C90007F04F9E76FF07704F6E700BF5D7F070088
:101CA000237D070070B5437B0546072B0C4686B0A5
:101CB00040F0A1800B7C062B10D8DFE803F0040471
:101CC0005A5A629528000B68CBB11B784BB1022B96
:101CD00013D00121494A4A4866F038F86FF01500E0
:101CE00009E0082301930623224600934549464B09
:101CF0002846FEF7A3FC06B070BD1623F2E71023BA
:101D000004212246CDE90031404B4149F0E7086803
:101D10000028E3D00678002EE0D14FF4245302A926
:101D20008DF80860ADF80A3064F0EAFB08B342F6BB
:101D30000213206803A98DF80C60ADF80E3064F032
:101D4000DFFBB0B142F60313206804A98DF81060E0
:101D5000ADF8123064F0D4FB58B142F60413206899
:101D600005A98DF81460ADF8163064F0C9FB0028A1
:101D7000B4D1082304222749CDE900322246264B5C
:101D8000B6E7086880B300264FF4205302A98DF807
:101D90000860ADF80A3064F0B3FB00289ED042F62C
:101DA0000103206803A98DF80C60ADF80E3064F0D3
:101DB000A7FB002892D042F60203206804A98DF800
:101DC0001060ADF8123064F09BFB002886D042F61C
:101DD0000303206805A98DF81460ADF8163064F08F
:101DE0008FFB00283FF47AAF04232246CDE900336D
:101DF0000A490B4B7CE76FF07F007CE7F38C0A000D
:101E000088870900358707008F820700F17F070068
:101E1000251E0100491F010021800700C122010089
:101E2000897F07002DE9F0478EB0064617461C460D
:101E3000169D31B12A4600216B680EB0BDE8F0470F
:101E4000184763B902213D4A3D4866F060F82A46CA
:101E5000002130466B6898470EB0BDE8F0871378D4
:101E6000062B08D0142B05D00121364A344865F0E2
:101E70006DFFECE702214FF00008C146013C8DF8F0
:101E80001010A4B207F1010A9C420CD2002CDED142
:101E9000B8F1000FDBD02A46414630460EB0BDE80F
:101EA000F04766F029BC1422002109A885F084FEC1
:101EB000BAF8002093B2002BC9D0BAF802101FFA6A
:101EC00081F8B8F1000FC2D04345C0D89DF810305A
:101ED00013B3022B25D02B7CADF80C10002B42F64F
:101EE000010308BF4FF42053ADF8063004AB029352
:101EF00001AB099302ABADF834200C932A4630466F
:101F00006B688DF8049009A998470028A4D03B7805
:101F1000E41AA4B29A44B7E7BAF80430ADF8123024
:101F2000D9E70AF104030DF111000AF1140C53F87A
:101F300004EB634540F804EBF9D1CCE7088D0A00C7
:101F400088870900128D0A002DE9F04F93B01746DB
:101F500080461C460A461C9D31B12A4600216B680A
:101F600013B0BDE8F04F1847297C022940F0838068
:101F70004BB99B4A9B4865F0CAFF2A460021404660
:101F80006B6898475BE03B78062B08D0082B05D0A0
:101F90000121954A934865F0D9FEEEE711460026E7
:101FA00042F6020A013C8DF82010A4B207F1010BA1
:101FB0009C420BD2002CE0D1002EDED02A463146C6
:101FC000404613B0BDE8F04F66F096BBBBF80090FA
:101FD0001FFA89F6002ED0D0BBF802009DF8202011
:101FE000ADF81C00BBF80410ADF81E1062B1022A57
:101FF00015D0296831B308A864F082FA10B33B7891
